:100000000C947A130C94A4130C94A4130C94A413BE
:100010000C94A4130C94A4130C94A4130C94A41384
:100020000C94A4130C94A4130C94A4130C94A41374
:100030000C94A4130C9486250C94A4130C94A41370
:100040000C94A4130C9465230C943FC20C94A41339
:100050000C94427E0C94387E0C94A4130C94A4133C
:100060000C94A4130C94A4130C94A4130C94A41334
:100070000C94A4130C94A4130C94A4130C94A41324
:100080000C9492790C94A4130C94A4134E414E49F1
:100090004E495459494E46CDCCCC3D0AD7233C1746
:1000A000B7D13877CC2B329595E6241FB14F0A0093
:1000B0000020410000C84200401C4620BCBE4CCA83
:1000C0001B0E5AAEC59D7400407A10F35A00A07200
:1000D0004E18090010A5D4E80000E8764817000083
:1000E000E40B54020000CA9A3B000000E1F5050051
:1000F0000080969800000040420F000000A086019A
:10010000000000102700000000E803000000006469
:1001100000000000000A00000000000100000000D4
:10012000002C76D888DC674F0823DFC1DFAE59E1A9
:10013000B1B796E5E3E453C63AE651997696E8E618
:10014000C28426EB898C9B62ED407C6FFCEFBC9CEB
:100150009F40F2BAA56FA5F490055A2AF75C936BFD
:100160006CF9676DC11BFCE0E40D47FEF520E6B5B8
:1001700000D0ED902E0300943577050080841E0892
:100180000000204E0A000000C80C333333330F98B0
:100190006E12831141EF8D2114893BE65516CFFE77
:1001A000E6DB18D1844B381BF77C1D901DA4BBE403
:1001B00024203284725E228100C9F124ECA1E53D45
:1001C0002741425300504C410042656400456E6334
:1001D0006C6F73757265002568753A2530326875E5
:1001E0000025303268753A253032687500202020AD
:1001F000202020200020202020003FFFF038007029
:1002000030FC3020FC102078102030102C00D02E34
:1002100031D02F7BD02F7BD02E31D02C00D020306E
:100220001020781020FC1030FC303800703FFFF0B8
:100230003FFFF03800703186302387102787902FDA
:1002400087D02F03D0203010207810207810203055
:10025000102F03D02F87D027879023871031863027
:100260003800703FFFF0041040020820020820040C
:100270001040082080104100104100082080041028
:10028000400000001FFFF81FFFF863616E63656C9C
:10029000005072696E742041626F72746564004D23
:1002A00032350050617573696E672E2E2E007265AF
:1002B00073756D65004D32340050726F6265205A5F
:1002C000204F66667365740046696C2E2044696130
:1002D0002E004F6666004F6E004520696E206D6DE2
:1002E0005E3300452073746570732F6D6D005A2066
:1002F00053746570732F6D6D00592053746570735E
:100300002F6D6D00582053746570732F6D6D004113
:100310006476616E6365642053657474696E677397
:100320000046696C616D656E740053746570732F5F
:100330006D6D00436F6E66696775726174696F6E8B
:100340000053746F77004465706C6F790053572DBC
:100350004D6F64650053656C662D5465737400526F
:100360006573657400436F6E666967757261746961
:100370006F6E00526573746F7265204465666175B7
:100380006C7473004C6F61642053657474696E679C
:10039000730053746F72652053657474696E67736C
:1003A00000424C546F7563680050726F6265205A4A
:1003B000204F666673657400416476616E636564A0
:1003C0002053657474696E6773004D61696E004DEA
:1003D0003139305335350A4732380A4732390A4DF8
:1003E0003430300A4D313034533231350A473238E7
:1003F0000A4D313039533231350A4D3432305331B0
:100400000A4731583130305931303046353030308C
:100410000A47315A300A4D3530300A4D31313720D4
:10042000536574205A204F6666736574004D3130F1
:1004300036533132380A4D33303343385332313545
:100440004530550A4D3530300A4D3131372050494D
:10045000442054756E6520446F6E65004D3139300F
:100460005335350A4D313034533231350A4732383D
:100470000A4732394C310A4731205831303059312E
:10048000303046353030300A47315A30004D353043
:10049000300A4D3131372053657474696E677320AB
:1004A00053746F726564005072657020666F7220BD
:1004B0005A2041646A7573740053746F72652053D7
:1004C000657474696E6773005049442054756E6595
:1004D000005365747570004D61696E003F004261A4
:1004E000636B0053746F70004D3231005072696E4F
:1004F000742066726F6D204D656469610052656C91
:1005000065617365204D65646961004D3232004C50
:100510006576656C696E6720546F6F6C7300436F0E
:100520006E66696775726174696F6E0054656D708F
:1005300065726174757265004D6F74696F6E0052FB
:100540006573756D65205072696E740041747461D5
:100550006368204D656469610054756E650053746D
:100560006F70205072696E74005061757365205011
:1005700072696E7400496E666F2053637265656EB2
:100580000043616E6E6F7420656E746572207375C2
:10059000626469723A2000022E2E00015265667272
:1005A000657368004D61696E002100486F74656E67
:1005B0006420746F6F20636F6C64004261636B0032
:1005C00050726F63656564004D6F74696F6E0044AF
:1005D000697361626C652053746570706572730035
:1005E0004D3834004175746F20486F6D6500473297
:1005F00038004D61696E0050726568656174202431
:1006000020456E6400507265686561742024204244
:1006100065640054656D706572617475726500C5BE
:1006200001C101436F6F6C646F776E005072656833
:1006300065617420240046616E2053706565640016
:10064000426564004E6F7A7A6C65004D61696E0098
:1006500050726F6265205A204F666673657400465B
:100660006C6F770046616E2053706565640042656B
:1006700064004E6F7A7A6C65005370656564004D56
:1006800061696E00486F6D696E67204661696C65CF
:1006900064006F70656E00545249474745524544A7
:1006A000003A20007A5F6D696E00795F6D696E00B7
:1006B000785F6D696E005265706F7274696E672045
:1006C000656E6473746F70207374617475730A005F
:1006D00020746F6F206C6F6E67206578747275730D
:1006E000696F6E2070726576656E7465640A0020AD
:1006F000636F6C6420657874727573696F6E2070B7
:10070000726576656E7465640A00486F6D652025B4
:100710007325732573204669727374005761726E76
:10072000696E673A20486F6D696E672042756D701B
:100730002044697669736F72203C20310A000202FE
:100740000400000000000000000000000000007A2B
:100750004300007A4300007A43000000410000009B
:10076000410000004000007A4300007A4300007A14
:10077000430000000000000000000000005365740A
:1007800074696E67732053746F72656400454550D9
:10079000524F4D20496E697469616C697A65640ACB
:1007A0000000803B4400803B440000204100009654
:1007B000420000A0420000A0420000C8430000BE6A
:1007C00042D0070000D0070000640000004B00008A
:1007D0000024F4D43050C38E20C2A24017828B7004
:1007E00011127A910D816CD90AA861E108C7586687
:1007F00007615143061E4B5D05C145A7041A41110F
:1008000004093D9803713931034036DB02653391A9
:1008100002D4305402802E1D02632CEE01752AC5CD
:1008200001B028A001102781018F2564012B244BE2
:1008300001E0223401AC211F018D200D01801FFC3D
:1008400000841EED00971DDF00B81CD200E61BC619
:1008500000201BBC00641AB200B219A8000A19A03B
:10086000006A189900D117910040178B00B51684C3
:100870000031167E00B31579003A157300C7146F66
:100880000058146A00EE1366008813630025135E97
:1008900000C7125B006C12570015125400C11151B1
:1008A0000070114F0021114B00D61049008D1047E8
:1008B000004610440002104200C00F4000800F3E6E
:1008C00000420F3C00060F3B00CB0E3800930E3762
:1008D000005C0E3500270E3400F30D3200C10D31DF
:1008E00000900D3000600D2E00320D2D00050D2CF6
:1008F00000D90C2B00AE0C2900850C29005C0C27BC
:1009000000350C27000E0C2600E80B2400C40B2435
:1009100000A00B23007D0B23005A0B2100390B2173
:1009200000180B2000F80A1F00D90A1E00BB0A1E7F
:10093000009D0A1D00800A1D00630A1C00470A1B57
:10094000002C0A1B00110A1A00F7091A00DD091908
:1009500000C4091900AB091900920917007B091896
:1009600000630917004C0916003609160020091605
:10097000000A091500F5081500E0081400CC081459
:1009800000B8081400A4081400900813007D081291
:10099000006B0813005808120046081200340811B2
:1009A00000230811001208110001081100F00710BF
:1009B00000E0071000D0071000C0071000B0070FBC
:1009C00000A107100091070E0083070F0074070FA6
:1009D0000065070E0057070E0049070E003B070D84
:1009E000002E070E0020070D0013070D0006070D4F
:1009F00000F9060C00ED060D00E0060C00D4060C14
:100A000000C8060C00BC060C00B0060C00A4060BC7
:100A10000099060C008D060B0082060B0077060B72
:100A2000006C060B0061060A0057060B004C060A14
:100A30000042060A0038060A002E060A0024060AAA
:100A4000001A060A001006090007060A00FD05093B
:100A500000F4050900EB050900E2050900D90509C4
:100A600000D0050900C7050900BE050900B5050845
:100A700000AD050800A50509009C050800940508BF
:100A8000008C050800840508007C05080074050832
:100A9000006C050700650508005D050700560508A0
:100AA000004E050700470507004005080038050708
:100AB00000310507002A050700230507001C05066D
:100AC00000160507000F05070008050600020507C8
:100AD00000FB040600F5040700EE040600E8040627
:100AE00000E2040700DB040600D5040600CF04067C
:100AF00000C9040600C3040600BD040600B70406CE
:100B000000B1040500AC040600A6040600A004051C
:100B1000009B04060095040500900406008A040565
:100B20000085040500800406007A040500750405AC
:100B300000700405006B04050066040500610405EF
:100B4000005C04050057040500520405004D04052F
:100B50000048040500430405003E0404003A04056F
:100B60000035040500300404002C040500270404AB
:100B700000230405001E0404001A040400160405E2
:100B800000110404000D0404000904050004040419
:100B90000000040400FC030400F8030400F4030450
:100BA00000F0030400EC030400E8030400E4030481
:100BB00000E0030400DC030400D8030400D40304B1
:100BC00000D0030400CC030400C8030300C50303E2
:100BD0000024F404D9201BC40C5C0E9804C4095FE3
:100BE0000265077101F405F900FB04B300480487AE
:100BF00000C10369005803550003034500BE023AD3
:100C0000008402310053022A002902250004022038
:100C100000E4011C00C8011900AF0117009801147D
:100C20000084011300710110006101100051010ED8
:100C30000043010D0036010B002B010B0020010BBE
:100C400000150109000C01090003010800FB000860
:100C500000F3000800EB000700E4000600DE0006D9
:100C600000D8000600D2000600CC000500C7000531
:100C700000C2000500BD000400B9000400B5000476
:100C800000B1000400AD000400A9000400A50003A9
:100C900000A20003009F0004009B000300980003D3
:100CA000009500020093000300900003008D0002F5
:100CB000008B00030088000200860002008400030D
:100CC00000810002007F0002007D0002007B000224
:100CD0000079000200770001007600020074000233
:100CE0000072000100710002006F0002006D00013F
:100CF000006C0002006A0001006900020067000148
:100D0000006600010065000100640002006200014D
:100D10000061000100600001005F0002005D000151
:100D2000005C0001005B0001005A00010059000155
:100D30000058000100570001005600010055000155
:100D40000054000100530000005300010052000154
:100D50000051000100500001004F0001004E000052
:100D6000004E0001004D0001004C0001004B00004E
:100D7000004B0001004A000100490001004800004A
:100D80000048000100470001004600000046000145
:100D90000045000000450001004400010043000040
:100DA0000043000100420000004200010041000039
:100DB0000041000100400001003F0000003F000131
:100DC000003E0000003E0001003D0000003D00012B
:100DD000003C0000003C0000003C0001003B000023
:100DE000003B0001003A0000003A00010039000019
:100DF0000039000100380000003800000038000110
:100E00000037000000370001003600000036000007
:100E100000360001003500000035000000350001FB
:100E200000340000003400000034000100330000F2
:100E300000330000003300010032000000320000E7
:100E400000320001003100000031000000310001DB
:100E5000003000000030000000300001002F0000D2
:100E6000002F0000002F0000002F0001002E0000C6
:100E7000002E0000002E0001002D0000002D0000BB
:100E8000002D0000002D0001002C0000002C0000AF
:100E9000002C0000002C0001002B0000002B0000A3
:100EA000002B0000002B0001002A0000002A000097
:100EB000002A0000002A000100290000002900008B
:100EC000002900000029000000290001002800007E
:100ED0000028000000280000002800000028000171
:100EE0000027000000270000002700000027000066
:100EF0000027000100260000002600000026000058
:100F0000002600000026000100250000002500004A
:100F1000002500000025000000250000002500013C
:100F20000024000000240000002400000024000031
:100F30000024000100230000002300000023000023
:100F40000023000000230000002300000023000114
:100F50000022000000220000002200000022000009
:100F600000220000002200010021000000210000FA
:100F700000210000002100000021000000210000ED
:100F800000210001002000000020000000200000DF
:100F900000200000002000000020000000200000D1
:100FA00000200001001F0000001F0000001F0000C3
:100FB000001F0000001F0000001F0000001F0001B4
:100FC000001E0000001E0000001E0000001E0000A9
:100FD00000043700001E290000511B0000581000BB
:100FE0000010090000CC040000780200004101005C
:100FF0000020436F756E7420583A004265640045C6
:101000003100626564002C2073797374656D207300
:10101000746F7070656421204865617465725F4902
:10102000443A200048656174696E67204661696CC6
:1010300065640048656174696E67206661696C6506
:1010400064004D3131322053687574646F776E00DF
:101050001000C90210012C01400122017001180189
:10106000B0010E01F00104015002FA00B002F000DC
:101070003003E600D003DC009004D2007005C80005
:10108000A006BE000008B400B009AA00D00BA00062
:10109000600E960060118C00001582002019780007
:1010A000C01D6E00A0226400B0275A00902C500092
:1010B00000314600E0343C0010383200903A2800FD
:1010C000603C1E00A03D1400803E0A00203F00004E
:1010D000544845524D414C2052554E4157415900BC
:1010E000546865726D616C2052756E61776179002C
:1010F0004572723A204D415854454D50004D41586B
:1011000054454D5020747269676765726564004587
:1011100072723A204D494E54454D50004D494E543F
:10112000454D502074726967676572656400202FB1
:10113000002042403A0020403A007C3C3E5E2B3D7D
:101140003F2F5B5D3B2C2A225C00434F4D4D554E9B
:1011500049434154494F4E0044525952554E00455F
:1011600052524F525300494E464F004543484F009C
:10117000486F74656E642049646C652054696D65C0
:101180006F757400486F74656E642049646C6520E7
:1011900054696D656F75740A002121204B494C4CD0
:1011A0002063617573656420627920746F6F206DB0
:1011B00075636820696E6163746976652074696D12
:1011C00065202D2063757272656E7420636F6D6D7E
:1011D000616E643A200053544F505045442E200015
:1011E0005072696E7465722073746F7070656420DC
:1011F00064756520746F206572726F72732E20465D
:10120000697820746865206572726F7220616E64FF
:1012100020757365204D39393920746F20726573DC
:10122000746172742E202854656D706572617475D6
:1012300072652069732072657365742E205365741E
:1012400020697420616674657220726573746172BE
:1012500074696E67290A004E6F20436865636B737B
:10126000756D2077697468206C696E65206E756D88
:101270006265722C204C617374204C696E653A2053
:10128000004E6F20436865636B73756D20776974DA
:1012900068206C696E65206E756D6265722C204CDD
:1012A000617374204C696E653A2000636865636BF6
:1012B00073756D206D69736D617463682C204C616A
:1012C0007374204C696E653A20004C696E65204E3F
:1012D000756D626572206973206E6F74204C617346
:1012E00074204C696E65204E756D6265722B312CD1
:1012F000204C617374204C696E653A20004D313189
:10130000300053657269616C207374617475732069
:101310006D69736D617463680A005344207265617E
:1013200064206572726F720A004D656469612049BC
:101330006E73657274656400506C656173652052EC
:1013400065736574005052494E5445522048414CD3
:101350005445440025533A20255300706F77657239
:101360006F6666004B494C4C45442E200050726914
:101370006E7465722068616C7465642E206B696C94
:101380006C28292063616C6C6564210A0053544FFA
:10139000505045442E20005072696E74657220735F
:1013A000746F707065642064756520746F20657259
:1013B000726F72732E20466978207468652065729A
:1013C000726F7220616E6420757365204D393939F2
:1013D00020746F20726573746172742E20285465B6
:1013E0006D706572617475726520697320726573C2
:1013F00065742E205365742069742061667465726B
:101400002072657374617274696E67290A0065637E
:10141000686F3A004572726F723A0042696C696E89
:10142000656172204C6576656C696E6720477269EC
:10143000643A0A0021212053544F502063616C6CA0
:1014400065642062656361757365206F6620424C38
:10145000546F756368206572726F72202D207265FB
:1014600073746172742077697468204D3939390A50
:101470000021212053544F502063616C6C6564201F
:1014800062656361757365206F6620424C546F75A9
:101490006368206572726F72202D207265737461AB
:1014A00072742077697468204D3939390A004265B1
:1014B00064204C6576656C696E6720004661696CD6
:1014C000656420746F20656E61626C65204265649E
:1014D000204C6576656C696E670A00496E76616CB2
:1014E0006964206D6573682E0A0050726F62696EC0
:1014F0006720506F696E740025532025692F256978
:10150000002E0A002F0050726F62696E67206D65B1
:10151000736820706F696E742000202844525952FD
:10152000554E2900473239204175746F2042656459
:10153000204C6576656C696E67003F20284C2C5204
:101540002C462C4229206F7574206F6620626F75BF
:101550006E64732E0A003F2856296572626F7365A8
:10156000206C6576656C20696D706C61757369625D
:101570006C652028302D34292E0A00426164205ADF
:101580002076616C75650A004E6F2062696C696E29
:1015900065617220677269640A0020496E76616C29
:1015A00069642065787472756465722000536C6597
:1015B00065702E2E2E005A2050726F626520506189
:1015C0007374204265640A005A2050726F6265206D
:1015D0005061737420426564004732384C300020FB
:1015E0005A3A200020593A200042656420583A2097
:1015F000004D65736820706F696E74206F7574207C
:101600006F662072616E67650A00436C69636B20C8
:10161000746F20526573756D652E2E2E004E6F20EF
:101620004D6F76652E00456E642066696C65206C92
:101630006973740A00426567696E2066696C65208B
:101640006C6973740A004E6F206D656469610A00ED
:10165000706175736500286E6F2066696C6529007E
:1016600043757272656E742066696C653A2000532A
:1016700044207072696E74696E67206279746520A7
:10168000004E6F74205344207072696E74696E67E7
:101690000A002E0A0044656C6574696F6E206661ED
:1016A000696C65642C2046696C653A200046696C5B
:1016B000652064656C657465643A0025697300256E
:1016C000696D20256973002569682025696D2025CD
:1016D000697300256964202569682025696D2025C6
:1016E00069730025697920256964202569682025AA
:1016F000696D20256973005072696E742074696D7C
:10170000653A20006F6B006F6666006B1166115FB3
:101710001158114A1144454255473A00544D33443B
:1017200020456E64657233204F46462E00204500EA
:10173000204D39322058004649524D574152455F9D
:101740004E414D453A4D61726C696E20322E302EFD
:10175000375F4457372E3320544D334420453345AB
:101760004D444242202841707220323420323032BF
:10177000312032313A35363A33342920534F5552DD
:1017800043455F434F44455F55524C3A687474700B
:10179000733A2F2F6769746875622E636F6D2F49D6
:1017A0006E73616E6974794175746F6D6174696F80
:1017B0006E2F4D61726C696E2F747265652F437266
:1017C00065616C6974794477696E5F322E302050A0
:1017D000524F544F434F4C5F56455253494F4E3A28
:1017E000312E30204D414348494E455F54595045B4
:1017F0003A544D334420456E646572332045585445
:1018000052554445525F434F554E543A3120555539
:1018100049443A63656465326132662D3431613220
:101820002D343734382D396231322D6335356336F6
:10183000326633363766660A002F2F004D31343555
:1018400020533C696E6465783E206F7574206F6626
:101850002072616E67652028302D31290A002054DE
:1018600000205200416363656C65726174696F6E3C
:101870003A2050005741524E494E4721204C6F7735
:10188000205A204A65726B206D6179206C65616415
:1018900020746F20756E77616E7465642070617559
:1018A0007365732E0A004D3230362058004F46467D
:1018B000004F4E0020580020204D61783A20002033
:1018C0000020204D696E3A2000536F667420656ECB
:1018D0006473746F70733A200046523A0020466C6D
:1018E0006F773A20003A200020536572766F20000F
:1018F000206F7574206F662072616E67650A0053F1
:101900006572766F200050726F6265204F66667355
:101910006574205A0050726F6265204F6666736569
:1019200074205A0020643A0020693A0020703A007E
:10193000496E76616C69642065787472756465724D
:101940000A0064697300656E0043290A0061626CD5
:10195000656420286D696E2074656D702000436F8A
:101960006C6420657874727564657320617265209B
:10197000004D34323120696E636F7272656374207A
:10198000706172616D657465722075736167650A57
:10199000004D65736820706F696E74206F757420D8
:1019A0006F662072616E67650A004F6666736574C4
:1019B00073204170706C696564004572723A2054FE
:1019C0006F6F206661722100546F6F206661722014
:1019D00066726F6D207265666572656E63652070F4
:1019E0006F696E740A00454550524F4D204F4B0AA7
:1019F00000290A0020746F20003F5A206F75742060
:101A00006F662072616E6765202800290A002074C5
:101A10006F20003F59206F7574206F662072616ED1
:101A2000676520282D00290A0020746F20003F5888
:101A3000206F7574206F662072616E676520282D97
:101A400000205A0020590050726F6265204F666670
:101A50007365742058004D383400446F6E652070F3
:101A600072696E74696E672066696C650A004D372D
:101A700037004D333100496E76616C6964206578BA
:101A80007472756465720A0020573A00436F6F6C78
:101A9000696E672E2E2E0048656174696E672E2E62
:101AA0002E00452025530020573A0042656420430C
:101AB0006F6F6C696E672E2E2E004265642048653C
:101AC0006174696E672E2E2E0023646566696E65EB
:101AD0002044454641554C545F004B6420004B69FF
:101AE00020004B702000504944204175746F74757C
:101AF0006E652066696E697368656421205075742F
:101B000020746865206C617374204B702C204B69C5
:101B100020616E64204B6420636F6E7374616E7419
:101B2000732066726F6D2062656C6F7720696E74CA
:101B30006F20436F6E66696775726174696F6E2E90
:101B4000680A00504944204175746F74756E6520B1
:101B50006661696C6564212074696D656F75740ACE
:101B600000504944204175746F74756E652066613C
:101B7000696C6564212054656D706572617475725D
:101B80006520746F6F20686967680A00204B643AAB
:101B90002000204B693A2000204B703A200020435F
:101BA0006C617373696320504944200A00205475A6
:101BB0003A2000204B753A2000206D61783A2000D1
:101BC000206D696E3A200020643A2000206269612D
:101BD000733A2000504944204175746F74756E65E6
:101BE0002073746172740A00504944204175746F07
:101BF00074756E65206661696C6564212054656D3D
:101C0000706572617475726520746F6F20686967A2
:101C1000680A00504944204175746F74756E6520E0
:101C20006661696C65642120426164206865617445
:101C300065722069640A00504944204175746F74CC
:101C4000756E65004572723A207574663820666F4D
:101C50006E74206E6F7420696E697469616C697A44
:101C600065642E004572723A207574663820666F7E
:101C70006E74206E6F7420696E697469616C697A24
:101C800065642E004572723A207574663820666F5E
:101C90006E74206E6F7420696E697469616C697A04
:101CA00065642E00000C0F00FE07022503BB017FB8
:101CB000FE08FE08FE05080806000040F0C88888F7
:101CC000987810050808060000C0F8888888888879
:101CD000F80505050600012030F830200508080643
:101CE00000002070F820202020E00509090600FFF0
:101CF0002070A8A8B888887020070505070001D8BB
:101D00006C366CD80509090600FFF8A88888888811
:101D100088A8F8050A0A0600FE205050505088A8EE
:101D2000A8887003030306000340A040FFFFFFFFE5
:101D3000FFFFFFFFFFFFFFFFFFFFFFFFFFFFFFFFB3
:101D4000FFFF0000000605FF010707060200808074
:101D50008080800080030303060105A0A0A0050683
:101D60000606000050F85050F8500509090600FF1B
:101D70002070A8A07028A87020050707060000C8DA
:101D8000C8102040989805070706000040A0A04012
:101D9000A8906801030306020580808003090906F4
:101DA00001FF204040808080404020030909060157
:101DB000FF804040202020404080050707060000AB
:101DC00020A8702070A8200505050600012020F835
:101DD00020200203030601FFC04080050101060028
:101DE00003F8020202060100C0C005070706000052
:101DF00008101020404080050707060000708898F2
:101E0000A8C8887003070706010040C04040404052
:101E1000E0050707060000708808102040F8050755
:101E200007060000F808103008887005070706004C
:101E30000010305090F81010050707060000F880D9
:101E4000F008088870050707060000304080F08819
:101E50008870050707060000F808101020202005EC
:101E600007070600007088887088887005070706D5
:101E7000000070888878081060020505060100C01F
:101E8000C000C0C00206060601FFC0C000C04080FE
:101E900003050506010120408040200503030600DC
:101EA00002F800F803050506010180402040800586
:101EB000070706000070881020200020050707068D
:101EC00000007088B8A8B880700507070600007089
:101ED0008888F8888888050707060000F048487059
:101EE0004848F005070706000070888080808870E9
:101EF000050707060000F04848484848F00507076E
:101F0000060000F88080F08080F8050707060000D2
:101F1000F88080F0808080050707060000708880C8
:101F200080988870050707060000888888F88888E8
:101F300088030707060100E04040404040E00507F5
:101F40000706000038101010109060050707060003
:101F5000008890A0C0A09088050707060000808038
:101F600080808080F805070706000088D8A8888848
:101F700088880507070600008888C8A8988888050B
:101F8000070706000070888888888870050707069C
:101F90000000F08888F08080800507070600007048
:101FA000888888A89068050707060000F08888F0F0
:101FB000A090880507070600007088807008887068
:101FC000050707060000F82020202020200507072D
:101FD0000600008888888888887005070706000042
:101FE0008888888850502005070706000088888860
:101FF00088A8A85005070706000088885020508848
:102000008805070706000088885020202020050743
:1020100007060000F80810204080F80309090601AF
:10202000FFE080808080808080E005070706000058
:10203000804040201010080309090601FFE020201D
:102040002020202020E005030306000520508805FD
:1020500001010600FEF80303030601058040200588
:102060000505060000700878887805070706000057
:102070008080F0888888F005050506000070808063
:1020800088700507070600000808788888887805A2
:1020900005050600007088F080700507070600003F
:1020A000304840E04040400507070600FE70888841
:1020B000887808700507070600008080F088888807
:1020C000880307070601004000C0404040E00409C3
:1020D000090601FE1000301010101090600507076F
:1020E00006000080808890E09088030707060100C2
:1020F000C04040404040E0050505060000D0A8A8CB
:10210000A8A8050505060000B0C88888880505054B
:1021100006000070888888700507070600FEF088B2
:102120008888F080800507070600FE788888887810
:102130000808050505060000B0C880808005050573
:1021400006000078807008F00507070600002020D0
:10215000F820202018050505060000888888986862
:10216000050505060000888888502005050506003D
:10217000008888A8A8500505050600008850205052
:10218000880507070600FE888888502040800505DE
:1021900005060000F8102040F80309090601FF2099
:1021A00040404080404040200109090602FF8080F5
:1021B000808080808080800309090601FF80404084
:1021C00040204040408005030306000248A890FFDD
:1021D00043616E6E6F74206F70656E2073756264FC
:1021E0006972200053442063617264206F6B0A009F
:1021F0006F70656E526F6F74206661696C65640AFA
:1022000000766F6C756D652E696E69742066616904
:102210006C65640A004E6F20534420636172640A47
:10222000000A4D3234004D3233202573002E0A004F
:102230006F70656E206661696C65642C2046696C00
:10224000653A200046696C652073656C656374654A
:10225000640A002053697A653A200046696C65205B
:102260006F70656E65643A2000454E4420535542B8
:10227000524F5554494E450A002220706F73002278
:1022800020706172656E743A2200535542524F5568
:1022900054494E452043414C4C207461726765742B
:1022A0003A220053756263616C6C204F76657266EA
:1022B0006C6F77004578636565646564206D61784F
:1022C00020535542524F5554494E45206465707411
:1022D000683A0057726974696E6720746F20666986
:1022E0006C653A2000667265736800646F696E679A
:1022F000002066696C653A20004E6F7720002F61E0
:1023000075746F25632E67006001F4017001EA01A6
:102310009001E001B001D601D001CC010002C20160
:102320003002B8016002AE019002A401D0029A010D
:102330002003900170038601C0037C013004720108
:10234000A004680120055E01B005540160064A0141
:1023500020074001F0073601F0082C01100A220185
:10236000500B1801C00C0E01500E04013010FA0081
:102370002012F0005014E600C016DC007019D200E4
:10238000501CC800501FBE007022B400B025AA0027
:10239000F028A000202C9600302F8C0010328200F4
:1023A000A0347800F0366E00E0386400803A5A00BD
:1023B000403B5500E03B5000F03C4600C03D3C0037
:1023C000603E3200E03E2800303F1E00503F1900C2
:1023D000703F1400A03F0A00C03F0000D03FF6FF4E
:1023E000E03FECFF2020506C616E6E6572427566B6
:1023F00066657242797465733A200020467265659D
:10240000204D656D6F72793A2000436F6D70696C75
:1024100065643A2041707220323420323032310A01
:1024200000204C61737420557064617465643A20B7
:10243000323032312D30342D3138207C20417574CA
:10244000686F723A2054696E794D616368696E6590
:102450007333440A00322E302E375F4457372E3301
:102460000A004D61726C696E0020536F667477616B
:1024700072652052657365740A0020576174636841
:10248000646F672052657365740A002042726F772B
:102490006E206F75742052657365740A002045784C
:1024A0007465726E616C2052657365740A00506FBA
:1024B00077657255700A0073746172740A0047324E
:1024C000385859004D31303031006F6B00657272F1
:1024D0006F722077726974696E6720746F20666905
:1024E0006C650A00446F6E6520736176696E6720C3
:1024F00066696C652E0A004D323900456E6473744E
:102500006F707300255320256320256320256320E9
:10251000256300205A3A0020593A0020583A0065B5
:102520006E6473746F7073206869743A20000000E1
:1025300000010200090A000000000403080700006F
:102540000000000000000000000000000000004D3E
:102550006F76652025736D6D004D6F766520302E8A
:10256000316D6D004D6F766520316D6D004D6F766C
:10257000652031306D6D004D6F766520417869734F
:10258000004578747275646572004D6F7665205AE7
:10259000004D6F76652059004D6F766520580050CC
:1025A00072696E742066726F6D204D65646961009A
:1025B000FFFFFF50726F62696E67204661696C654C
:1025C000640A0050726F62696E67204661696C65CB
:1025D0006400205A3A200020593A200042656420C5
:1025E000583A2000220A00556E6B6E6F776E20639A
:1025F0006F6D6D616E643A202200544D3344204566
:102600006E646572332052656164792E0050726980
:102610006E74696E672E2E2E005072696E74205093
:1026200061757365640020453A00205A3A002059CC
:102630003A00583A004572726F7220777269746975
:102640006E6720746F20454550524F4D210A00207F
:10265000746F6F206C6F6E67206578747275736924
:102660006F6E2070726576656E7465640A00206313
:102670006F6C6420657874727573696F6E20707208
:102680006576656E7465640A00526573656E643ABA
:10269000200000002200250028002B00000021005F
:1026A000240027002A00020202020202020204049D
:1026B00004040404040403030303030303030101E8
:1026C0000101010101010102040810204080010202
:1026D000040810204080010204081020408080403F
:1026E0002010080402012F2F616374696F6E3A0095
:1026F000DAD4F9DB11241FBECFEFD0E4DEBFCDBFAB
:1027000012E0A0E0B1E0E2E5F4ED01E00BBF02C0B1
:1027100007900D92A034B107D9F728E1A0E4B2E008
:1027200001C01D92A630B207E1F713E1C9E7D3E17A
:1027300004C02197FE010E9488E7C837D107C9F776
:102740000E94C9D50C941CEA0C9400000F931F93AF
:10275000CF93DF93CDB7DEB760970FB6F894DEBFA7
:102760000FBECDBF8C01DC01ED91FC910280F381A5
:10277000E02DBE016F5F7F4F0995882309F464C087
:102780008981807CC9F56F81637070E0762F662740
:10279000770F770F8885B4E08B9FC0011124682BD9
:1027A000792B89858295869586958370682B6F5FD6
:1027B0007F4F90E080E02A852370220F3B8537FB16
:1027C000332730F9232B3E813F70230F3327331FEC
:1027D0002750310904C0660F771F881F991F2A955B
:1027E000D2F760960FB6F894DEBF0FBECDBFDF9173
:1027F000CF911F910F910895803419F568856695E2
:10280000669570E090E080E0CB01772766272A8507
:10281000622B098510E0102F0027012E000C220BDF
:10282000330B602B712B822B932B6F5F7F4F8F4F5E
:102830009F4F4AE0660F771F881F991F4A95D1F76F
:10284000D0CF8BE0F801848360E070E0CB01C9CF8A
:102850000895FC0182810895CF92DF92EF92FF925A
:1028600080917002882309F457C0C0906C02D09008
:102870006D02E0906E02F0906F0220E030E0A9015E
:10288000C701B6010E949BE0882309F445C020E0FF
:1028900030E040E05FE3C701B6010E9401E19B0127
:1028A000AC010E9401E12BED3FE049E450E40E94BD
:1028B00001E19B01AC0160E070E080E89FE30E94D1
:1028C00015E86B017C01C0926702D0926802E09229
:1028D0006902F0926A0260911C0170911D01072E3D
:1028E000000C880B990B0E94A2E02AE037ED43E22E
:1028F0005CE30E9401E1A70196010E9401E160935F
:102900006401709365018093660190936701FF9065
:10291000EF90DF90CF900895C12CD12C80E8E82E65
:102920008FE3F82ED0CF8F929F92AF92BF92CF922B
:10293000DF92EF92FF92FC01C080D180E280F380B1
:1029400020E030E040E251E4C701B6010E9401E11D
:1029500020E030E040E251E40E9401E14B015C01E3
:1029600020E030E0A901C701B6010E949BE020E011
:1029700030E040EA50E487FF04C020E030E040EA65
:1029800050ECC501B4010E9492E720E030E040E243
:1029900051E40E9415E80E9487E89B018BE237FF13
:1029A00005C022273327261B370B8DE2809335067F
:1029B000C90168EE73E00E9474E7CB01EAE0F0E041
:1029C000BF010E9474E7805D80933606C90164E60A
:1029D00070E00E9474E7CB01BF010E9474E7805D44
:1029E00080933706C901BF010E9474E7282FCB01ED
:1029F000BF010E9474E7805D809338068EE2809369
:102A00003906205D20933A0685E396E0FF90EF902B
:102A1000DF90CF90BF90AF909F908F9008959C01D2
:102A200097FF26C0EE27FF27E81BF90B2D398FEF04
:102A300038070CF05DC08DE280933706CF0164E665
:102A400070E00E9474E7CB012AE030E0B9010E94F7
:102A500074E7805D80933806CF01B9010E9474E766
:102A6000CB01B9010E9474E7805D809339062AC0CA
:102A7000283E83E03807B4F1C90168EE73E00E9494
:102A800074E7CB01EAE0F0E0BF010E9474E7805DEB
:102A900080933706C90164E670E00E9474E7CB01B9
:102AA000BF010E9474E7805D80933806C901BF01B1
:102AB0000E9474E7CB01BF010E9474E7805D8093A0
:102AC0003906F901CF016AE070E00E9474E7805D89
:102AD00080933A0687E396E008958DE237FDC5CFEF
:102AE00080E2C3CFF90180E2243631050CF0A4CF97
:102AF00080E28093370680933806EA30F1056CF364
:102B00008DE237FF80E280933806CF016AE070E003
:102B10000E9474E7605D60933906D4CF9C0197FDF5
:102B20002DC080E2243631055CF0C90164E670E016
:102B30000E9474E7CB016AE070E00E9474E7805D58
:102B40008093380680E22A3031055CF0EAE0F0E05C
:102B5000C901BF010E9474E7CB01BF010E9474E765
:102B6000805D80933906C9016AE070E00E9474E7D5
:102B7000805D80933A0688E396E00895319521952B
:102B800031098DE2DDCF282F81E3243609F080E280
:102B90008093370690E22A3040F03AE0822F632F8C
:102BA0000E9446E70E9446E7905D90933806822F88
:102BB0006AE00E9446E7905D9093390685E2809333
:102BC0003A0687E396E0089560911C0170911D011B
:102BD000072E000C880B990B0E94A2E02AE037ED2B
:102BE00043E25CE30E9401E12091670230916802B8
:102BF0004091690250916A020E9401E16093640170
:102C00007093650180936601909367010895CF9357
:102C1000DF93EC01CB01BA010E94A2E029EC38EC71
:102C200048EC5EE30E9415E820E030E040E05FE31E
:102C30000E9492E70E948EE86883DF91CF91089509
:102C40000E94A2E029EC38EC48EC5EE30E9415E813
:102C500020E030E040E05FE30E9492E70E948EE8CF
:102C600024E6629FC001112481589F4F6FEF70E0EE
:102C70000E9474E7862F0C94C315CF93DF93EC0169
:102C8000CB01BA010E94A2E020E030E0A9010E943D
:102C900092E70E9487E879836883DF91CF91089556
:102CA0000E94A2E020E030E0A9010E9492E70E9489
:102CB00087E8CB010C948E1580914206811104C0E7
:102CC0008091FA058093A4060895809119178823AE
:102CD000C1F0815080931917E2E5F5E1882351F0A6
:102CE0008150990B2BE1289FF001299FF00D1124B1
:102CF000E55FF94E8BE1A7E3B5E101900D928A956E
:102D0000E1F720911917211105C0809124178062E5
:102D10008093241781E090E0A0E0B0E0211103C08F
:102D200080E090E0DC018093300690933106A09320
:102D30003206B093330610922B0681E080932D0665
:102D400083E080935B0108958F929F92AF92BF9230
:102D5000CF92DF92EF92FF92CF936B017C0120E044
:102D600030E0A9010E949BE087FDAAC06DEB77E3EC
:102D700086E095E3A70196010E9492E76B017C0132
:102D800020E030E0A9010E949BE087FF9EC0C701C0
:102D9000B601905820E030E040E251E40E9401E1A9
:102DA00020E030E040E251E40E9401E120E030E028
:102DB00040EA50E40E9492E720E030E040E251E433
:102DC0000E9415E80E9487E86B017C0180E28093F5
:102DD000340660E280E1C81687E2D806E104F10417
:102DE0008CF0C701B60120E137E240E050E00E94DC
:102DF00005E7CA01B9012AE030E040E050E00E9456
:102E000005E7605D6093350660E288EEC81683E0F2
:102E1000D806E104F1048CF0C701B60128EE33E0D6
:102E200040E050E00E9405E7CA01B9012AE030E025
:102E300040E050E00E9405E7605D6093360660E286
:102E400084E6C816D104E104F1048CF0C701B60190
:102E500024E630E040E050E00E9405E7CA01B901F5
:102E60002AE030E040E050E00E9405E7605D6093BA
:102E700037068AE0882E912CA12CB12CC701B6010F
:102E8000A50194010E9405E7C62FCA01B901A50159
:102E900094010E9405E7605D609338068EE280939E
:102EA0003906C05DC0933A0684E396E0CF91FF9067
:102EB000EF90DF90CF90BF90AF909F908F9008954C
:102EC0006DEB77E386E095EB55CF20E030E040E214
:102ED00051E4C701B60162CFCF93DF93EC01CB0180
:102EE000BA010E94A2E020E030E040E251E40E94FA
:102EF00015E820E030E0A9010E9492E76883798319
:102F00008A839B83DF91CF9108950E94A2E020E005
:102F100030E040E251E40E9415E820E030E0A901F1
:102F20000E9492E70C94A416CF93DF93EC01CB019F
:102F3000BA010E94A2E020E030E04AE754E40E9497
:102F400015E820E030E0A9010E9492E768837983C8
:102F50008A839B83DF91CF9108958091B8159091DA
:102F6000B915891B8F7051F480915D06813031F065
:102F70008091241782FB882780F9089581E00895C5
:102F8000FC0184910895FC0180810895209104063C
:102F90003091050621153105E9F0809102069091E6
:102FA0000306029624503109821793079CF49093EC
:102FB0001A05809319050E949EC1605E70448D4F72
:102FC0009F4F60931B0570931C0580931D05909384
:102FD0001E05089510921B0510921C0510921D05E8
:102FE00010921E0508958F929F92AF92BF92EF921A
:102FF000FF920F931F93CF93DF93EC018B01E42E8D
:10300000F22E8091CA159091CB158C179D0709F46B
:103010003EC02091460227FD109246022CE5C333A4
:10302000D20709F03FC08D51924671F40E949EC1B3
:103030006E517B4F8F4F9F4F609364047093650474
:103040008093660490936704D093CB15C093CA1500
:1030500030E020E0009330061093310620933206D2
:1030600030933306E0922B06F0922C06CD51D246D7
:1030700021F410922A061092630482E080935B018F
:1030800081E080932D0610926A0410922906DF9148
:10309000CF911F910F91FF90EF90BF90AF909F90B5
:1030A0008F90089522E6CD31D20771F683539C4567
:1030B00019F0CDE1D2E6C8CF0E949EC18090640491
:1030C00090906504A0906604B0906704681979092F
:1030D0008A099B0997FFEDCF80914506877087305D
:1030E00041F7C4E0D6E5B0CF20E040E070E060E01A
:1030F00080EB9DE10C94F3178091B506811114C00B
:103100008091680190916901019720910915309192
:103110000A152817390744F420E040E070E060E029
:1031200085EB9DE10C94F3170C94741821E0209327
:103130002A06FC0180819181A281B38180931201D2
:1031400090931301A0931401B093150120E040E087
:1031500070E060E080911706909118060C94F317C8
:10316000CF93DF9300D000D0CDB7DEB78DEC9CECD1
:10317000ACECBCE389839A83AB83BC83CE0101961C
:103180000E9496180F900F900F900F90DF91CF91A3
:103190000895CF93DF9300D000D0CDB7DEB78DEC8C
:1031A0009CECACECBDE389839A83AB83BC83CE01FA
:1031B00001960E9496180F900F900F900F90DF913C
:1031C000CF910895CF93DF9300D000D0CDB7DEB775
:1031D00080E090E0A0E8BFE389839A83AB83BC835F
:1031E000CE0101960E9496180F900F900F900F90AD
:1031F000DF91CF910895CF93DF9300D000D0CDB76A
:10320000DEB780E090E0A0E2B1E489839A83AB83EB
:10321000BC83CE0101960E9496180F900F900F90DC
:103220000F90DF91CF9108950F931F930E949EC13D
:1032300000912704109128042091290430912A0438
:10324000601B710B820B930B97FD0CC089B183FB44
:10325000882780F991E089274A9B8260309B8460AF
:10326000809326048091260481709091260491FD1C
:10327000826090912504981749F0813009F148F057
:10328000823079F0833091F0809325041F910F9163
:103290000895913079F09230B9F7909124049150CB
:1032A0000CC0992339F09330C1F3EECF9130A9F3DC
:1032B000923051F7909124049F5F90932404E4CFBF
:1032C000992359F3933001F7F5CFCF92DF92EF9224
:1032D000FF92CF93C82F0E949EC16B017C0124EA0C
:1032E00030E74DE75FE36091120170911301809127
:1032F0001401909115010E949BE087FD18C08AEF90
:1033000090E0A0E0B0E08C0D9D1DAE1DBF1D809330
:10331000180490931904A0931A04B0931B04C0934B
:103320001001CF91FF90EF90DF90CF90089580E053
:1033300090E0DC01E8CFCF93DF93EC018D810E9418
:10334000F97E60E08B81DF91CF910C94A7C0DF9272
:10335000EF92FF920F931F93CF93DF938C01C62FB1
:10336000D22FF32EE42ED52E0E949B190E941DC24F
:103370008C2F80640E94ED7E8D2D0E94ED7E8E2D1F
:103380000E94ED7E8F2D0E94ED7E8D2F0E94ED7E9E
:1033900087E8C11101C085E90E94ED7ECC3011F4AF
:1033A0000E94F27EC0E00E94F27EF801868387FFD1
:1033B00004C0CF3F11F0CF5FF6CFDF91CF911F91C7
:1033C0000F91FF90EF90DF90089561E0FC01838101
:1033D0000E94A7C08FEF0C94ED7E0F931F93CF93A5
:1033E0008C010E949B190E941DC2C82F882371F076
:1033F0008DEF0E94ED7E0E941DC2C82FC8010E9461
:10340000E5198C2FCF911F910F91089582E1F8015A
:103410008483F4CF8F929F92AF92BF92CF92DF922C
:10342000EF92FF920F931F93CF93DF93EC016A010A
:103430007B01590120E030E0A90167E30E94A71950
:10344000A501980167E1CE010E94A719811127C04B
:103450008F81833039F089E0CC0CDD1CEE1CFF1C21
:103460008A95D1F7A701960169E1CE010E94A719BB
:1034700011E0882319F010E087E08C83CE010E94D0
:10348000E519812FDF91CF911F910F91FF90EF9060
:10349000DF90CF90BF90AF909F908F90089589E07C
:1034A0008C8310E0EBCFCF93DF93EC016EBDFA017C
:1034B000CA019E5F0DB407FEFDCF20812EBD0DB465
:1034C00007FEFDCF21812EBD3296E817F90791F74F
:1034D0000DB407FEFDCF8FEF0E94ED7E8FEF0E94AF
:1034E000ED7E0E94F27E8E838F71853049F083E1FC
:1034F0008C83CE010E94E51980E0DF91CF91089581
:1035000081E0FBCF0F931F93CF93DF93EC018B01EF
:103510000E949B190E941DC281110CC085E18C8301
:1035200010E0CE010E94E519812FDF91CF911F910C
:103530000F910895A8016CEFCE010E94531A182F25
:10354000882361F3EECF0F931F93CF93DF93EC01AA
:1035500089018F81833039F089E0440F551F661F40
:10356000771F8A95D1F79A01AB0168E1CE010E94DD
:10357000A71981112AC0A8016EEFCE010E94531A2B
:10358000182F8823B1F00E941DC2182F8823D1F074
:1035900020E030E0A9016DE0CE010E94A719882348
:1035A00021F086E18C8310E004C00E94F27E81113C
:1035B000F8CFCE010E94E519812FDF91CF911F91A5
:1035C0000F91089587E18C83F4CF86E0EBCF1F93B2
:1035D000CF93DF93EC010E949B1920E030E0A9011A
:1035E0006CE0CE010E94A71911E0882319F010E0C9
:1035F00083E08C83CE010E94E519812FDF91CF916A
:103600001F9108951F93CF93DF93EC018F81833037
:1036100039F089E0440F551F661F771F8A95D1F74F
:103620009A01AB0162E1CE010E94A71911E0882343
:1036300019F010E085E08C83CE010E94E519812FFE
:10364000DF91CF911F9108958F929F92AF92BF9279
:10365000EF92FF920F931F93CF93DF938C01EB01B7
:103660007A010E949EC14B015C012CE2820E21E096
:10367000921EA11CB11C0E94F27EF80186838F3F2E
:1036800069F40E949EC1681979098A099B0997FD0E
:10369000F2CF81E1F8018483C0E021C08E3F71F553
:1036A000F1E0EF1AF1088FEF8EBDFE012FEF0DB4A0
:1036B00007FEFDCF8EB581932EBDCF018C1B9D0BD8
:1036C0008E159F05A0F30DB407FEFDCF8EB5CE0D70
:1036D000DF1D88830E94F27E0E94F27EC1E0C80155
:1036E0000E94E5198C2FDF91CF911F910F91FF90D0
:1036F000EF90BF90AF909F908F9008958FE0CACFCA
:103700000F931F93CF93DF93EC018B010E949B19C2
:1037100040E052E0B801CE01DF91CF911F910F91AF
:103720000C94241B0F931F93CF93DF93EC0189011B
:103730008F81833039F089E0440F551F661F771F52
:103740008A95D1F79A01AB0161E1CE010E94A719D8
:1037500081110AC040E052E0B801CE01DF91CF9163
:103760001F910F910C94241B84E08C83CE010E9446
:10377000E51980E0DF91CF911F910F9108958F920D
:103780009F92AF92BF92CF92DF92EF92FF920F93F0
:103790001F93CF93DF93EC01162F1F821C824B8364
:1037A0000E949EC16B017C0120EDC20E27E0D21E5B
:1037B000E11CF11CA89561E08B810E94A7C08B8160
:1037C0000E940EB8249A2C9A279A2698259A81E06E
:1037D0000E94F97E85E08D830E94F97E0AE08FEFDA
:1037E0000E94ED7E0150D9F7A89520E030E0A901B4
:1037F00060E0CE010E94A7198E83813081F00E9483
:103800009EC16C197D098E099F0997FDEECF81E05D
:103810008C83CE010E94E5191A8280E06AC0A895C7
:103820002AEA31E040E050E068E0CE010E94A719AA
:10383000853041F581E08F83A8958F81812C912C73
:103840005401823029F4812C912CA12C80E4B82ED3
:1038500020E030E0A90167E3CE010E94A719A5018D
:10386000940169E2CE010E94A7198E838823F1F0AA
:103870000E949EC16C197D098E099F0997FDE8CFB2
:103880008AE0C6CF04E00E94F27E8E830150D9F711
:103890008A3A11F482E0CFCF0E949EC16C197D0953
:1038A0008E099F0997FDBCCF82E0B2CF8F81823015
:1038B000C1F420E030E0A9016AE3CE010E94A7191B
:1038C000882311F088E0A4CF0E94F27E807C803CA7
:1038D00011F483E08F830E94F27E0E94F27E0E94A8
:1038E000F27ECE010E94E51981E08A83173070F4E0
:1038F0001D83DF91CF911F910F91FF90EF90DF908B
:10390000CF90BF90AF909F908F90089588E18C8367
:1039100084CF0F931F93CF93DF93EC018B0120E0B3
:1039200030E0A90169E00E94A71981110AC040E1B5
:1039300050E0B801CE01DF91CF911F910F910C940F
:10394000241B80E18C83CE010E94E51980E0DF9189
:10395000CF911F910F910895CF93C82FCB010E9453
:10396000697A81EA96E00E94697A82E996E0CC233E
:1039700011F087E996E00E94697A8AE0CF910C9471
:10398000517A0C94AAC10C94AAC14091E50221E09D
:1039900042276CE070E00C9450B94091E50221E0C0
:1039A000422764E070E00C9450B94091E50221E0B8
:1039B000422761E070E00C9450B94091E50221E0AB
:1039C000422762E070E00C9450B94091E50221E09A
:1039D000422761E070E00C9450B94091E50221E08B
:1039E000422768E070E00C9450B94091E50221E074
:1039F00042276CE070E00C9450B941E061E070E067
:103A00000C9450B94091E50221E042270C9450B942
:103A100062E070E00C9436C16CE070E00C9436C14A
:103A200064E070E00C9436C161E070E00C9436C143
:103A300061E070E00C9436C16CE070E00C9436C12B
:103A4000CF93DF938091B8159091B915891B80951C
:103A50008F7019F40E942E83F5CF8091B8158F5F77
:103A60008F70A091B8159BE4A99FD0011124FD018E
:103A7000E854F94FEF0119929A95E9F798E090838D
:103A8000A353B94F90E1EAEBF5E101900D929A95BD
:103A9000E1F72091B8159091B915291303C094E668
:103AA0009093B5158093B815DF91CF910C949277D0
:103AB000CF92DF92EF92FF920F931F93C12CD12CE4
:103AC00076018C0128E736E044E756E060E776E0CF
:103AD0008CE696E00E94A8B81F910F91FF90EF909E
:103AE000DF90CF900895CF93DF9300D000D0CDB773
:103AF000DEB784EF91E0A0E0B0E089839A83AB83E6
:103B0000BC83BE016F5F7F4F88E70E9407790F90EB
:103B10000F900F900F90DF91CF910895CF93DF9387
:103B2000CDB7DEB720E24F8158856E818D810E942E
:103B300021BDDF91CF9108956FEF8091FA050C942C
:103B40003ABF6FE17EE482E00C94C1D264E27EE48D
:103B500081E00C94C1D269E27EE480E00C94C1D291
:103B60006EE27EE483E00C94C1D20F931F9309EAC6
:103B700015E02BEA35E044E758E16BEB75E080ECAB
:103B800095E00E94BCC41F910F9108950F931F935D
:103B90000CED14E02EE535E04EEC5EE56EED74E0E4
:103BA00083EE94E00E94BCC41F910F910895CF92C0
:103BB000DF92EF92FF92CF93DF9300D000D0CDB78A
:103BC000DEB70E94A2E020E030E04AE754E40E9421
:103BD00015E820E030E0A9010E9492E76B017C012A
:103BE00020E030E0A9010E949BE02DEB37E346E0A6
:103BF00055E387FF04C02DEB37E346E055EBC701E3
:103C0000B6010E9492E769837A838B839C83CE01FD
:103C100001960E94DABD0F900F900F900F90DF91E8
:103C2000CF91FF90EF90DF90CF90089580915B014E
:103C3000882341F0609168047091690441E081E05B
:103C40000C94C4BC0895CF93DF93EC010E94E4CBA5
:103C50001B82DF91CF910895CF93DF93EC01462F24
:103C600041706C857D858E859F850E94B1C88823B3
:103C700051F0888920E2829FC00111248C509D4E12
:103C8000DF91CF91089590E080E0FACFCF93DF935A
:103C9000EB01FC012381211104C080E0DF91CF9171
:103CA00008952250223028F48FE28883198281E01F
:103CB000F5CF60E00E942C1E009779F3DC0160E0F4
:103CC00080E09EE22D91203299F0883031F49E01FF
:103CD000260F311DF90190836F5F9E01260F311D64
:103CE000AD0141505109FA014081F90140836F5FF4
:103CF0008F5F8B3039F7FE01E60FF11D1082D7CFB1
:103D00003F924F925F926F927F928F929F92AF926B
:103D1000BF92CF92DF92EF92FF920F931F93CF93B8
:103D2000DF93CDB7DEB72C970FB6F894DEBF0FBE8A
:103D3000CDBF5C01DC0159968D909C90F40181858A
:103D40009285A385B4859C01AD012F5F3F4F4F4FF6
:103D50005F4F29873A874B875C87D50114964D9032
:103D60005D906D907C90179741145104610471042B
:103D700009F459C0BFEF4B1A5B0A6B0A7B0A312C5E
:103D8000730162011D821E821F821886F4018185E3
:103D90009285A385B4852D813E814F815885281752
:103DA00039074A075B0708F056C089859A85AB85B5
:103DB000BC858C159D05AE05BF0550F482E0C82E6C
:103DC000D12CE12CF12C92E0492E512C612C712C3C
:103DD0009E012F5F3F4FB701A601C4010E94EBCAAD
:103DE0008823C9F189819A81AB81BC81892B8A2B77
:103DF0008B2B01F1260137019FEF491A590A690AF5
:103E0000790A2D813E814F8158852F5F3F4F4F4F5B
:103E10005F4F2D833E834F8358873FEFC31AD30AEA
:103E2000E30AF30AB3CF4080518062807380332469
:103E30003394A6CFC414D504E604F70411F70FEFAA
:103E40001FEF2FEF3FE0B701A601C4010E9459CA3E
:103E5000782E81111AC0712C872D2C960FB6F894EC
:103E6000DEBF0FBECDBFDF91CF911F910F91FF90AD
:103E7000EF90DF90CF90BF90AF909F908F907F900A
:103E80006F905F904F903F900895F5014481558168
:103E900066817781411551056105710539F09701FA
:103EA0008601C4010E9459CA8823A9F2D50114963B
:103EB000CD92DD92ED92FC921797332051F0D7010D
:103EC000C6010196A11DB11DF40180839183A283D7
:103ED000B383F50185899689A789B08D892B8A2BB3
:103EE0008B2B09F0B9CFC58AD68AE78AF08E8181FB
:103EF00080688183B1CF40E050E0BA010C9433CCAC
:103F00004F925F926F927F92AF92BF92CF92DF9269
:103F1000EF92FF920F931F93CF93DF931F92CDB732
:103F2000DEB78C017B015A01C22EDB0159968D91BF
:103F30009C91F801928F818FCB010E947B1F712C85
:103F4000F70180859185A285B3854189528963896E
:103F5000748984179507A607B70708F052C055E083
:103F6000B695A795979587955A95D1F7F82FFF7035
:103F7000DF2ED70113968C91823010F480E0DBC0E5
:103F800041E050E0BE016F5F7F4FC7010E945BCDF3
:103F90000197A1F7F70180859185A285B3854F969A
:103FA000A11DB11D80879187A287B387F0E2DF9EB4
:103FB000B00111246C507D4E61157105F9F2DB01E1
:103FC0008C91882341F0853E09F04CC0772029F080
:103FD00077247394B5CF71100EC08091F414909132
:103FE000F514A091F614B091F714F8018487958721
:103FF000A687B787D08ADB018C918111E9CF77241E
:1040000073948C2D8274823409F0B8CF772009F430
:10401000A2C0F801D08861E0C8010E942C1E009760
:1040200009F4ACCF20E2DC011D922A95E9F72BE0E0
:10403000F501DC0101900D922A95E1F721E238E2C9
:10404000FC01318B208B40E058E057874687338B4B
:10405000228B318F208F578B468B0E9468C881112D
:1040600009C08CCF4BE050E0C5010E94A7E9892B25
:1040700009F066CFF0E2DF9ED00111249D012C50A3
:104080003D4EF9018385817121F08C2D827109F0FB
:1040900001C1F801818D928D4091F4145091F51475
:1040A0006091F6147091F714448755876687778777
:1040B000D08AFD01EC50FD4E44885588712C612C4E
:1040C000320155244424D80155964D925D926D924B
:1040D0007C925897428D538D70E060E044295529B9
:1040E0006629772955964D935D936D937C935897E8
:1040F000D9011B962C91287109F0BEC0848D958D35
:10410000A68DB78DF801818B928BA38BB48B81E048
:1041100083838C2D8F70F80181831482158216821F
:104120001782108611861286138681E0C4FE03C0B2
:10413000C8010E94C7CC0F90DF91CF911F910F91C2
:10414000FF90EF90DF90CF90BF90AF907F906F90F7
:104150005F904F900895D70113968C9113978230FA
:1041600009F40CCF51968D919D910D90BC91A02D8D
:10417000803E9F4FAF41B10508F000CFC7010E94BC
:10418000801E882309F4FACE0E9468C8882309F4A7
:10419000F5CED7015996ED91FC915A9714964D9012
:1041A0005D906D907C901797B2E04B1A51086108B2
:1041B0007108858504C0440C551C661C771C8A95C3
:1041C000D2F786859785A089B189480E591E6A1E47
:1041D0007B1E81E08093F8144092F4145092F51401
:1041E0006092F6147092F714E4EFF2E180E092E04E
:1041F000DF019C011D9221503040E1F7DD24D39472
:10420000D7015996ED91FC918481D816C0F4809124
:10421000F9149091FA14DC01ED91FC910288F38974
:10422000E02D24EF32E1B301A2014D0D511D611DBE
:10423000711D0995882309F4A1CED394E1CF25857A
:1042400080E092E0A0E0B0E004C0880F991FAA1FB0
:10425000BB1F2A95D2F7F701418952896389748976
:10426000840F951FA61FB71F818B928BA38BB48BD6
:1042700084EF92E1D12CD6CE203161F498012F5EEB
:104280003F4F0E946ECB882329F084E0D80113961B
:104290008C933FCFD80113961C9270CEFC012381E2
:1042A00021110C94231E08952F923F924F925F92FA
:1042B0006F927F928F929F92AF92BF92CF92DF9236
:1042C000EF92FF920F931F93CF93DF93CDB7DEB79B
:1042D000C354D1090FB6F894DEBF0FBECDBF4C0159
:1042E0005B016A01222E19821C821C8E1F8E6115B1
:1042F000710521F510E0CE014C960E944E21CE01B1
:1043000001960E944E21812FCD5BDF4F0FB6F894AE
:10431000DEBF0FBECDBFDF91CF911F910F91FF90F8
:10432000EF90DF90CF90BF90AF909F908F907F9055
:104330006F905F904F903F902F900895FC01838184
:104340008111D8CFFA0180818F32A1F18B01CE018A
:1043500001967C013C0180E2382E2E019CE1490E41
:10436000511C2396EFAE23972496FFAE24972296F6
:104370003FAE229721963FAE21973FAE3EAE3DAE77
:104380003CAE3BAE3AAE39AE38AE3FAA960190E0B5
:1043900047E0D9018D91882309F447C08F3209F491
:1043A00044C08E3209F54A3009F4A4CF98E04AE0BF
:1043B0009D01EFCFFB01838182508B01823060F041
:1043C000618D728DCE014C960E94A3D18E01045E48
:1043D0001F4F882309F48ECFC6016C010196F601A8
:1043E00020812F32D1F3B3CFEAE3F1E124912223EC
:1043F00021F031968213FACF7DCF491708F47ACF96
:10440000813208F477CF8F3709F474CF3FE9380F42
:104410003A3108F420EEE7E3F0E0EC0FFD1FE90F7E
:10442000F11D820F80839F5FC3CF8FA9803209F473
:1044300061CF6901F90180812F5F3F4F8F32C9F34E
:10444000882301F121E0AE01495C5F4FB801C7014B
:104450000E94801F882309F44DCF0A151B0519F00F
:10446000C8010E94231E942D852D6E147F0431F007
:1044700023969FAD239724968FAD24978701E92E2D
:10448000F82E75CF222DAE01495C5F4FB801C401F3
:104490000E94801F182F2FCF8F929F92AF92BF92B2
:1044A000CF92DF92EF92FF92CF936B017C01B42EFB
:1044B00020E030E0A9010E949BE087FF07C08DE269
:1044C0000E94517AF7FAF094F7F8F094C0E060E0B7
:1044D00070E080E09FE3CB1541F02DEC3CEC4CEC20
:1044E0005DE30E9401E1CF5FF6CFA70196010E9434
:1044F00092E76B017C010E948EE84B015C014AE06F
:104500000E944EC7CC2379F1C501B4010E94A0E0FE
:104510009B01AC01C701B6010E9491E76B017C01D0
:104520008EE20E94517AC150F0F020E030E040E28B
:1045300051E4C701B6010E9401E16B017C010E94B8
:104540008EE84B015C014AE00E944EC7C501B401F0
:104550000E94A0E09B01AC01C701B6010E9491E757
:104560006B017C01E0CFCF91FF90EF90DF90CF9077
:10457000BF90AF909F908F900895EF92FF920F930E
:104580001F93CF937C018B01C2E44F3F09F0C4E538
:1045900080E20E94517A8C2F0E94517A8AE30E9415
:1045A000517AF701608171818281938142E00E949A
:1045B0004C228EE291E10E94697AF801608171815A
:1045C0008281938142E00E944C2262E070E080E0B0
:1045D00090E0CF911F910F91FF90EF900C9403C149
:1045E0001F93CF93DF93CDB7DEB728970FB6F8941C
:1045F000DEBF0FBECDBF182F60910B1570910C154B
:10460000072E000C880B990B0E94A2E06D837E831D
:104610008F8398876091091570910A15072E000CF9
:10462000880B990B0E94A2E069837A838B839C8319
:104630004AEFBE016B5F7F4FCE0101960E94BD2203
:104640006091040670910506072E000C880B990BEB
:104650000E94A2E06D837E838F839887609102061B
:1046600070910306072E000C880B990B0E94A2E0A4
:1046700069837A838B839C834FEFBE016B5F7F4F8F
:10468000CE0101960E94BD22609106061F3F39F0BF
:1046900085E11802F0011124EB5FFA4E608570E0AD
:1046A00086E391E10E94147B6091060670E081E34D
:1046B00091E10E94147B28960FB6F894DEBF0FBEDE
:1046C000CDBFDF91CF911F9108950F930FB70F9337
:1046D00000916E000B7F00936E0078940F930BB7E0
:1046E0000F930CB70F921F922F933F934F935F93AB
:1046F0006F937F938F939F93AF93BF93EF93FF93AA
:1047000011240E944F29FF91EF91BF91AF919F918A
:104710008F917F916F915F914F913F912F911F905A
:104720000F900CBF0F910BBF0F910460F894009392
:104730006E000F910FBF0F911895CF93DF93C5E0D7
:10474000D5E11F821E820E94AAC118865D98CEEF15
:10475000D5E01F821E820E94C61718865C98DF91E2
:10476000CF9108954F925F926F927F928F929F9216
:10477000AF92BF92EF92FF920F931F93CF93DF936D
:10478000B0E2A0E06A2F70E0AB014B0F511D5595D0
:104790004795411117C0E2E5F0E185919491282FEA
:1047A000822FDF91CF911F910F91FF90EF90BF90DB
:1047B000AF909F908F907F906F905F904F900895F3
:1047C000B42FE2CFA41711F0B41303C0EEECF0E164
:1047D000E4CF9A0121503109220F331F220F331FDA
:1047E000F901E05BFF4EE590F490F901EC5AFF4EC1
:1047F000059114918E159F051CF3A42F0817190716
:104800000CF4C0CFBC01F901EE5AFF4EC591D49112
:10481000F901EA5AFF4EA590B4906E197F09072E50
:10482000000C880B990B0E94A2E02B013C01B50102
:104830006C1B7D0B072E000C880B990B0E94A2E0CD
:104840009B01AC01C301B2010E9401E14B015C017B
:10485000B8016E197F09072E000C880B990B0E9476
:10486000A2E09B01AC01C501B4010E9415E84B0117
:104870005C01BE01DD0F880B990B0E94A2E09B0139
:10488000AC01C501B4010E9492E70E9487E8262F7F
:10489000972F86CFCF93DF93C5E0D5E18A819B81A7
:1048A0000E946CB69D838C83CEEFD5E08A819B817C
:1048B0000E94B2239D838C83A8951092E802DF9119
:1048C000CF910895EF92FF920F931F93CF93C82F2C
:1048D0007B018A018091F9058130A1F40E941E7B41
:1048E000C7010E94697A86E090E10E94697AC7FD5B
:1048F00020C08C2F0C2E000C990B0E9404B78AE06C
:104900000E94517A0E949D23A8958091FF048111F5
:1049100015C081E08093FF0480E88093F9056BEF78
:104920007FE0CF3F11F06FEF7FE040E0C8010E94D1
:10493000A07D82E090E10E94697AE1CFCF911F9142
:104940000F91FF90EF9008954F925F926F927F9238
:104950008F929F92AF92BF92CF92DF92EF92FF928F
:104960000F931F93CF93DF93EC016B014A01B22E9B
:10497000FA014080518062807380A30192016D81B1
:104980007E818F8198850E949BE08823A1F04D82D3
:104990005E826F827886AA24A39420E030E0A90189
:1049A000F40160817181828193810E9415E918165A
:1049B0000CF0A12CAC828C818230A1F0833009F400
:1049C0005AC08130C9F52D813E814F815885F6014D
:1049D00060817181828193810E949BE087FD2CC060
:1049E00082E08C83B701FF0C880B990B0E94A2E038
:1049F0009B01AC016D817E818F8198850E9491E73A
:104A00009B01AC01F60160817181828193810E94DA
:104A100015E987FD22C00E949EC16B017C019801AF
:104A2000A8EEB3E00E9437E7C60ED71EE81EF91EB7
:104A3000C882D982EA82FB82DF91CF911F910F91C8
:104A4000FF90EF90DF90CF90BF90AF909F908F90AE
:104A50007F906F905F904F9008950E949EC1088153
:104A600019812A813B81601B710B820B930B97FD8F
:104A7000E3CF83E08C8340ED50E160EE70E18B2D5D
:104A8000DF91CF911F910F91FF90EF90DF90CF902A
:104A9000BF90AF909F908F907F906F905F904F905E
:104AA0000C946224CF93DF93EC01488159816A8191
:104AB0007B8181EF9FE00E942B7F4C815D816E8125
:104AC0007F818EE296E20E942B7F488559856A8518
:104AD0007B858AE296E20E942B7F8AE0DF91CF916C
:104AE0000C94517ABC012091E0043091E104409192
:104AF000E0045091E1042417350731F481E02617D2
:104B0000370709F080E008959A01F1CF0F930FB7AE
:104B10000F9300916E000F930B7F00936E00009136
:104B20006F000D7F00936F000F930BB70F930CB7BF
:104B30000F921F922F933F934F935F936F937F93A7
:104B40008F939F93AF93BF93EF93FF9311240E9492
:104B5000DD2AFF91EF91BF91AF919F918F917F914E
:104B60006F915F914F913F912F911F900F900CBFCC
:104B70000F910BBF0F910260F89400936F000F919B
:104B800000936E000F910FBF0F9118950000000069
:104B9000000000008091E80580FF27C0459A8FEF54
:104BA000809396048091E805869580FF21C0479AFE
:104BB0008FEF809397048091E8058695869580FF16
:104BC0001AC02A988FEF809398048091E805869503
:104BD0008695869580FF12C0289A8FEF809399045E
:104BE00000000000000000000895459881E0D8CF43
:104BF000479881E0DECF2A9A81E0E5CF289881E0CE
:104C0000EDCFAF92BF92CF92DF92EF92FF920F93D0
:104C10001F93CF93DF93C9E6DBE00CE816E089E74A
:104C2000A82E8BE0B82EC12CD12C7601C3946991AB
:104C30007991899199910E94A0E0288939894A89BE
:104C40005B890E9401E10E948EE8F80161937193F3
:104C5000819391938F01C616D706E806F90610F4E2
:104C60006B017C01AC16BD0611F76FEF7FEFCB0136
:104C7000A70196010E94E3E620939C0630939D06CF
:104C800040939E0650939F06DF91CF911F910F9105
:104C9000FF90EF90DF90CF90BF90AF9008950F936B
:104CA0001F93CF93DF930DE71BE0C5EAD6E0F80131
:104CB00021913191419151918F0160E070E080E844
:104CC0009FE30E9415E86993799389939993F6E09D
:104CD000C53BDF0761F70E940AB9DF91CF911F91B1
:104CE0000F910C9401260C944F260C944F260C9493
:104CF0004F260C944F269091B8158091B9159813B2
:104D000006C08091B6069091B706892B19F00E94D3
:104D10002E83F1CF08959091B8158091B91598130D
:104D200008C08091B6069091B706892B11F40C94B7
:104D3000D3770E942E83EFCFCF93DF9320916B0226
:104D4000222379F0EC010E94B6749B01AC016885C6
:104D500079858A859B850E9491E7688779878A870C
:104D60009B87DF91CF910895CF93DF9320916B02C2
:104D7000222379F0EC010E94B6749B01AC01688596
:104D800079858A859B850E9492E7688779878A87DB
:104D90009B87DF91CF9108954F925F926F927F92A0
:104DA0008F929F92AF92BF92CF92DF92EF92FF923B
:104DB0000F931F93CF93DF93CDB7DEB76A970FB6EC
:104DC000F894DEBF0FBECDBF9A8F898F5B018A0139
:104DD000DC01D6966D917D918D919C91D9970E9421
:104DE000A0E06B017C01F50120813181428153817A
:104DF0000E9401E10E94FEE72B013C01D8012D91A8
:104E00003D914D915C91C701B6010E9401E10E9464
:104E1000FEE74B015C01C301B2010E948EE8698B81
:104E20007A8B8B8B9C8B683771058105910540F4DB
:104E300028E730E040E050E0298B3A8B4B8B5C8BCD
:104E4000C501B4010E948EE86D877E878F87988B9D
:104E5000683771058105910540F488E790E0A0E08E
:104E6000B0E08D879E87AF87B88BE98DFA8DEE5BBA
:104E7000FF4F208131814281538129833A834B83C3
:104E80005C83CA01B9010E94A2E02B013C0169893F
:104E90007A898B899C890E94A0E069877A878B87B1
:104EA0009C8720E030E0A901C301B2010E949BE091
:104EB000882309F43BC1A7019601C701B6010E94EE
:104EC00001E14B015C0129853A854B855C85CA016E
:104ED000B9010E9401E19B01AC01C501B4010E942E
:104EE00091E74B015C01A3019201C301B2010E9451
:104EF00092E79B01AC01C501B4010E9415E80E9434
:104F0000FEE70E948EE86D837E838F839887698198
:104F10007A818B819C8190958095709561957F4F6A
:104F20008F4F9F4F0E94A2E04B015C016D857E85F3
:104F30008F8598890E94A0E069837A838B839C8304
:104F400020E030E0A901C501B4010E949BE0882364
:104F500009F4F0C029813A814B815C81CA01B90111
:104F60000E9401E16D8B7E8B8F8B988FA70196013C
:104F7000C701B6010E9401E19B01AC016D897E89E8
:104F80008F89988D0E9491E76B017C01A5019401A6
:104F9000C501B4010E9492E79B01AC01C701B601B3
:104FA0000E9415E80E94BDE8A98DBA8D95968D9056
:104FB0009D90AD90BC909897750164012D813E81C4
:104FC0004F815885C21AD30AE40AF50A0E948EE876
:104FD000C61AD70AE80AF90AF7FE6EC020E030E0E8
:104FE000A901C301B2010E949BE0882309F4A6C075
:104FF000C501B4010E94A0E06B017C01A3019201F4
:10500000C301B2010E9492E79B01AC01C701B60146
:105010000E9401E16B017C0129853A854B855C8505
:10502000CA01B9010E9401E19B01AC01C701B601AF
:105030000E9491E76B017C0129813A814B815C815F
:10504000CA01B9010E9401E19B01AC01C701B6018F
:105050000E9492E76B017C0120E030E040E850E4E0
:10506000C301B2010E9401E19B01AC01C701B6017D
:105070000E9415E80E94FEE76B017C0120E030E011
:10508000A9010E9415E918161CF0C12CD12C76013B
:10509000C701B6010E948EE86D837E838F83988757
:1050A00086169706A806B90620F48D829E82AF82E6
:1050B000B886C12CD12C76018D819E81AF81B885B7
:1050C000E98DFA8D81A792A7A3A7B4A7C80ED91E10
:1050D000EA1EFB1EC5A6D6A6E7A6F0AA29893A892C
:1050E0004B895C8922AF33AF44AF55AFFE962D8517
:1050F0003E854F85588920833183428353836A9646
:105100000FB6F894DEBF0FBECDBFDF91CF911F91D8
:105110000F91FF90EF90DF90CF90BF90AF909F9056
:105120008F907F906F905F904F90089560E070E057
:10513000CB01E5CE60E070E0CB0134CF60E070E001
:10514000CB0198CF90916F0081E091FD02C080E08B
:10515000089590916F009D7F90936F000895CF9375
:10516000C82F0E94A22894E0C99F90011124F90140
:10517000ED51FB4F21513B4FD9014D915D916D9107
:105180007C91408351836283738391E09093E20426
:10519000882319F0CF910C949277CF910895CF92F4
:1051A000DF92EF92FF928091E705811105C0809117
:1051B0004606882309F46EC080917504329B64C052
:1051C00081608093750480917504339B5FC0826019
:1051D0008093750480917504349B5AC084608093D9
:1051E0007504C090D304C0FE10C08091E80580FF14
:1051F0000CC08091750480FF08C08091F805816023
:105200008093F80580E00E94AF28D12CF12CE12C8E
:10521000D701C601B695A7959795879580FF11C0D0
:105220008091E805869580FF0CC08091750481FF10
:1052300008C08091F80582608093F80581E00E94A3
:10524000AF2882E0F694E794D794C7948A95D1F773
:10525000C0FE20C08091E8058695869580FF1AC023
:10526000809146068823B1F08091750482FF12C0B8
:105270008091F80584608093F80582E0FF90EF90BC
:10528000DF90CF900C94AF288E7F9BCF8D7FA0CFE7
:105290008B7FA5CFFF90EF90DF90CF9008950F9375
:1052A0001F93CF93DF9380913E018F3708F441C065
:1052B0008F5790910D15909322059923C1F15D9A16
:1052C00090910606909321059923E1F15C9A8F5FF6
:1052D00080933E018091200591E0892780932005ED
:1052E00081110E94141980913D01C1E0C80F8530E1
:1052F0000CF0C0E0823009F4CEC034F58823D1F13F
:10530000813009F4BDC0C0933D010E94CF28809137
:10531000B6069091B706009729F001979093B706CB
:105320008093B606DF91CF911F910F9108955D98FC
:10533000C7CF90912205891708F05D9890912105BB
:10534000891728F25C98C3CF843009F4BBC00CF4F1
:10535000B5C08530C1F690911F05911102C08093B0
:105360001F0580911F05815080931F05882359F2E6
:10537000C5E0C9CF80913C018F5F80311CF48093E0
:105380003C01C1CF10923C018091E802811113C011
:105390008091051590910615909308158093071537
:1053A0008091FE059091FF05909301068093000681
:1053B00081E08093E8021092061510920515109274
:1053C000FF051092FE0500910715109108158091B8
:1053D0000B1590910C15D1E0181619062CF0809140
:1053E0000D15811101C0D0E08091540190915501BB
:1053F000081719073CF440EF50E16DEF70E180E0D1
:105400000E946224DD2371F080915201909153013A
:10541000801791073CF44FE051E16CE171E180E0CD
:105420000E94622400910406109105062091000656
:10543000309101068091E4059091E5052817390720
:105440003CF440EF50E16DEF70E18FEF0E94622479
:10545000101611060CF057CF20910006309101066E
:105460008091500190915101821793070CF04BCF1E
:105470004FE051E16CE171E18FEF0E94622443CF74
:1054800010927B0087E480937C0080917A00806496
:1054900080937A0038CF80917A0086FD26C02091D3
:1054A0007800309179008091051590910615820F52
:1054B000931F909306158093051525CF10927B00BE
:1054C00086E4E1CF80917A0086FD11C020917800BA
:1054D000309179008091FE059091FF05820F931F16
:1054E0009093FF058093FE050ECFC2E00CCFC4E081
:1054F0000ACF0E94A2281092A0061092A106109234
:10550000A2061092A30681110C94927708950F932E
:105510001F938091B8159091B915891B8F7009F46C
:1055200049C09091B515992361F0833040F48FEF15
:10553000890F29F08093B51590E080E038C0109273
:10554000B5158091B9152BE4829FC00111248854B0
:10555000994FFC01208120FDEFCF4091A006509192
:10556000A1066091A2067091A306E95BFF4F00813E
:10557000118122813381401B510B620B730B4093CD
:10558000A0065093A1066093A2067093A3062091F3
:10559000B9152F5F2F702093B6153091B915209152
:1055A000B715321304C02091B6152093B7151F917B
:1055B0000F9108950E94792ABFCF2F923F924F9268
:1055C0005F926F927F928F929F92AF92BF92CF9293
:1055D000DF92EF92FF920F931F93CF93DF9300D050
:1055E00000D0CDB7DEB78FEF9FEF90938900809307
:1055F00088000AE00983312C212C78948091DC0406
:105600009091DD04A091DE04B091DF04892B8A2BF8
:105610008B2B09F0C4C18091E2048823E1F08091D2
:10562000E0049091E1041092E204892B09F4B7C1DF
:105630001092E1041092E0041092D3049091B815F6
:105640008091B915981709F4AAC18091B9158F5F97
:105650008F708093B9158091E0049091E104892BBB
:1056600009F49DC14091D8045091D9046091DA04A5
:105670007091DB048091D4049091D504A091D6045C
:10568000B091D7040091C60410E030E020E0841B04
:10569000950BA60BB70B081719072A073B0710F441
:1056A000D901C8018A83840F951FA61FB71F809355
:1056B000D8049093D904A093DA04B093DB04E1E01A
:1056C000C0909E04D0909F04E090A004F090A104AC
:1056D0008091AE049091AF04A091B004B091B10458
:1056E000C80ED91EEA1EFB1EC092AE04D092AF04B3
:1056F000E092B004F092B104F7FC33C040919604FC
:10570000042E000C550B660B770B8091EF049091E3
:10571000F004A091F104B091F204840F951FA61F2C
:10572000B71F8093EF049093F004A093F104B0931B
:10573000F20480919A0490919B04A0919C04B091F2
:105740009D04A7019601281B390B4A0B5B0BDA015C
:10575000C9018093AE049093AF04A093B004B093BA
:10576000B1040091A2041091A3042091A4043091EB
:10577000A5048091B2049091B304A091B404B091B7
:10578000B504080F191F2A1F3B1F0093B204109382
:10579000B3042093B4043093B50437FD33C0809133
:1057A0009704082E000C990BAA0BBB0B4091F30435
:1057B0005091F4046091F5047091F604840F951FE4
:1057C000A61FB71F8093F3049093F404A093F504ED
:1057D000B093F60480919A0490919B04A0919C044C
:1057E000B0919D04B901A801481B590B6A0B7B0BB2
:1057F000DB01CA018093B2049093B304A093B40474
:10580000B093B5044091A6045091A7046091A804F8
:105810007091A9048091B6049091B704A091B80446
:10582000B091B904480F591F6A1F7B1F4093B604FB
:105830005093B7046093B8047093B90477FD33C0F4
:1058400080919804082E000C990BAA0BBB0B80903A
:10585000F7049090F804A090F904B090FA04880D31
:10586000991DAA1DBB1D8093F7049093F804A09383
:10587000F904B093FA0480919A0490919B04A0914A
:105880009C04B0919D042A013B01481A590A6A0AF6
:105890007B0AD301C2018093B6049093B704A0930E
:1058A000B804B093B9048090AA049090AB04A0907F
:1058B000AC04B090AD048091BA049091BB04A09167
:1058C000BC04B091BD04880D991DAA1DBB1D809319
:1058D000BA049093BB04A093BC04B093BD04B7FD7D
:1058E00033C040909904042C000C550866087708D2
:1058F0008090FB049090FC04A090FD04B090FE0406
:10590000840C951CA61CB71C8092FB049092FC048E
:10591000A092FD04B092FE0480909A0490909B04A3
:10592000A0909C04B0909D042C013D01481859089A
:105930006A087B08530142018092BA049092BB042A
:10594000A092BC04B092BD04E11104C0E0918400B7
:10595000F0918500F7FE5F9A37FF469A77FF2B9A02
:10596000B7FF299AE0918400F0918500E0918400CE
:10597000F0918500F7FE5F9837FF469877FF2B98E8
:10598000B7FF29985A80552021F08091840090918A
:1059900085000A8101500A83E0E0011191CE8090D8
:1059A000600190906101A0906201B0906301811448
:1059B0009104A104B10409F047C080914B06909175
:1059C0004C06009709F42FC023B1247015980000ED
:1059D000000000000000181619060CF0D7C02A9A23
:1059E00000000000000000002B9A34E03A9500000F
:1059F000E9F72B980000000000000000222309F4C2
:105A0000C7C02A9A000000000000000018161906FE
:105A10000CF0C0C080914B0690914C06019790937A
:105A20004C0680934B060E949877882309F4B8C0EF
:105A300080ED97E0A0E0B0E0809360019093610179
:105A4000A0936201B09363018091DC049091DD0426
:105A5000A091DE04B091DF04892B8A2B8B2B09F0F7
:105A600050C4E091E004F091E104309709F424C5BA
:105A70008091D8049091D904A091DA04B091DB040C
:105A80004091D4045091D5046091D6047091D7040C
:105A900084179507A607B70708F486C01092E1049B
:105AA0001092E0041092D3049091B8158091B9152A
:105AB000981709F401C58091B9158F5F8F70809395
:105AC000B91580EDC82E87E0D82EE12CF12C8091FD
:105AD000E0049091E104892B09F00BC40E94872A0D
:105AE0009093E1048093E004892B09F402C4409070
:105AF000E0045090E1045C824B82D2018C9183FFE0
:105B0000B3C2F201858D968DA78DB0A1418D528DC6
:105B1000638D748D058916892789308D0093EF0474
:105B20001093F0042093F1043093F2044093F304B3
:105B30005093F4046093F5047093F6048093F70493
:105B40009093F804A093F904B093FA0481A192A170
:105B5000A3A1B4A18093FB049093FC04A093FD0443
:105B6000B093FE041092E1041092E0041092D3046A
:105B70009091B8158091B915981709F4AFCF80911D
:105B8000B9158F5F8F708093B915A8CF2A9828CF49
:105B90002A9838CF80914B0690914C0601963FCFC2
:105BA0008FEF9FEFDC0148CF4091CF045091D0049C
:105BB0006091D1047091D204481759076A077B0796
:105BC00008F4DEC08091CB049091CC04A091CD0468
:105BD000B091CE0441A952A963A974A91127859F48
:105BE000412C969F9001A69F300DA59F200D311D41
:105BF000869F400C211D311F959F400C211D311F98
:105C0000A49F400C211D311F949F410C211F311F67
:105C10004694211F311F789F200D311D799F300D33
:105C2000112442AD53AD64AD75AD420F531F611DDC
:105C3000711D4093C7045093C8046093C9047093C6
:105C4000CA0406A917A920AD31AD04171507260708
:105C5000370740F40093C7041093C8042093C90485
:105C60003093CA044090C7045090C8046090C9049F
:105C70007090CA0421ED3FE001E00A83F9014591EB
:105C8000559165917491441555056605770570F435
:105C900076946794579447941A81110F1A832C5F56
:105CA0003F4F4DEE5FE04217530741F75A81509343
:105CB000C60460E2461651046104710428F410E23F
:105CC000412E512C612C712C70E2471A5108610849
:105CD00071084114E8E05E066104710408F42EC006
:105CE000F4E05F9E900111242F52344FF901329657
:105CF00045915491042DEE27059FB001049F610D3D
:105D00007E1F06946E1F7E1F1124AB0170E060E0C1
:105D1000F901C590D490F12CE12CC41AD50AE60AF9
:105D2000F70A8C0D9D1DAE1DBF1D8093CB04909373
:105D3000CC04A093CD04B093CE04C9CEB301A2018C
:105D400076956795579547959A012C7F2F52384F36
:105D5000F901C590D490F901329645915491142DD2
:105D60001770149F9001159F300D1124F3E03695A4
:105D70002795FA95E1F7C21AD30AF12CE12CD1CF7D
:105D80004091C2045091C3046091C4047091C50451
:105D9000481759076A077B0708F0D4C08091BE04F2
:105DA0009091BF04A091C004B091C10441A952A92F
:105DB00063A974A92227859F312D969F8001A69FF4
:105DC000100DA59F000D111D869F300D011D121F86
:105DD000959F300D011D121FA49F300D011D121F34
:105DE000949F310D021F121F3695021F121F789FBC
:105DF000000D111D799F100D112430E020E040911D
:105E0000C7045091C8046091C9047091CA04FE96F9
:105E1000408051806280738004171507260737077A
:105E200058F4401B510B620B730B44165506660663
:105E3000770610F42A013B0121ED3FE041E04A835F
:105E4000F901459155916591749144155505660583
:105E5000770570F476946794579447945A81550F58
:105E60005A832C5F3F4F6DEE7FE06217730741F757
:105E70007A817093C604E0E24E1651046104710405
:105E800028F400E2402E512C612C712CF0E24F1AC4
:105E9000510861087108411408E05006610471045A
:105EA00008F42EC014E0519E900111242F52344F5B
:105EB000F901329645915491F42DEE27F59FB001EA
:105EC000F49F610D7E1F06946E1F7E1F1124AB018F
:105ED00070E060E0F901C590D490F12CE12CC41A77
:105EE000D50AE60AF70A8C0D9D1DAE1DBF1D8093D5
:105EF000BE049093BF04A093C004B093C104E7CD47
:105F0000B301A20176956795579547959A012C7F25
:105F10002F52384FF901C590D490F901329645912E
:105F20005491042D0770049F9001059F300D11249A
:105F300013E0369527951A95E1F7C21AD30AF12C8A
:105F4000E12CD1CF8091380190913901A0913A0193
:105F5000B0913B01B7FF5DC0C6A8D7A8E0ACF1ACDB
:105F600081ED9FE021E0FC0145915591659174918F
:105F70004C155D056E057F0558F4F694E794D794AB
:105F8000C794220F04964DEE5FE04817590759F762
:105F90002093C60450E2C516D104E104F10428F4AC
:105FA00070E2C72ED12CE12CF12C60E2C61AD10888
:105FB000E108F108C11478E0D706E104F10408F41F
:105FC00031C0A4E0DA9EC00111248F52944FFC012D
:105FD000329625913491BC2D6627B39FA001B29FC4
:105FE000410D561F0694461F561F112470E060E0B5
:105FF000FC0185919491B0E0A0E0841B950BA60B69
:10600000B70B8093380190933901A0933A01B09374
:106010003B01C0903801D0903901E0903A01F090F6
:106020003B0155CDD701C601B695A79597958795A4
:106030008C7F8F52984FFC0125913491FC01329650
:1060400045915491EC2DE770E49FC001E59F900DC0
:10605000112463E0969587956A95E1F7281B390B23
:10606000C901B0E0A0E0CDCFAB81BC8155960D91C8
:106070001D912D913C91589781E001151105210545
:10608000310509F480E0EB81FC81C18CD28CE38C7A
:10609000F48CC114D104E104F10409F08260AB81F5
:1060A000BC815D964D915D916D917C91909741156C
:1060B00051056105710509F084608093D304109245
:1060C000BE041092BF041092C0041092C10410923A
:1060D000CB041092CC041092CD041092CE04EB812C
:1060E000FC8185A196A1A7A1B0A58093D40490932B
:1060F000D504A093D604B093D70444245524320188
:10610000481A590A6A0A7B0A4092AE045092AF04B8
:106110006092B0047092B1044092B2045092B30401
:106120006092B4047092B5044092B6045092B704E1
:106130006092B8047092B9044092BA045092BB04C1
:106140006092BC047092BD0441A052A063A074A0F0
:10615000440C551C661C771C000F111F221F331F97
:1061600000939E0410939F042093A0043093A104F5
:10617000CC0CDD1CEE1CFF1CC092A204D092A30428
:10618000E092A404F092A504440F551F661F771FE8
:106190004093A6045093A7046093A8047093A904A5
:1061A0004092AA045092AB046092AC047092AD0489
:1061B000880F991FAA1FBB1F80939A0490939B047A
:1061C000A0939C04B0939D041092D8041092D9041B
:1061D0001092DA041092DB0481A592A5A3A5B4A5C0
:1061E0008093CF049093D004A093D104B093D204B1
:1061F00085A596A5A7A5B0A98093C2049093C304D2
:10620000A093C404B093C50485A99091E8058917AB
:1062100021F08093E8050E94C6250E94CF284424DF
:106220004A94542C320140923801509239016092C4
:106230003A0170923B01AB81BC81DA964D915D9140
:106240006D917C91DD974093C7045093C80460938F
:10625000C9047093CA0481ED9FE0A1E0FC0105919F
:10626000159125913491041715072607370758F41F
:106270007695679557954795AA0F0496EDEEFFE042
:10628000E817F90759F7A093C60440325105610594
:10629000710520F440E250E060E070E040525109A6
:1062A000610971094115F8E05F076105710508F49E
:1062B000DAC004E0509FC00111248F52944FFC01BA
:1062C000329625913491AA27439FF001429FE10D18
:1062D000FA1F0694EA1FFA1F1124AF0170E060E074
:1062E000FC01C590D490F12CE12CC41AD50AE60A21
:1062F000F70AC092DC04D092DD04E092DE04F09252
:10630000DF0489288A288B28C9F48091DC049091C5
:10631000DD04A091DE04B091DF048A3F9105A10560
:10632000B10560F42AEF30E040E050E02093DC0457
:106330003093DD044093DE045093DF04409160010C
:106340005091610160916201709163010091DC04E0
:106350001091DD042091DE043091DF044F3F8FEF78
:1063600058076807780799F0D901C801B695A7952D
:1063700097958795481759076A077B0740F48093DC
:10638000600190936101A0936201B0936301409119
:1063900060015091610160916201709163014F3F12
:1063A0009FEF59076105710508F07DC04B835A8343
:1063B000F62FE72F8B819A81AF2FBE2F0817190771
:1063C0002A073B0710F4D901C801081B190B2A0B37
:1063D0003B0B0093DC041093DD042093DE04309328
:1063E000DF044F3FEFEF5E076E077E0761F0481B4B
:1063F000590B6A0B7B0B40936001509361016093D2
:10640000620170936301F8942091840030918500BB
:10641000205F3F4F098101500983002309F44AC0DE
:10642000280E391E2216330610F40C94FD2A3092E1
:1064300089002092880078940F900F900F900F9011
:10644000DF91CF911F910F91FF90EF90DF90CF9050
:10645000BF90AF909F908F907F906F905F904F9084
:106460003F902F900895DB01CA01B695A7959795A7
:1064700087958C7F8F52984FFC01C590D490FC017A
:106480003296259134914770429FC001439F900DF1
:106490001124A3E096958795AA95E1F7C81AD90A21
:1064A000F12CE12C26CFAFEFAB83BFEFBA83F0E046
:1064B000E0E080CF1901BBCF80EDC82E87E0D82E59
:1064C000E12CF12C0BCBFC012081318142815381E5
:1064D0006091890B70918A0B80918B0B90918C0B42
:1064E0000E9401E10E941AE96093C6157093C715D6
:1064F0008093C8159093C9159091B8158091B915DE
:1065000098130C94201D0E947B260E94A228409183
:10651000C6155091C7156091C8157091C915409363
:10652000FB045093FC046093FD047093FE048111FE
:106530000C94927708954F925F926F927F928F9210
:106540009F92AF92BF92CF92DF92EF92FF920F9302
:106550001F93CF93DF93EC018B015A01F901209136
:10656000890B30918A0B40918B0B50918C0B608181
:106570007181828193810E9401E10E941AE96B017D
:106580007C012091850B3091860B4091870B5091B7
:10659000880BF50160817181828193810E9401E104
:1065A0000E941AE94B015C012091810B3091820B12
:1065B0004091830B5091840BF8016081718182813D
:1065C00093810E9401E10E941AE92B013C01209174
:1065D0007D0B30917E0B40917F0B5091800B688139
:1065E00079818A819B810E9401E10E941AE960936E
:1065F000BA157093BB158093BC159093BD1540924E
:10660000BE155092BF156092C0157092C115809250
:10661000C2159092C315A092C415B092C515C09230
:10662000C615D092C715E092C815F092C915909181
:10663000B8158091B915981791F0DF91CF911F91FE
:106640000F91FF90EF90DF90CF90BF90AF909F9011
:106650008F907F906F905F904F900C94201D0E94C0
:106660007B260E94A2284091C2155091C3156091CB
:10667000C4157091C5150091BE151091BF152091DC
:10668000C0153091C115C090BA15D090BB15E090DF
:10669000BC15F090BD15C092EF04D092F004E092CA
:1066A000F104F092F2040093F3041093F4042093A5
:1066B000F5043093F6044093F7045093F804609384
:1066C000F9047093FA044091C6155091C715609172
:1066D000C8157091C9154093FB045093FC04609356
:1066E000FD047093FE04882391F0DF91CF911F91F8
:1066F0000F91FF90EF90DF90CF90BF90AF909F9061
:106700008F907F906F905F904F900C949277DF9175
:10671000CF911F910F91FF90EF90DF90CF90BF909E
:10672000AF909F908F907F906F905F904F90089563
:10673000CF92DF92EF92FF92CF93DF93C82F0E9408
:10674000A22894E0C99FE0011124FE01E151FB4F12
:10675000C080D180E280F38081110E949277CB5576
:10676000D94FC701B6010E94A2E0288139814A8130
:106770005B810E9401E1DF91CF91FF90EF90DF906C
:10678000CF900895CF92DF92EF92FF92CF93DF9355
:10679000C82F0E94A22894E0C99FE0011124FE01A5
:1067A000ED51FB4FC080D180E280F38081110E94C7
:1067B0009277CB55D94FC701B6010E94A2E028813C
:1067C00039814A815B810E9401E1DF91CF91FF9085
:1067D000EF90DF90CF900895CF930E94A228C82F0A
:1067E0008091B9158093B8158093B7158093B6152D
:1067F00084E68093B5150E94792A80ED93E090930A
:10680000B7068093B606C1110E94927781E080930B
:10681000E204CF910895CF93DF9324E0829FC001DB
:106820001124EC01C25AD94FFC01E651FA4F855AA6
:106830009D4FDC012D913D914D915C916081718165
:10684000828193810E9492E7688379838A839B8304
:10685000DF91CF91089580FF04C09091880490FD4E
:106860008E7F81FF05C090918804969590FD8D7F65
:1068700082FF06C0909188049695969590FD8B7F37
:106880000895EF92FF920F931F93CF93DF93CDB7AD
:10689000DEB762970FB6F894DEBF0FBECDBF0E9481
:1068A0002B34882309F43FC04FE352E082FF02C03B
:1068B0004CE352E02FE332E081FF02C025E232E0F8
:1068C00080FD2EC08FE392E05F934F933F932F9311
:1068D0009F938F938AE097E09F938F938E010F5F32
:1068E0001F4F1F930F930E9432E00E94227BC8012A
:1068F0000E94587AC8010E942DB80FB6F894DEBFE6
:106900000FBECDBF81E062960FB6F894DEBF0FBE1A
:10691000CDBFDF91CF911F910F91FF90EF90089520
:1069200087E292E0D1CF80E0EECF80918404909115
:106930008504A0918604B0918704809318019093F8
:106940001901A0931A01B0931B01809182049091C8
:106950008304909317018093160108958091180184
:1069600090911901A0911A01B0911B0180938404A8
:1069700090938504A0938604B093870480911601B8
:1069800090911701909383048093820484E690E0B1
:10699000909317018093160108954F925F926F9222
:1069A0007F928F929F92AF92BF92CF92DF92EF929F
:1069B000FF920F931F93CF93DF93CDB7DEB72C9742
:1069C0000FB6F894DEBF0FBECDBF2B013C01298767
:1069D0003A874B875C8747015801F601E080F180D8
:1069E0000281138120E030E0A901B701C8010E94B3
:1069F0009BE0882309F488C05E2D4F2D302F212F76
:106A0000852F942FA32FB22F89839A83AB83BC83C6
:106A100020E030E0A901B701C8010E949BE081118C
:106A200008C0E0905C01F0905D0100915E01109162
:106A30005F01C701D8018D839E83AF83B887A5010D
:106A4000940160917406709175068091760690911C
:106A500077060E949BE087FF0CC08092740690929C
:106A60007506A0927606B0927706CE0101960E9436
:106A7000581D40926C0650926D0660926E067092A0
:106A80006F0689859A85AB85BC8580937006909347
:106A90007106A0937206B0937306CE0105960E940C
:106AA000581DA5019401609174067091750680913E
:106AB0007606909177060E9415E9181664F4809284
:106AC000740690927506A0927606B0927706CE0173
:106AD00001960E94581D0E947B262C960FB6F894B2
:106AE000DEBF0FBECDBFDF91CF911F910F91FF9001
:106AF000EF90DF90CF90BF90AF909F908F907F905E
:106B00006F905F904F90089550E040E030E820E4AF
:106B100077CFCF92DF92EF92FF920F931F936A018C
:106B2000E0907406F0907506009176061091770655
:106B3000FB012081318142815381FC01608171819F
:106B4000828193810E94CD341F910F91FF90EF902D
:106B5000DF90CF900895CF92DF92EF92FF920F9344
:106B60001F936B01FC01E080F18002811381ECE650
:106B7000F6E024813581468157816081718182816F
:106B800093810E94CD341F910F91FF90EF90DF9081
:106B9000CF900895AF92BF92CF92DF92EF92FF9283
:106BA0000F931F93CF93DF9300D000D0CDB7DEB704
:106BB000FC01E080F18002811381611112C0A0907C
:106BC0007406B0907506C0907606D0907706950151
:106BD000A601B701C8010E949BE087FF02C07501B2
:106BE000860120E030E04AE753E4B701C8010E9483
:106BF0009BE087FD04C0E12CF12C0AE713E4C701F8
:106C0000D80189839A83AB83BC8363EC71E0CE01A6
:106C100001960E94AB350F900F900F900F90DF916F
:106C2000CF911F910F91FF90EF90DF90CF90BF9089
:106C3000AF9008958F929F92AF92BF92CF92DF92C2
:106C4000EF92FF921F93CF93DF93CDB7DEB760979C
:106C50000FB6F894DEBF0FBECDBF182F80E00E94A4
:106C600098334B015C018092760490927704A09255
:106C70007804B092790481E00E9498336B017C0122
:106C8000C0927A04D0927B04E0927C04F0927D045E
:106C900082E00E94983360937E0470937F04809317
:106CA0008004909381041D861E861F86188A89821F
:106CB0009A82AB82BC82CD82DE82EF82F8866987BF
:106CC0007A878B879C8783E00E9498336D877E87C5
:106CD0008F87988BCE0101960E949C261E3FD9F487
:106CE00080E1FE013196ACE6B6E001900D928A9506
:106CF000E1F760960FB6F894DEBF0FBECDBFDF910F
:106D0000CF911F91FF90EF90DF90CF90BF90AF9009
:106D10009F908F90089584E0189FF0011124DF0167
:106D2000A459B94F81E090E08C0F9D1FE80FF91F27
:106D300040815181628173814D935D936D937C930A
:106D40001397D7CF0C940AB92F923F924F925F922C
:106D50006F927F928F929F92AF92BF92CF92DF926B
:106D6000EF92FF920F931F93CF93DF93CDB7DEB7D0
:106D70006C970FB6F894DEBF0FBECDBF8091E702CF
:106D8000811151C18091E60281113CC18091E802DC
:106D9000811119C06C960FB6F894DEBF0FBECDBF3F
:106DA000DF91CF911F910F91FF90EF90DF90CF90E7
:106DB000BF90AF909F908F907F906F905F904F901B
:106DC0003F902F9008950E944A240E949EC14B013B
:106DD0005C010091091510910A158091580190915C
:106DE0005901801791070CF449C260910B157091FD
:106DF0000C15072E000C880B990B0E94A2E06D83E6
:106E00007E838F839887B801110F880B990B0E949E
:106E1000A2E069837A838B839C832AE0E22EF12CA3
:106E20000CE310E020E0AE014B5F5F4FBE016F5FEF
:106E30007F4F8DE695E10E94A424009109151091E1
:106E40000A158091560190915701801791070CF413
:106E5000F1C060E060930D158091011590910215CD
:106E6000A0910315B09104150097A105B10539F162
:106E7000A5019401281B390B4A0B5B0BDA01C901F0
:106E8000B7FD1DC08091FF149091001508171907D8
:106E90000CF414C280910B1590910C15009739F0E9
:106EA0000E5F1F4F0497081719070CF41DC21092AC
:106EB000011510920215109203151092041580917D
:106EC000020690910306873991050CF0E3C1809189
:106ED0001B0590911C05A0911D05B0911E05009702
:106EE000A105B10561F1A5019401281B390B4A0BDD
:106EF0005B0BDA01C901B7FD22C0809102069091B7
:106F000003062091190530911A05821793070CF496
:106F1000CDC120910406309105062115310539F0C7
:106F2000029624503109821793070CF4F0C1109295
:106F30001B0510921C0510921D0510921E058091D4
:106F4000150590911605A0911705B0911805A5019A
:106F50009401281B390B4A0B5B0BDA01C901B7FD01
:106F600019CF38E8830E33E1931EA11CB11C809227
:106F7000150590921605A0921705B092180560911C
:106F8000040670910506072E000C880B990B0E94D1
:106F9000A2E06D837E838F83988760910206709153
:106FA0000306072E000C880B990B0E94A2E0698350
:106FB0007A838B839C8382E0E82EF12C02E310E03D
:106FC0002FEFAE014B5F5F4FBE016F5F7F4F86E7D4
:106FD00095E10E94A42480910206909103069C01F1
:106FE000255031092239310508F05CC12091040691
:106FF00030910506821793070CF468C180E08093F6
:107000000606C8CE1092E6020E94EC330E947B2650
:107010008EEF0E941A360E94A2368091E8028823E1
:1070200009F4B8CED0CE41E070E060E082E490E1B7
:107030000E94A07D8091580190915901081719076D
:107040000CF007CFE0900B15F0900C15B801012E55
:10705000000C880B990B0E94A2E01B012C01E1148B
:10706000F10409F43CC1B701601B710B072E000C41
:10707000880B990B0E94A2E06B017C0120E030E0BC
:1070800040E251EC0E949BE087FD29C120E030E006
:1070900040E251E4C701B6010E9415E918160CF44C
:1070A00049C180911405811149C120910C0530918D
:1070B0000D0540910E0550910F0529873A874B87A2
:1070C0005C878091100590911105A0911205B091F7
:1070D00013058D879E87AF87B88BA20191016091C0
:1070E00000057091010580910205909103050E94B1
:1070F00091E7209116153091171540911815509170
:1071000019150E9401E129853A854B855C850E940D
:1071100091E720ED3CEC4CE45DE30E9401E1298520
:107120003A854B855C850E9492E7698B7A8B8B8BC5
:107130009C8B60930C0570930D0580930E059093C6
:107140000F0520911215309113154091141550918F
:1071500015152D8B3E8B4F8B588F2D853E854F857A
:107160005889C701B6010E9492E7762E672E89875B
:107170009D8720E030E0A9010E949BE087FDE9C0E7
:107180002D893E894F89588D60E070E08FE793E448
:107190000E9415E8698F7A8F8B8F9C8F272D362D53
:1071A00049855D850E949BE087FF06C0798C6A8CCB
:1071B0003B8D39874C8D4D87872D962DA985BD85B3
:1071C0008093100590931105A0931205B0931305B9
:1071D00020910E1530910F154091101550911115F9
:1071E000C701B6010E9401E16B017C01C092040558
:1071F000D0920505E0920605F0920705272D362D61
:1072000049855D856D897E898F89988D0E9401E110
:107210009B01AC01209308053093090540930A05B2
:1072200050930B05C701B6010E9492E729893A895C
:107230004B895C890E9492E720E030E0A9010E941E
:1072400092E76B017C0120E030E0A9010E949BE005
:1072500087FD48C020E030E04FE753E4C701B601A6
:107260000E9415E91816A4F56FE7209200053092E8
:1072700001054092020550920305ECCD40EF50E12C
:107280006DEF70E180E00E94622400910915109179
:107290000A15ABCD40EF50E16DEF70E18FEF0E942A
:1072A000622415CE109206065C9874CD44E250E13B
:1072B00063E370E18FEF0E94622441CE44E250E12B
:1072C00063E370E180E00E946224F9CD8FE797CEFE
:1072D000C701B6010E9487E875956795C6CF81E022
:1072E0008093140560E0C1CF109300150093FF1444
:1072F0000E949EC1605B7C438F4F9F4F609301153E
:10730000709302158093031590930415D8CD909334
:107310001A05809319050E949EC1605E70448D4FCE
:107320009F4F60931B0570931C0580931D059093E0
:107330001E0505CE81E08093140596CF10921405AA
:107340001D861E861F86188A19861A861B861C862D
:10735000C4CE712C612C19861D862ECF2F923F92A0
:107360004F925F926F927F928F929F92AF92BF9255
:10737000CF92DF92EF92FF920F931F93CF93DF9301
:10738000CDB7DEB7A6970FB6F894DEBF0FBECDBF60
:1073900080911E01882309F4CDC080918804C82EF5
:1073A000D12CF12CE12C80FF3CC0809020019090EA
:1073B0002101A0902201B090230120914B02309135
:1073C0004C0240914D0250914E02C501B4010E9401
:1073D00015E9181644F480924B0290924C02A09248
:1073E0004D02B0924E0280902C0190902D01A09001
:1073F0002E01B0902F0120914B0230914C02409110
:107400004D0250914E02C501B4010E949BE087FFDE
:1074100008C080924B0290924C02A0924D02B09212
:107420004E02D701C601B695A7959795879580FF1F
:107430003CC08090240190902501A0902601B0903E
:10744000270120914F0230915002409151025091FA
:107450005202C501B4010E9415E9181644F4809245
:107460004F0290925002A0925102B092520280902C
:10747000300190903101A0903201B0903301209101
:107480004F02309150024091510250915202C50179
:10749000B4010E949BE087FF08C080924F02909247
:1074A0005002A0925102B092520292E0F694E794F8
:1074B000D794C7949A95D1F7C0FE3CC0C0902801DC
:1074C000D0902901E0902A01F0902B0120915302E5
:1074D000309154024091550250915602C701B601B5
:1074E0000E9415E9181644F4C0925302D092540237
:1074F000E0925502F0925602C0903401D0903501CE
:10750000E0903601F09037012091530230915402FF
:107510004091550250915602C701B6010E949BE06E
:1075200087FF08C0C0925302D0925402E0925502E5
:10753000F09256028091680B83FD7EC02091780600
:107540003091790640917A0650917B0660915702FE
:10755000709158028091590290915A020E949BE0CA
:10756000882309F469C01091B506111161C080919A
:1075700068019091690101972091091530910A15D0
:10758000281739073CF40E94227B8FEE96E00E9478
:10759000697A11E0209178063091790640917A0657
:1075A00050917B0660915702709158028091590268
:1075B00090915A020E9491E76B017C0120E030E03B
:1075C000A9010E9415E987FF04C0F7FAF094F7F8C3
:1075D000F0942091640130916501409166015091D1
:1075E0006701C701B6010E9401E120E030E84BE3EA
:1075F00054E40E9415E91816ECF40E94227B80EDF9
:1076000096E00E94697A8091570290915802A09169
:107610005902B0915A028093780690937906A0930C
:107620007A06B0937B0687E592E00E94633204C03D
:1076300010E0B0CF1111E7CF2AE037ED43E25CE371
:10764000609118017091190180911A0190911B01AC
:107650000E9401E16B017C0160911601709117019C
:10766000072E000C880B990B0E94A2E09B01AC0135
:10767000C701B6010E9401E1698B7A8B8B8B9C8BD1
:1076800080916B02882309F46CC020916C063091C4
:107690006D0640916E0650916F0660914B0270919D
:1076A0004C0280914D0290914E020E9491E76D8BA9
:1076B0007E8B8F8B988F2091700630917106409150
:1076C00072065091730660914F0270915002809142
:1076D0005102909152020E9491E7698F7A8F8B8FAD
:1076E0009C8F2091740630917506409176065091DA
:1076F00077066091530270915402809155029091E7
:1077000056020E9491E76D8F7E8F8F8F98A32091F4
:1077100078063091790640917A0650917B06609107
:107720005702709158028091590290915A020E941A
:1077300091E76B017C0120E030E0A9016D897E8931
:107740008F89988D0E949BE081110FC020E030E06E
:10775000A901698D7A8D8B8D9C8D0E949BE0811192
:1077600004C0C12CD12C76012CC12D893E894F89B2
:10777000588DCA01B9010E9401E14B015C01298DBC
:107780003A8D4B8D5C8DCA01B9010E9401E19B01CC
:10779000AC01C501B4010E9492E74B015C012D8D43
:1077A0003E8D4F8D58A1CA01B9010E9401E19B0194
:1077B000AC01C501B4010E9492E74B015C01A70135
:1077C0009601C701B6010E9401E19B01AC01C50110
:1077D000B4010E9492E70E9453E94B015C012DEB3A
:1077E00037E346E855E30E949BE087FF0FC020E0A7
:1077F00030E0A901C701B6010E9415E94601570111
:1078000087FF04C0B7FAB094B7F8B0942DEB37E314
:1078100046E855E3C501B4010E949BE087FDDEC048
:1078200020E030E040EA51E4C501B4010E9415E8CF
:107830000E948EE81B01672B19F422242394312C1B
:10784000B10190E080E00E94A0E09B01AC0160E00B
:1078500070E080E89FE30E9415E82B013C01AC0139
:107860009B01C501B4010E9401E14B015C01A30130
:1078700092016D897E898F89988D0E9401E16D8BBF
:107880007E8B8F8B988FA3019201698D7A8D8B8D62
:107890009C8D0E9401E1698F7A8F8B8F9C8FA30151
:1078A00092016D8D7E8D8F8D98A10E9401E16D8F6B
:1078B0007E8F8F8F98A3A3019201C701B6010E940A
:1078C00001E169A37AA38BA39CA380E1ECE6F6E037
:1078D0008E010F5F1F4FD80101900D928A95E1F73D
:1078E0000E949EC12B013C0128EC420E511C611CE0
:1078F000711C0DA31EA381E0281A310809F45FC092
:107900000E949EC18B019C010419150926093709A3
:1079100037FD86C02B013C0128EC420E511C611C36
:10792000711C0E942E832D893E894F89588D698153
:107930007A818B819C810E9492E769837A838B8311
:107940009C83298D3A8D4B8D5C8D6D817E818F81DD
:1079500098850E9492E76D837E838F8398872D8D13
:107960003E8D4F8D58A169857A858B859C850E94B7
:1079700092E769877A878B879C8729A13AA14BA1D7
:107980005CA16D857E858F8598890E9492E76D87C1
:107990007E878F87988B750164018E010F5E1F4F64
:1079A0009E01235F3F4FAE01475F5F4FBE016B5F9C
:1079B0007F4F8DA19EA10E94A8B881119CCF750117
:1079C00064018E010F5E1F4F27E532E043E552E070
:1079D0006FE472E08BE492E00E94A8B880E1EBE4EF
:1079E000F2E0ACE6B6E001900D928A95E1F7A6963A
:1079F0000FB6F894DEBF0FBECDBFDF91CF911F91C0
:107A00000F91FF90EF90DF90CF90BF90AF909F903D
:107A10008F907F906F905F904F903F902F90089540
:107A20000E94A43680CFCF930E94AB358091F80599
:107A3000C82FC47082FD0CC01092F80582E00E942D
:107A40001A360E94A23681E0C11180E0CF910895DC
:107A50000E94147D882381F3F9CFCF93DF93CDB7B4
:107A6000DEB72C970FB6F894DEBF0FBECDBF0E94D5
:107A700086B90E94A2289CE0EFEEF4E0DE011196A8
:107A800001900D929A95E1F781110E949277CE01B3
:107A900001960E9452252C960FB6F894DEBF0FBEB9
:107AA000CDBFDF91CF9108952F923F924F925F9279
:107AB0006F927F928F929F92AF92BF92CF92DF92FE
:107AC000EF92FF920F931F93CF93DF9300D01F92FB
:107AD000CDB7DEB780906C0690906D06A0906E06D4
:107AE000B0906F06409070065090710660907206DC
:107AF00070907306C0907406D0907506E09076067C
:107B0000F09077060E9401260E942C1401E717E0EE
:107B100080E291E09B838A8385E6282E87E0382ED9
:107B2000198289810E940B34C8010E947473EA8112
:107B3000FB816193719381939193FB83EA83C101EC
:107B40000E947473EA81FB816087718782879387C3
:107B5000F981FF5FF9830C5F1F4F84E0280E311C11
:107B6000F330F9F60E9435770E944F26A501940163
:107B700060916C0670916D0680916E0690916F0613
:107B80000E949BE081111CC0A301920160917006CC
:107B90007091710680917206909173060E949BE02D
:107BA00081110EC0209174063091750640917606C1
:107BB00050917706C701B6010E949BE08823B9F077
:107BC0000F900F900F90DF91CF911F910F91FF9029
:107BD000EF90DF90CF90BF90AF909F908F907F906D
:107BE0006F905F904F903F902F900C942D3D0F9091
:107BF0000F900F90DF91CF911F910F91FF90EF9019
:107C0000DF90CF90BF90AF909F908F907F906F90BC
:107C10005F904F903F902F9008952F923F924F92F8
:107C20005F926F927F928F929F92AF92BF92CF920C
:107C3000DF92EF92FF920F931F93CF93DF93CDB715
:107C4000DEB7C358D1090FB6F894DEBF0FBECDBF63
:107C5000CDB6DEB641E064E070E0CE0187589F4FBC
:107C60000E9450B941E062E070E0CE0183589F4F1E
:107C70000E9450B943E050E0BE0167587F4F8BEC43
:107C800091E00E94F4E9892B31F181E08093950421
:107C90009091950481E089270FB6F894DEBE0FBE5F
:107CA000CDBECD57DF4F0FB6F894DEBF0FBECDBFB0
:107CB000DF91CF911F910F91FF90EF90DF90CF90C8
:107CC000BF90AF909F908F907F906F905F904F90FC
:107CD0003F902F900895E9961CAE1DAE1EAE1FAECC
:107CE000E99710921B1510921A15CE018F579F4FCE
:107CF0000E94FD1CADB6BEB6CF57DF4F0881C158FC
:107D0000D04010E00D5F1F4F000F111F000F111F1B
:107D10008DB79EB7801B910B0FB6F8949EBF0FBE18
:107D20008DBFEDB7FEB73196CE57DF4FF983E883AD
:107D3000C258D040801B910B0FB6F8949EBF0FBE67
:107D40008DBFEDB7FEB731964F01801B910B0FB67B
:107D5000F8949EBF0FBE8DBFEDB7FEB731967F0181
:107D6000B801CE57DF4F88819981C258D0400E9418
:107D7000021D4091E50281E0482764E070E089E758
:107D80009BE00E9450B9B801C4010E94021DB801D5
:107D9000C7010E94021D1091E502111153C0CF5777
:107DA000DF4F8881C158D04090E00296A9E6BBE041
:107DB00070E060E030E020E04DEC57E08217930780
:107DC0000CF498C0CE57DF4FE881F981C258D040FB
:107DD000E60FF71F40805180628073804D925D9264
:107DE0006D927D92821793070CF48AC0F401E60F1E
:107DF000F71F208031800281E3812101602E7E2ED9
:107E000050964D925D926D927C9253978217930794
:107E10000CF480C0F701E60FF71F2080318002814B
:107E2000E3812101602E7E2E90964D925D926D929F
:107E30007C9293972F5F3F4F6C5F7F4F24303105CB
:107E400009F0BCCF8DE99BE00E94CD1C81EA9BE04C
:107E50000E94CD1C85EA9BE00E94CD1C89EA9BE034
:107E60000E94CD1C8DEA9BE00E94CD1C41E0412781
:107E700060E170E08CE796E00E9450B9CE018B582B
:107E80009F4F0E94CD1C0FB6F894BEBE0FBEADBE74
:107E90008AEE95E00E94F51CCE0183599F4F0E9407
:107EA000D51C8E010F5F1F4FC8010E94CD1CCE0153
:107EB0008B589F4F0E94CD1CCE018B589F4F0E9424
:107EC000CD1CC8010E94FD1CCE0183599F4F0E940A
:107ED000FD1CE980AE968FADAE97E89E700111242F
:107EE000F1E0EF1AF10800F1CE018B589F4F0E948C
:107EF000CD1CF6CFFA0145905590659074906ECFE9
:107F0000EDEBF7E045905590659074901201062DC9
:107F1000E72D73CFEDEAF7E04590559065907490AA
:107F20001201062DE72D7DCF87EA95E10E94F51C11
:107F30008AE0F82EFA94CE01FF2029F08B589F4F4B
:107F40000E94CD1CF7CF81589F4F0E94FD1CCE018F
:107F500080589F4F0E94FD1CC158DF4F8881CF572A
:107F6000D040853009F049C1C058DF4F8881C058E2
:107F7000D040853009F041C18091E502811102C0F5
:107F80000E94A3768DED92E00E94ED1C85ED92E0BB
:107F90000E94ED1C4091E50281E0482764E670E014
:107FA00081E792E00E9450B9C8010E94E51CCE0111
:107FB00083599F4F0E94D51C4091E502FF24F39402
:107FC0004F2564E070E0C8010E9450B989EE95E049
:107FD0000E94E51C4091E5024F256CE070E087E0CF
:107FE00096E00E9450B94091E5024F2564E170E0AF
:107FF000C8010E9450B9F090E502F11038C08980A4
:108000009A80AB80BC80A5019401C501B4010E9497
:1080100093E981112CC080920E1590920F15A092B9
:108020001015B09211152CEA35EC47E25EE36D8134
:108030007E818F8198850E9401E160931215709373
:10804000131580931415909315152CEA35EC47E21F
:108050005EE369857A858B859C850E9415E860932F
:108060001615709317158093181590931915C8015C
:108070000E94DD1CC8010E94C51CC8010E94C51CCD
:10808000C8010E94D51CC8010E94DD1C85E0F801D2
:1080900011928A95E9F7EE24E3944F2D4E2565E081
:1080A00070E0C8010E9450B9C8010E94E51C4091CF
:1080B000E5024E2560E270E0C8010E9450B9CE0191
:1080C00083599F4F0E94E51C4091E5024E2569E0CF
:1080D00070E0C8010E9450B94091E50241110FC003
:1080E0008981809370028A819B81AC81BD8180935C
:1080F0006C0290936D02A0936E02B0936F02FF2406
:10810000F3944F2560E270E0C8010E9450B940919D
:10811000E5024F2560E470E0C8010E9450B940912B
:10812000E5024F2560E170E0C8010E9450B940911E
:10813000E5024F2560E170E0C8010E9450B9C80116
:108140000E94CD1C4091E5024F256CE070E0C80113
:108150000E9450B94091E5024F256CE670E0C801DD
:108160000E9450B919821A821B821C821D821E82B3
:108170001F82188619861A861B861C86C8010E94D3
:10818000C51C4091E5024F2568E070E0C8010E94DF
:1081900050B94091E5024F256CE070E0C8010E94A3
:1081A00050B9CE0181589F4F0E94D51CCE018359F2
:1081B0009F4F0E94CD1C80916A0690916B0681347E
:1081C000934069F41092950420911A1530911B1573
:1081D000EF968EAD9FADEF972817390719F081E024
:1081E000809395048091E502811152CD8091950490
:1081F00081114ECD0E94543D4BCDC8010E94ED1C13
:10820000CE0183599F4F0E94ED1CC158DF4FE8807B
:10821000CF57D040C058DF4F8881C058D040E89E2B
:108220007001112481E0E81AF10808F4BDCECE01F6
:108230008B589F4F0E94CD1CF5CF84E690E0909321
:108240006B0680936A0610921B1510921A150C94F7
:108250000D3ECF93DF9300D000D0CDB7DEB784EFD3
:1082600091E0A0E0B0E089839A83AB83BC83BE0138
:108270006F5F7F4F8CE30E94077986EB96E00E9448
:10828000697A86B160EB76E082FB882780F90E94EC
:10829000AC1C86B16AEA76E083FB882780F90E94ED
:1082A000AC1C86B164EA76E0829581700E94AC1CB9
:1082B000349909C00E9441790F900F900F900F9050
:1082C000DF91CF9108950E9426790F900F900F9023
:1082D0000F90DF91CF9108958091E705811104C03F
:1082E00080914606882331F062E070E080E090E003
:1082F0000C94AF770895CF93DF93CDB7DEB72C976B
:108300000FB6F894DEBF0FBECDBFA9E6BBE090E08C
:1083100080E0FC01EF53F84F4591559165917491C0
:108320004D935D936D937D93FC01EF54F84F459110
:1083300055916591749150964D935D936D937C9397
:108340005397FC01EF55F84F459155916591749104
:1083500090964D935D936D937C93939704968031A3
:108360009105B9F680E29EE4A0E0B0E08093790B3D
:1083700090937A0BA0937B0BB0937C0B80E090E8FA
:10838000ABE3B4E480939D0B90939E0BA0939F0B63
:10839000B093A00B80E090E0AAE7B4E48093A10B37
:1083A0009093A20BA093A30BB093A40B80E090E05A
:1083B000A6E9B3E48093A50B9093A60BA093A70B1B
:1083C000B093A80B1092A90B1092AA0B1092AB0BB2
:1083D0001092AC0B1092AD0B1092AE0B1092AF0B33
:1083E0001092B00B80E090E0A0E2B1E480937C06B4
:1083F00090937D06A0937E06B0937F0680E090E088
:10840000A0EAB0E48093800690938106A093820650
:10841000B09383064AE959E969E97EE3409384060B
:10842000509385066093860670938706809388062E
:1084300090938906A0938A06B0938B061092F2055A
:108440001092F3051092F4051092F5051092EE05C6
:108450001092EF051092F0051092F1051092EA05C6
:108460001092EB051092EC051092ED050E94F1764A
:108470008CE0EAE6F1E0DE01119601900D928A951A
:10848000E1F789819A81AB81BC818093A715909394
:10849000A815A093A915B093AA158D819E81AF81CF
:1084A000B8858093AB159093AC15A093AD15B093A0
:1084B000AE1589859A85AB85BC858093AF15909361
:1084C000B015A093B115B093B21584EB90E09093E2
:1084D00008068093070686E490E090930A0680934E
:1084E000090610920C0610920B0680EF90E0909314
:1084F0000E0680930D068EE690E090931006809312
:108500000F06109212061092110686E696E6A6E86D
:10851000B1E480930E1590930F15A0931015B093AE
:1085200011158CE993E5A9E4BEE3809312159093AD
:108530001315A0931415B093151580EE95EBA5EACD
:10854000B3E48093161590931715A0931815B09364
:1085500019151092700280E090E0A0EEBFE38093C6
:108560006C0290936D02A0936E02B0936F02109212
:10857000E7051092E6050E946C412C960FB6F89420
:10858000DEBF0FBECDBFDF91CF910C94543D0C9454
:108590007B413F924F925F926F927F928F929F9218
:1085A000AF92BF92CF92DF92EF92FF920F931F9301
:1085B000CF93DF9300D000D0CDB7DEB7382E80E068
:1085C00090E0A0E2B1E489839A83AB83BC83C0903E
:1085D000AF15D090B015E090B115F090B21520E035
:1085E00030E0A901C701B6010E949BE087FF0CC0E3
:1085F000A701960160E070E080E291E40E9491E7BB
:1086000069837A838B839C8360E0CE0101960E940C
:10861000CA3540906C0650906D0660906E06709062
:108620006F068090700690907106A0907206B090D0
:108630007306332089F10E94577D19821A821B82AA
:108640001C82E0907406F0907506009176061091F9
:108650007706CE0101966C01A5019401C301B20118
:108660000E94CD34309246060E946C410F900F90CC
:108670000F900F90DF91CF911F910F91FF90EF908E
:10868000DF90CF90BF90AF909F908F907F906F9032
:108690005F904F903F9008950E94147DCECF2F920F
:1086A0003F924F925F926F927F928F929F92AF9282
:1086B000BF92DF92EF92FF920F931F93CF93DF93BE
:1086C000CDB7DEB764970FB6F894DEBF0FBECDBF4F
:1086D000D82E282E312CF101E055FA4DF49082E08D
:1086E000D81234C080914606811103C081E00E94F7
:1086F000C9420E94577D81115AC181E697E00E94CC
:10870000747320E030E0A9010E949BE08823F1F01F
:108710006F2DFF0C770B880B990B0E94A2E02B01A9
:108720003C0181E697E00E9474734B015C0120E0FC
:1087300030E040EA50E40E949BE087FF1BC0812CA0
:10874000912C90EAA92E90E4B92E14C06F2DFF0C45
:10875000770B880B990B0E94A2E02B013C01C10111
:10876000880F991F880F991F875A984F0E9474731A
:108770004B015C01A3019201C501B4010E9401E11A
:108780004B015C017101EE0CFF1CEE0CFF1CC701DC
:10879000835B984F0E94747320E030E040EC5FE30D
:1087A0000E9401E1A30192010E9401E1AB01BC0121
:1087B00000E010E098018D2D0E94FFBB92E0D912DD
:1087C00030C10E94147D20E030E0A901C501B40150
:1087D0000E949BE000E010E020E431E4811118C029
:1087E000809145068460809345068091880484606A
:1087F00080938804C7018F5B984F0E9474736093C5
:1088000074067093750680937606909377063DC044
:10881000B501A40170588D2D0E94FFBBE2E0DE1669
:1088200009F4C0C0A5019401C501B4010E9492E7FA
:10883000698B7A8B8B8B9C8BF2E0DF12D0C000E0CF
:1088400010E020EC30E449895A896B897C898D2DB0
:108850000E94FFBB82E0D812F0C00E94147D80917C
:1088600045068460809345068091880484608093E7
:108870008804C7018F5B984F0E947473F701E45915
:10888000F94F60837183828393832091AF15309178
:10889000B0154091B1155091B21560917406709168
:1088A000750680917606909177060E9491E7609315
:1088B0007406709375068093760690937706F70199
:1088C000E55AFD4F10821182128213828D2D0E9473
:1088D0000B340E94A236F701E459F94F808191814F
:1088E000A281B381F701E55BFD4F80839183A28371
:1088F000B38392E0D91609F48FC08CE0E6E7F1E08B
:10890000DE01119601900D928A95E1F7E1E0F0E029
:10891000EC0FFD1FEE0DFF1D80809180A280B380C3
:1089200020E030E0A901C501B4010E949BE088234A
:10893000F1F120E030E0A901C501B4010E9415E980
:1089400087FF04C0B7FAB094B7F8B094F701E459C0
:10895000F94F7F01A5019401C301B2010E9401E119
:108960009B01AC01F70160817181828193810E943A
:1089700091E7F7016083718382839383F2E080E063
:1089800090E0A0E4B1E4DF1621F080E090E0A8E4FC
:10899000B2E48D879E87AF87B88BCE010D960E947B
:1089A000581D05C00E94577D882309F43BCF64966B
:1089B0000FB6F894DEBF0FBECDBFDF91CF911F91F0
:1089C0000F91FF90EF90DF90BF90AF909F908F90AE
:1089D0007F906F905F904F903F902F900895F1019E
:1089E000E25CF84F6491611107C00E94227B8CE128
:1089F00097E00E94697A6AE070E090E080E00E946F
:108A0000A0E09B01AC0160E070E088E492E40E9489
:108A100015E88B019C0117CF0E947A738111C7CF93
:108A20006CCF20E030E0A901C501B4010E949BE0B9
:108A300000E010E098018111EBCE81E090E0A0E031
:108A4000B0E00D2C04C0880F991FAA1FBB1F0A9409
:108A5000D2F720914506282B2093450620918804C3
:108A6000822B80938804C7018F5B984F0E94747398
:108A7000F701E459F94F60837183828393831FCF99
:108A80008091F805882319F01092F805089540E0C8
:108A900070E060E084E896E00E94A07D0F931F9351
:108AA00080915D06813019F50E949EC1009171048C
:108AB000109172042091730430917404601B710B47
:108AC000820B930B28EE33E040E050E00E94E3E697
:108AD00060916D0470916E0480916F0490917004A8
:108AE000620F731F841F951F1F910F91089560914E
:108AF0004702709148028091490290914A02D6CF74
:108B000010925D0610927104109272041092730418
:108B10001092740410924702109248021092490277
:108B200010924A0210926D0410926E0410926F041B
:108B300010927004089580915D068130F1F08230CA
:108B4000C9F40E944E4560936D0470936E04809347
:108B50006F049093700481E080935D060E949EC133
:108B600060937104709372048093730490937404FF
:108B700081E008950E948045EECF80E008950E9434
:108B8000EBB90E94E777882351F08091241782FD8A
:108B900006C085EB92E09093F7058093F6058EEA88
:108BA00092E00E9454B50C949B4580915D068150E3
:108BB000823070F410925D060E949EC1609347025D
:108BC000709348028093490290934A0281E008958D
:108BD00080E00895833B21E0920714F083EB91E05D
:108BE00090930C1580930B150C94AAC1E09163042B
:108BF000E63010F581E08E0F8093630440913006DB
:108C000050913106609132067091330690912B0697
:108C100080912C0628E0E29FF0011124ED5CFB4FCF
:108C20002091CA153091CB15318320834283538321
:108C300064837583968387830895CF93DF93EC01D4
:108C40000E94F64520E040E070E060E0CE01DF9158
:108C5000CF910C94F31720E040E070E060E08DE1EC
:108C600092E60C94F3171092A4060E949D230C9494
:108C70002B46E0916304EE2389F0E150E093630416
:108C800088E0E89FF0011124ED5CFB4F6281738165
:108C900027814681808191810C94F3170C942B4697
:108CA0007F928F929F92AF92BF92CF92DF92EF927C
:108CB000FF920F931F93CF93DF930E9475BEC091D5
:108CC0002B067C2E85E0882E8C0ED6E0DC1B85E002
:108CD000D82EDC1AEE24EA94F12C84E0C82ECC1AAB
:108CE00083E0B82EBC1A82E0A82EAC1A81E0982E40
:108CF0009C1AC11166C080912E06882309F445C0D4
:108D000080915B01882361F0672D619581E09091EE
:108D10002E06911180E024E04FE756E00E9421BD2D
:108D20008091A4068093FA05C43009F0EBC010923C
:108D3000420680912E06843009F4D1C080915B01F7
:108D40008823E1F011E080912E06843009F010E0D4
:108D50008091FA0524E6829FC001112481589F4F1B
:108D6000B7010E9474E7862F0E94C31500E09C01A2
:108D700044E656E06C2D812F0E94A971CF5FC81187
:108D8000B8CF87E080932C060EC080912806109201
:108D90002806882309F4B4CF0E94394680912D0615
:108DA000882309F4ADCFDF91CF911F910F91FF90F0
:108DB000EF90DF90CF90BF90AF909F908F907F907B
:108DC0000895C130C1F580912E068130E9F080917F
:108DD0005B018823A1F011E080912E06813009F01B
:108DE00010E080911601909117010E948E1500E00D
:108DF0009C0149E756E0692D812F0E94A97180915D
:108E0000A4068093FA05BACF80912806109228060E
:108E10008823E9F210E000E027EE33E04AE050E07A
:108E200066E171E089E796E00E9484BF80912D069B
:108E3000882369F2B8CFC23009F0C0C080912E06F5
:108E40008230C9F080915B018823C9F211E08091E2
:108E50002E06823009F010E080910B1590910C15D0
:108E60000E948E1500E09C0142E756E06A2D812F9A
:108E70000E94A97155CF8091280610922806882358
:108E800009F30E94CEBD01EC1CE123EB31E050E080
:108E900040E06BE075E182E796E00E9484BF80913C
:108EA0002D06882379F27FCF80912806109228061C
:108EB000882309F48BC00E94CEBD06EC17E12CE894
:108EC00030E050E040E064E076E08EE696E00E941C
:108ED00084BF80912D06882309F478C064CF8091E7
:108EE000280610922806882309F428CF0E94CEBDB8
:108EF00084E696E00E9442C080912D06882309F402
:108F00001DCF51CFC53091F580912E068530B9F037
:108F100080915B01882309F431CF11E080912E0606
:108F2000853009F010E080911C0190911D010E9494
:108F30008E1500E09C014FE556E06D2D1CCF809111
:108F4000280610922806882319F304EE15E127EE6F
:108F500033E04AE050E06CE171E08FE596E00E947A
:108F600084BF80912D06882399F21DCFC63009F069
:108F700005CF80912E06863091F080915B01882389
:108F800009F4FCCE81E090912E06963009F080E045
:108F900023E040E556E06D2F0E9421BDEFCE809189
:108FA000280610922806882341F384E096E50E9463
:108FB0001D4680912D06882301F3F5CEC33009F0BC
:108FC000AFCE80912E06833009F46ECF80915B0185
:108FD000882309F414CF11E080912E06833009F024
:108FE00010E080910406909105060E948E1500E025
:108FF0009C014EE656E06B2D3ACF3F924F925F9226
:109000006F927F928F929F92AF92BF92CF92DF9298
:10901000EF92FF920F931F93CF93DF93FF24F3946C
:1090200080910B1590910C15892B09F4F12C0E945D
:1090300075BEC0912B065C2E95E0692E6C0EAA249D
:10904000AA94B12C83E0E82EEC1A82E0982E9C1AA8
:1090500081E0882E8C1A4C2E419433E3C32E36E4E3
:10906000D32E86E0782E7C1AC11195C080912E06F1
:10907000882309F470C080915B01882359F081E056
:1090800090912E06911180E024E04BE456E0642D8F
:109090000E9421BD10E000E0D4E03C2E3518009382
:1090A000FA05CD131FC0F801EE0FFF1FE15EF94F67
:1090B00085919491909344068093430680912E0667
:1090C0008C1709F41EC180915B01882359F081E05F
:1090D00090912E069D1380E023E04CE256E0632D34
:1090E0000E9421BD8D2F0F5F1F4FD5E08530B9F64F
:1090F0008091040690910506892B19F4FF2009F44C
:1091000020C1C630F9F480912E06863009F40AC1D8
:1091100080915B018823B1F0DF92CF9283E296E0E9
:109120009F938F937F9281E090912E06963009F065
:1091300080E08F930E948E1D0F900F900F900F90E4
:109140000F900F9087E0FF24F394CF5FC6118CCF70
:1091500080932C060EC08091280610922806882342
:1091600009F489CF0E94394680912D06882309F49D
:1091700082CFDF91CF911F910F91FF90EF90DF9001
:10918000CF90BF90AF909F908F907F906F905F90A7
:109190004F903F900895C13009F069C080912E062C
:1091A000813009F449C080915B01882309F472CFB2
:1091B000D1E080912E06813009F0D0E080910B152E
:1091C00090910C150E948E1500E09C0144E456E03D
:1091D000682D8D2F0E94A9718091A4068093FA05B5
:1091E000C33009F057CF1092420680912E0683308B
:1091F00009F474C080915B01882309F44BCFD1E05E
:1092000080912E06833009F0D0E08091FA0524E6A3
:10921000829FC001112481589F4FB5010E9474E7BD
:10922000862F0E94C31500E09C0146E356E06E2D98
:109230008D2F0E94A9712ECF8091280610922806AA
:10924000882309F4B0CF0E94CEBD03EC1CE123EBD0
:1092500031E050E040E06BE075E184E496E00E948C
:1092600084BF80912D06882309F49DCF82CFC23020
:1092700009F0B2CF80912E068230B9F080915B0167
:10928000882309F407CFD1E080912E06823009F0BF
:10929000D0E080910406909105060E948E1500E0B2
:1092A0009C0140E456E0692D94CF809128061092ED
:1092B0002806882319F30E94CEBD06EC17E12CE89E
:1092C00030E050E040E064E076E080E496E00E9428
:1092D00084BF80912D06882389F24BCF8091280688
:1092E00010922806882309F485CF0E94CEBD86E31C
:1092F00096E00E9442C080912D06882309F47ACF1F
:1093000038CF8091280610922806882309F4DBCEF6
:1093100083EA99E40E941D4680912D06882309F472
:10932000D2CE27CF8091280610922806882309F4F0
:10933000EFCE0E94334680912D06882309F4E8CEB3
:1093400018CF86E002CF4F925F926F927F928F92FA
:109350009F92AF92BF92CF92DF92EF92FF920F93C4
:109360001F93CF93DF930091FA050E9475BEC091C1
:109370002B0610E0000F111F015E194F95E0592ECA
:109380005C0E25E0E22E26E0F22ED3E0DC1B3CE969
:10939000C32E3DE1D32E47EFA42E45E0B42E82E04C
:1093A000782E7C1A5CE2852E56E0952E81E0682EA0
:1093B0006C1A4C2E4194C11137C080912E0688231F
:1093C000B1F080915B01882359F081E090912E06E5
:1093D000911180E024E043E156E0642D0E9421BD1C
:1093E000CF5F5C12E8CF84E080932C060CC08091A4
:1093F000280610922806882321F30E94394680917E
:109400002D068823F1F2DF91CF911F910F91FF90EC
:10941000EF90DF90CF90BF90AF909F908F907F9014
:109420006F905F904F900895C13059F5F801859184
:109430009491909344068093430680912E06813048
:1094400081F080915B01882359F21F929F928F9245
:109450006F9281E090912E06913009F474C080E003
:1094600072C08091280610922806882351F38091BB
:10947000FA05682F0E943ABF80912D06882309F3D0
:10948000C2CFC23009F042C0F80185919491909307
:1094900044068093430680912E068230D1F080915D
:1094A0005B01882309F49CCFDF92CF92BF92AF92E9
:1094B0007F9281E090912E06923009F080E08F93A8
:1094C0000E948E1D0F900F900F900F900F900F9095
:1094D00087CF8091280610922806882301F30E94E6
:1094E0009C1D80912D068823D1F28DCF8091280676
:1094F000109228068823C1F06091FA058FEF0E9430
:109500003ABF80912D06882379F07DCFC33009F0D2
:1095100067CFF80185919491909344068093430618
:1095200080912E06833011F380915B01882309F42A
:1095300057CF1F92FF92EF92DF9381E090912E061A
:10954000933009F08CCF8F930E948E1D0F900F9057
:109550000F900F900F9044CFAF92BF92CF92DF92B7
:10956000EF92FF920F931F93CF93DF930E9475BEEC
:10957000C0912B0685E0B82EBC0E90EEE92E95E04A
:10958000F92ED3E0DC1B2EEEC22E25E0D22E12E007
:109590001C1B01E00C1BAC2EA194C11131C08091A9
:1095A0002E068823B1F080915B01882359F081E079
:1095B00090912E06911180E024E042EF55E06A2D53
:1095C0000E9421BDCF5FCB11E8CF84E080932C06B1
:1095D0000CC08091280610922806882321F30E944F
:1095E000394680912D068823F1F2DF91CF911F91AA
:1095F0000F91FF90EF90DF90CF90BF90AF900895C4
:10960000C13011F580912E06813079F080915B0197
:109610008823C1F281E090912E06913009F080E01C
:1096200023E047E755E2602FCBCF809128061092C8
:109630002806882359F38BE69BE40E941D468091FF
:109640002D06882319F3D1CFC23081F590912E06D3
:10965000923071F080915B01882309F4B3CF81E0EF
:10966000923009F080E020E244EE55E0612FA8CF6F
:109670008091280610922806882361F3D092F7057E
:10968000C092F60580912D06882321F3AECF8091FC
:10969000280610922806882381F0F092F705E092C0
:1096A000F60580912D06882341F09FCFC33009F045
:1096B00089CF90912E06933051F380915B018823DE
:1096C00009F480CF81E0933009F080E020E24FEC94
:1096D00055E06D2F75CFDF92EF92FF920F931F939E
:1096E000CF93DF930E9475BEC0912B0685E0E82ED4
:1096F000EC0ED4E0DC1B13E01C1B02E00C1B81E031
:10970000F82EFC1ADC2ED194C1112EC080912E06A9
:109710008823B1F080915B01882359F081E090911A
:109720002E06911180E024E048EC55E06D2D0E945A
:1097300021BDCF5FCE11E8CF85E080932C060CC011
:109740008091280610922806882321F30E9439462A
:1097500080912D068823F1F2DF91CF911F910F9117
:10976000FF90EF90DF900895C13011F580912E06A3
:10977000813079F080915B018823D9F281E090916A
:109780002E06913009F080E023E048E955E26F2D84
:10979000CECF8091280610922806882359F38BEAB1
:1097A0009DE10E941D4680912D06882319F3D4CF98
:1097B000C23009F055C080912E06823081F0809130
:1097C0005B01882309F4B5CF81E090912E06923099
:1097D00009F080E023E041E955E2602FA8CF8091B5
:1097E000280610922806882351F386EA9DE10E94FC
:1097F0001D4680912D06882311F3AECF80912E0651
:10980000833081F080915B01882309F492CF81E05D
:1098100090912E06933009F080E023E04AE855E26B
:10982000612F85CF8091280610922806882351F356
:1098300081EA9DE10E941D4680912D06882311F347
:109840008BCF8091280610922806882391F08CE710
:1098500098E10E941D4680912D06882351F07CCF0F
:10986000C33061F2C43009F064CF80912E06843099
:1098700041F380915B01882309F45BCF81E09091F3
:109880002E06943009F080E023E041E855E26D2F88
:109890004ECF0C9439462F923F924F925F926F9227
:1098A0007F928F929F92AF92BF92CF92DF92EF9270
:1098B000FF921F93CF93DF93CDB7DEB72C970FB6F0
:1098C000F894DEBF0FBECDBF1C01162F8091280675
:1098D000109228068823E1F010922A060E94394649
:1098E0002C960FB6F894DEBF0FBECDBFDF91CF919F
:1098F0001F91FF90EF90DF90CF90BF90AF909F901F
:109900008F907F906F905F904F903F902F90089531
:109910008091300690913106A0913206B0913306C5
:109920008D839E83AF83B887892B8A2B8B2B09F479
:1099300060C080911E01882309F4BDC080911F0181
:109940008111B9C0613009F494C0623009F4A2C039
:109950008090200190902101A0902201B0902301DD
:10996000C0902C01D0902D01E0902E01F0902F019D
:10997000612E712C6D817E818F8198850E94A2E07D
:109980002091120130911301409114015091150161
:109990000E9401E1D301AA0FBB1FAA0FBB1FBC8706
:1099A000AB87A459B94FBA87A9872D913D914D91A5
:1099B0005C910E9492E72B013C018D819E81AF81D9
:1099C000B885B7FF8FC0A5019401C301B2010E9401
:1099D0009BE087FD7FC0EB85FC85E459F94F408211
:1099E000518262827382812F0E94651981E0809387
:1099F0005B011092300610923106109232061092DE
:109A0000330680915B01882309F46ACFF4E01F9F3D
:109A1000C0011124FC01E459F94F825A994FDC012D
:109A20002D913D914D915C916081718182819381F5
:109A30000E9492E76B017C01C982DA82EB82FC8290
:109A40002DEC3CEC4CEC5DE3609112017091130144
:109A500080911401909115010E9415E987FD52C073
:109A6000CE0101960E949314BC01C1010E942A718B
:109A700037CF8090240190902501A0902601B090CE
:109A80002701C0903001D0903101E0903201F09078
:109A900033016ECF8090280190902901A0902A0177
:109AA000B0902B01C0903401D0903501E090360188
:109AB000F09037015DCF812C30E5932E33ECA32E4F
:109AC00037ECB32EC12C40E5D42E43ECE42E47E412
:109AD000F42E4ECFA985BA858D929D92AD92BC92FF
:109AE000139781CFA7019601C301B2010E9415E926
:109AF00018160CF070CFE985FA85C082D182E28217
:109B0000F38271CF20E030E040E251E4C701B601BA
:109B10000E9401E120E030E04AE754E40E9401E1C4
:109B20004B015C0120E030E0A901C701B6010E94B1
:109B30009BE020E030E040EA50E487FF04C020E0F2
:109B400030E040EA50ECC501B4010E9492E720E009
:109B500030E040E251E40E9415E80E9487E86B0182
:109B60007C01F7FC62C020EA36E841E050E00E9448
:109B700005E7CA01B9012AE030E040E050E00E9468
:109B800005E7605D60933406C701B60120E137E266
:109B900040E050E00E9405E78AE0882E912CA12C3D
:109BA000B12CCA01B901A50194010E9405E7605DCD
:109BB00060933506C701B60128EE33E040E050E07F
:109BC0000E9405E7CA01B901A50194010E9405E7B9
:109BD000605D609336068EE280933706C701B6015A
:109BE00024E630E040E050E00E9405E7CA01B901F8
:109BF000A50194010E9405E7605D60933806C701E6
:109C0000B601A50194010E9405E7162FCA01B9010A
:109C1000A50194010E9405E7605D60933906105D1F
:109C200010933A0684E396E01FCFF094E094D0942A
:109C3000C094C11CD11CE11CF11C6DE2A3CF62E0F9
:109C40008AE895E20C944B4C61E081E995E20C9432
:109C50004B4C60E088E995E20C944B4CCF93DF933A
:109C600000D000D0CDB7DEB780912806109228062C
:109C7000882359F010922A060E9439460F900F90BF
:109C80000F900F90DF91CF91089560913006709101
:109C90003106809132069091330661157105810578
:109CA000910561F10E94A2E020911201309113010F
:109CB00040911401509115010E9401E12091780614
:109CC0003091790640917A0650917B060E9492E786
:109CD000609378067093790680937A0690937B065A
:109CE00083E00E94651981E080935B011092300649
:109CF00010923106109232061092330680915B0169
:109D0000882309F4BBCF20911306309114064091AB
:109D1000150650911606609178067091790680912B
:109D20007A0690917B060E9491E769837A838B8300
:109D30009C83CE0101960E949314BC0181E895E2B8
:109D40000E942A719BCF2F923F924F925F926F9207
:109D50007F928F929F92AF92BF92CF92DF92EF92BB
:109D6000FF920F931F93CF93DF93CDB7DEB7ED979D
:109D70000FB6F894DEBF0FBECDBF80912F068823AB
:109D800069F18091241700E010E083FF23C087E38E
:109D900095E10E947B1F8BE1E7E3F5E1DE019196FF
:109DA00001900D928A95E1F710E000E0BE016F5F2F
:109DB0007F4FCE0181960E9454CE18163CF4CE01FE
:109DC00001960E9437C8080F111DF0CFCE01819671
:109DD0000E944E2100936B0410936C040E9475BE88
:109DE00010912B061CAF85E0810F8DAF312E319481
:109DF00085E6C82E86E1D82E97E9A92E95E0B92EE2
:109E000081E0782E711A2BE9822E25E0922E111115
:109E100013C080912E06882391F180915B018823E5
:109E200059F081E090912E06911180E024E044EAFF
:109E300055E0632D0E9421BD8091241785FF55C0F8
:109E40001130D9F480912E068130F1F180915B01BF
:109E5000882309F45BC11F929F928F927F9281E0C9
:109E600090912E06913009F080E08F930E948E1D14
:109E70000F900F900F900F900F9082E066C080912E
:109E8000280610922806882341F20E9439468091C4
:109E90002D06882311F2ED960FB6F894DEBF0FBEA3
:109EA000CDBFDF91CF911F910F91FF90EF90DF9089
:109EB000CF90BF90AF909F908F907F906F905F906A
:109EC0004F903F902F900895809128061092280679
:109ED000882309F4BBCF10922B060E94F3D1809106
:109EE0002D06882309F4B2CFD6CF83FF2DC01130C1
:109EF00021F680912E068130D1F080915B0188237C
:109F000009F404C1DF92CF92BF92AF927F9281E0B9
:109F100090912E06913009F080E08F930E948E1D63
:109F20000F900F900F900F900F900F90A6CF8091F1
:109F3000280610922806882301F30E946516809156
:109F40002D068823D1F2A7CF81E090915B01992360
:109F500009F4DDC0582E082FF12CE12C412E9CADC8
:109F6000491A802F20916B0430916C04E216F3069D
:109F700008F0CDC00113A5C087E395E10E947B1FC7
:109F8000202E25188BE1E7E3F5E1DE0191960190A3
:109F90000D928A95E1F7612CBE016F5F7F4FCE0174
:109FA00081960E9454CE18167CF4CE0101960E9430
:109FB00037C8882389F326106BC0BE016F5F7F4FBF
:109FC00080E596E00E9452C8CE0181960E944E2103
:109FD0008091241790912E0684FF78C0911366C05B
:109FE0008091280610922806882309F45FC0198200
:109FF0001C8280913A1562E575E1882311F067E3D0
:10A0000075E121E040E556E0CE0101960E94542121
:10A01000882309F43FC08BE1FE013196A7E3B5E147
:10A0200001900D928A95E1F7809124178F7D80939E
:10A030002417A0911917AA3080F481E08A0F809329
:10A0400019178BE18A9FD0011124A55FB94EE7E370
:10A05000F5E101900D928A95E1F7CE0101960E94FB
:10A060004E2110922B0682E090E0A0E0B0E08093B9
:10A07000300690933106A0933206B093330681E008
:10A0800080932D0610926A0483E080935B0103CFD6
:10A09000639482CF0E94227B60E576E081E895E0C0
:10A0A0000E9424838AE00E94517AD7CF80915B017D
:10A0B000882339F081E0911380E041E0642D0E9413
:10A0C00062BD8FEFE81AF80A0F5F4BCF911759F076
:10A0D00080915B018823A9F381E090912E06911372
:10A0E00080E040E0EBCF809128061092280688237C
:10A0F00079F380E596E00E94D9C70E942B460E9422
:10A10000EBB980912D06882319F3C5CE82E01F5F3D
:10A110009DAD91137CCE80932C06BDCE3F924F9285
:10A120005F926F927F928F929F92AF92BF92CF92E7
:10A13000DF92EF92FF920F931F93CF93DF930E94D2
:10A1400075BEC0912B063C2E85E0482E4C0E9DE836
:10A15000C92E94E0D92E09EB14E0D4E0DC1B2CE5E9
:10A16000A22E24E0B22E37EAE32E34E0F32E83E071
:10A17000782E7C1A4DE2842E44E0942E82E0682EE4
:10A180006C1A81E0582E5C1AC11139C080912E06DC
:10A190008823B9F080915B01882361F0632D61957C
:10A1A00081E090912E06911180E024E047ED54E08B
:10A1B0000E9421BDCF5FC411E7CF85E080932C06BC
:10A1C0000CC08091280610922806882319F30E945B
:10A1D000394680912D068823E9F2DF91CF911F91B6
:10A1E0000F91FF90EF90DF90CF90BF90AF909F9036
:10A1F0008F907F906F905F904F903F900895C13007
:10A2000041F580912E06813089F080915B01882391
:10A2100089F21F9281ED94E09F938F935F9281E08A
:10A2200090912E06913061F180E02AC0809128063D
:10A2300010922806882349F38FEC93E09093F7055A
:10A240008093F6050E942B4680912D068823E9F223
:10A25000C4CFC23009F064C080912E068230C9F0AC
:10A2600080915B01882309F4A5CF1F9288EC94E0CC
:10A270009F938F936F9281E090912E069230A1F67A
:10A280008F930E948E1D0F900F900F900F900F9044
:10A2900091CF8091280610922806882309F3909286
:10A2A000F7058092F6050E942B4680912D068823A3
:10A2B000B9F293CF80912E06833081F080915B01BB
:10A2C000882309F477CF1F92FF92EF927F9281E06B
:10A2D00090912E06933009F0A7CFD2CF8091280617
:10A2E00010922806882351F3B092F705A092F60544
:10A2F0000E942B4680912D06882301F36ECF80911A
:10A300002806109228068823A1F0D092F705C09263
:10A31000F6050E942B4680912D06882351F05DCFD3
:10A32000C33041F2C43009F045CF80912E0684300D
:10A3300031F380915B01882309F43CCF1F921F9376
:10A340000F93DF9381E090912E06943009F06CCF4B
:10A3500097CFDF92EF92FF920F931F93CF93DF93EC
:10A360000E94AD17082F0E9475BEC0912B06FC2ECF
:10A3700085E0E82EEC0E11E01C1BDC2ED194C111FF
:10A3800014C080912E068823F9F080915B01882308
:10A3900009F477C081E090912E06911180E024E0CD
:10A3A00043E353E06D2D0E9421BD01113DC0D2E079
:10A3B000C130D9F580912E068130D1F080915B01BA
:10A3C000811125C0D2E047C080912806109228064E
:10A3D0008823D9F20E94394680912D068823A9F25C
:10A3E000DF91CF911F910F91FF90EF90DF90089533
:10A3F0008091280610922806882301F388E793E5C8
:10A400000E941D4680912D068823C1F2E9CF81E08C
:10A4100090912E06913009F080E023E04AE253E06B
:10A42000612F0E9421BDCECFD1E0DC1314C08091FA
:10A430002E068D17B9F080915B01882361F06C2F97
:10A440006F1981E090912E069C1380E023E041E299
:10A4500053E00E9421BDCF5FCE1191CFDF5FD0933B
:10A460002C06BECF8091280610922806882319F367
:10A4700087EA94E50E941D4680912D068823D9F233
:10A48000AFCFD1E0002309F49DCFE5CF6F927F924B
:10A490008F929F92AF92BF92CF92DF92EF92FF92F4
:10A4A0000F931F93CF93DF930E9475BEC0912B062D
:10A4B0006C2E85E0782E7C0E9CE5E92E99E7F92E2E
:10A4C0002DE4C22E23E0D22ED5E0DC1B36E2A32EF3
:10A4D00039E7B32E14E01C1B03E00C1B82E0982E1E
:10A4E0009C1A81E0882E8C1AC11136C080912E06EC
:10A4F0008823B9F080915B01882361F0662D619516
:10A5000081E090912E06911180E024E045E653E031
:10A510000E9421BDCF5FC711E7CF86E080932C0654
:10A520000CC08091280610922806882319F30E94F7
:10A53000394680912D068823E9F2DF91CF911F9152
:10A540000F91FF90EF90DF90CF90BF90AF909F90D2
:10A550008F907F906F900895C13029F580912E06DD
:10A560008130A1F080915B018823A1F287E799E710
:10A570009F938F938FE593E09F938F938F9281E0CA
:10A5800090912E06913049F180E027C080912806F5
:10A5900010922806882331F30E94777980912D0646
:10A5A000882301F3CACFC23009F085C080912E06FE
:10A5B0008230E9F080915B01882309F4ABCF83E717
:10A5C0009DE19F938F9385E593E09F938F939F9257
:10A5D00081E090912E069230B9F68F930E948E1DE5
:10A5E0000F900F900F900F900F900F9093CF80913E
:10A5F0002806109228068823E9F20E94731D809194
:10A600002D068823B9F299CF80912E068330A9F0C8
:10A6100080915B01882309F47DCF81E499E79F93C2
:10A620008F9386E493E09F938F930F9381E09091B3
:10A630002E06933009F0A8CFD0CF80912806109233
:10A640002806882329F30E94417980912D068823CA
:10A65000F9F273CF80912E06843099F080915B01DE
:10A66000882309F457CFBF92AF9281E493E09F9380
:10A670008F931F9381E090912E06943009F084CF40
:10A68000ACCF8091280610922806882339F30E94C7
:10A69000267980912D06882309F34FCF80912806D3
:10A6A00010922806882399F00E945C7980912D06EB
:10A6B000882369F042CFC33009F4A6CFC43051F2E9
:10A6C000C53009F027CF80912E06853039F380916F
:10A6D0005B01882309F41ECFFF92EF92DF92CF92A5
:10A6E000DF9381E090912E06953009F04DCF75CF24
:10A6F000BF92CF92DF92EF92FF920F931F93CF936F
:10A70000DF930E9475BEC0912B0685E0C82ECC0E4B
:10A71000D4E0DC1B13E01C1B82E0F82EFC1A81E065
:10A72000E82EEC1ABC2EB194C11130C080912E06D7
:10A730008823B1F080915B01882359F081E09091EA
:10A740002E06911180E024E04FE053E06B2D0E9433
:10A7500021BDCF5FCC11E8CF85E080932C060CC0E3
:10A760008091280610922806882321F30E943946FA
:10A7700080912D068823F1F2DF91CF911F910F91E7
:10A78000FF90EF90DF90CF90BF900895C130B9F562
:10A7900080912E068130F1F080915B018823C9F20F
:10A7A000DD24D39480912E06813009F0D12C609164
:10A7B0007D0B70917E0B80917F0B9091800B0E949E
:10A7C000A41600E09C0144E053E06E2D8D2D0E9404
:10A7D000A971BFCF80912806109228068823E1F244
:10A7E0000E94CEBD49E756E26DE77BE084E093E04E
:10A7F0000E94CBBE80912D06882371F2BDCFC2305E
:10A8000009F07FC080912E068230E1F080915B01DB
:10A81000882309F49ECFDD24D39480912E068230C4
:10A8200009F0D12C6091810B7091820B8091830B88
:10A830009091840B0E94A41600E09C0149EF52E025
:10A840006F2DC4CF80912806109228068823F1F23C
:10A850000E94CEBD47E756E261E87BE089EF92E0D7
:10A860000E94CBBE80912D06882381F285CF8091F6
:10A870002E068330E1F080915B01882309F469CFD3
:10A88000DD24D39480912E06833009F0D12C609181
:10A89000850B7091860B8091870B9091880B0E949D
:10A8A000A41600E09C014EEE52E0612F8FCF809104
:10A8B0002806109228068823F1F20E94CEBD45E7B3
:10A8C00056E265E87BE08EEE92E00E94CBBE80917E
:10A8D0002D06882381F250CF8091280610922806F9
:10A8E0008823C9F00E94CEBD43E756E269E87BE0C9
:10A8F00083EE92E00E94CBBE80912D06882359F012
:10A900003BCFC33009F4B3CFC43009F022CF8091DC
:10A910002E06843009F380915B01882309F419CF56
:10A92000DD24D39480912E06843009F0D12C6091DF
:10A93000890B70918A0B80918B0B90918C0B0E94EC
:10A94000A41600E09C0143EE52E06D2F3FCF2F9202
:10A950003F924F925F926F927F928F929F92AF92AF
:10A96000BF92CF92DF92EF92FF920F931F93CF93FC
:10A97000DF93CDB7DEB729970FB6F894DEBF0FBED1
:10A98000CDBF0E9475BE10912B0685E0810F8E838E
:10A9900091E0911B9F83812F819588878CE6282EDB
:10A9A00082E0382E9CED892E95E0992EA12CB12CB9
:10A9B00026ED422E26E0522E612C712C82E0811B66
:10A9C0008987111148C080912E068823F9F0809163
:10A9D0005B01882359F081E090912E06911180E06F
:10A9E00024E04FE053E068850E9421BD8091700211
:10A9F000882309F407C1123009F461C083E01F5FA6
:10AA00009E819113DECF80932C060CC08091280686
:10AA1000109228068823D9F20E94394680912D068B
:10AA20008823A9F229960FB6F894DEBF0FBECDBFDA
:10AA3000DF91CF911F910F91FF90EF90DF90CF901A
:10AA4000BF90AF909F908F907F906F905F904F904E
:10AA50003F902F900895113049F680912E06813055
:10AA6000C9F080915B01882309F281E090912E0664
:10AA7000913009F080E09091700226ED32E0911162
:10AA800002C022ED32E001E049ED52E06F810E9408
:10AA9000A971ACCF8091700290912806109228067F
:10AAA0009923F9F281278093700283E080935B0100
:10AAB0000E942C1480912D06882399F2B3CF8091A7
:10AAC0002E068230D1F180915B01882309F496CF64
:10AAD00081E08D8380912E06823009F01D82C09026
:10AAE0006C02D0906D02E0906E02F0906F0220E058
:10AAF00030E0A901C701B6010E949BE02DEB37E3CE
:10AB000046E055EB87FD04C02DEB37E346E055E307
:10AB1000C701B6010E9492E769837A838B839C8385
:10AB2000CE0101960E94DABD00E09C0148EC52E0A3
:10AB300069858D810E94A97161CF8091280610924C
:10AB40002806882309F4BFCF0E94CEBD20E030E064
:10AB50004AE754E460916C0270916D0280916E023C
:10AB600090916F020E9401E120E030E0A9010E9473
:10AB700092E720E030E84BEB54E40E9491E70E941A
:10AB80008EE86B0191E090932D060E94F64583E0DC
:10AB900080935B0188EC92E09093270680932606D1
:10ABA000309225062092240680922006909221065B
:10ABB000A0922206B092230640921C0650921D06D7
:10ABC00060921E0670921F06F12CE12CC092300696
:10ABD000D0923106E0923206F09233068DE397E58B
:10ABE0009093CB158093CA158CE294E190931B0649
:10ABF00080931A061092190680912D06882309F475
:10AC000062CF10CF82E0FBCECF92DF92EF92FF9225
:10AC1000CF93DF938091280610922806882351F065
:10AC200010922A06DF91CF91FF90EF90DF90CF90A6
:10AC30000C94394681E080932A06809130069091E9
:10AC40003106A0913206B09133060097A105B105F7
:10AC500009F44BC02AE0289FE001299FD00D112460
:10AC6000109230061092310610923206109233067E
:10AC7000BE010D2E000C880B990B0E94A2E02091C2
:10AC8000AD063091AE064091AF065091B0060E94DD
:10AC900001E12091AF153091B0154091B11550915F
:10ACA000B2150E9492E76B017C0120E030E040E1A8
:10ACB00051EC0E9415E987FD18C020E030E040E12A
:10ACC00051E4C701B6010E949BE0181674F0CE0152
:10ACD0000E94D7C1C092AF15D092B015E092B115C5
:10ACE000F092B21582E080935B0180915B01882332
:10ACF00079F08FEA95E10E94DABDBC0189EB92E020
:10AD0000DF91CF91FF90EF90DF90CF900C942A715C
:10AD1000DF91CF91FF90EF90DF90CF9008950F9348
:10AD20001F93CF93DF93FC01EB018091300690914C
:10AD30003106A0913206B0913306B7FF08C01092D9
:10AD4000300610923106109232061092330680912E
:10AD50001C0690911D06A0911E06B0911F06409101
:10AD60003006509131066091320670913306841797
:10AD70009507A607B70744F48093300690933106F1
:10AD8000A0933206B093330680915B018823E1F0F3
:10AD900060913006709131068091320690913306B1
:10ADA0000091200610912106209122063091230661
:10ADB000600F711F821F931F0995BC0180912606A9
:10ADC000909127060E942A7180912806811108C05F
:10ADD000809119068823D1F180915B018823B1F11C
:10ADE00080912406909125060097B1F0409130069D
:10ADF0005091310660913206709133060091200621
:10AE0000109121062091220630912306400F511FF8
:10AE1000621F731FFE010995E0911A06F0911B064F
:10AE2000309741F080911906811103C08091280666
:10AE3000811109958091280610922806882331F007
:10AE4000DF91CF911F910F910C943946DF91CF91F3
:10AE50001F910F91089567E076E180E296E10C94EE
:10AE60008F566DE376E180E596E10C948F566CE6A3
:10AE700077E185E897E10C948F5664E977E187EDF7
:10AE80009DE10C948F56CF93DF93CDB7DEB78D81C4
:10AE90009091F312891768F08093F3129E01285F56
:10AEA0003F4F4E815F816AE270E088EC92E10E9440
:10AEB00062E0DF91CF9108950F931F93CF93DF93BB
:10AEC0008C016F3F19F41092F31260E02091F3129D
:10AED000862F062E000C990B2817190609F0F4F49A
:10AEE0006093F312C8010E94E8DF800F911FEC010C
:10AEF000C01BD10BCB32D1053CF00197FC01249152
:10AF0000207C2038D1F3F3CFDD27AE01B80188ECE7
:10AF100092E10E9409E0C853DD4E1882DF91CF9183
:10AF20001F910F910895DF92EF92FF920F931F935D
:10AF3000CF93DF93CDB7DEB7C658D1090FB6F894DB
:10AF4000DEBF0FBECDBFC358DF4F188219821A82F1
:10AF50001B82CD57D0408091290290912A02A09166
:10AF60002B02B0912C02CF57DF4F88839983AA839D
:10AF7000BB83C158D04084E690E090936B068093E9
:10AF80006A0610921B1510921A151092950464E02F
:10AF900070E0CE018F579F4F0E9436C180916A06A4
:10AFA00090916B06029690936B0680936A061092BE
:10AFB0001B1510921A1581E0CA57DF4F8883C658B7
:10AFC000D040CE018A579F4F0E94181D68E470E060
:10AFD00089E69BE00E9436C160E170E08CE796E074
:10AFE0000E9436C18AE097EDA3EABCE3C358DF4F65
:10AFF00088839983AA83BB83CD57D040CE018358E1
:10B000009F4F0E94101D8AEE95E00E941C1D7E013C
:10B010008DE6E80EF11C8FEFD7018C93C7010E94DB
:10B02000181D19821A821B821C828E010F5F1F4F0E
:10B03000C8010E94101D19821A821B821C82C8013D
:10B040000E94101DC358DF4F188219821A821B827A
:10B05000CD57D04083E0F70180838983CE018358A8
:10B060009F4F0E94101DC7010E94181DC8010E9419
:10B07000181D4AE0D42EDA94DD2031F0CE01835839
:10B080009F4F0E94101DF7CF87EA95E10E941C1D7B
:10B09000C358DF4F188219821A821B82CD57D040C5
:10B0A0003AE0D32EDA94DD2031F0CE0183589F4F61
:10B0B0000E94101DF7CF85E0D82ED982D701DC92EF
:10B0C000C8010E94181DC7010E94181D68E070E0A9
:10B0D0008DED92E00E9436C168E070E085ED92E06F
:10B0E0000E9436C164E670E081E792E00E9436C1BA
:10B0F00019828FEFF7018083C8010E94141DC701D8
:10B100000E94181D64E070E087EC91E00E9436C157
:10B110008091E9058983C8010E94141D6CE070E0EC
:10B1200087E096E00E9436C1198A1A8A1B8A1C8A17
:10B1300080E090E0A0E8BFE38D879E87AF87B88B63
:10B1400080910E1590910F15A0911015B0911115C9
:10B1500089839A83AB83BC832CEA35EC47E25EE3B8
:10B160006091121570911315809114159091151519
:10B170000E9415E86D837E838F8398872CEA35ECD7
:10B1800047E25EE3609116157091171580911815CE
:10B19000909119150E9401E169877A878B879C87B6
:10B1A00064E170E0C8010E9436C184E190E09A83B6
:10B1B0008983C8010E94081D8CE0E2E8F1E0D80113
:10B1C00001900D928A95E1F7C8010E940C1D8CE058
:10B1D000E2E8F1E0D80101900D928A95E1F7C8010B
:10B1E0000E940C1D1982C8010E94181D8FE790E073
:10B1F0009A838983C8010E94081DEEE8F1E0D80116
:10B2000001900D92DA94E1F765E070E0C8010E94C8
:10B2100036C11982C8010E94141D80E2E3E9F1E001
:10B22000D80101900D928A95E1F760E270E0C801C3
:10B230000E9436C1D7011C92C7010E94141D80E7ED
:10B2400092E00E94141D8CE692E00E94101DC358EB
:10B25000DF4F188219821A821B82CD57D040CE014F
:10B2600083589F4F0E94101D80E2F80111928A9529
:10B27000E9F760E270E0C8010E9436C1FE01F9966C
:10B2800088E0DF011D928A95E9F744E650E060E02E
:10B2900070E049835A836B837C834D835E836F8325
:10B2A000788783E090E0A0E0B0E089879A87AB8759
:10B2B000BC874D875E876F87788B498B5A8B6B8BEA
:10B2C0007C8B8D8B9E8BAF8BB88F898F9A8FAB8F3A
:10B2D000BC8F8D8F9E8FAF8FB8A38EE190E0A0E0E2
:10B2E000B0E089A39AA3ABA3BCA38DA39EA3AFA3F5
:10B2F000B8A789A79AA7ABA7BCA78DA79EA7AFA7FA
:10B30000B8AB89AB9AABABABBCAB8DAB9EABAFABC9
:10B31000B8AF60E470E0C8010E9436C190E1D92E58
:10B32000F8018D2D11928A95E9F760E170E0C8016E
:10B330000E9436C1D8011D92DA94E9F760E170E00D
:10B34000C8010E9436C1C358DF4F188219821A8281
:10B350001B82CD57D040CE0183589F4F0E94101DB5
:10B360002CE0D22EF8018D2D11928A95E9F76CE030
:10B3700070E0C8010E9436C18CE6D8011D928A9502
:10B38000E9F76CE670E0C8010E9436C189E894E0F4
:10B390000E940C1DF7011082118212821382148206
:10B3A00015821682178268E070E0C7010E9436C1DC
:10B3B000F7011192DA94E9F7CB57DF4F1882C5589D
:10B3C000D04080E090E0A0E4B0E4ED968CAF9DAF7B
:10B3D000AEAFBFAFED97C7010E941C1DCE018B57CA
:10B3E0009F4F0E94181DCE0187589F4F0E94101D2D
:10B3F00080919504811124C000916A0610916B061A
:10B4000080911A1590911B15D7018D939C9384E61A
:10B4100090E090936B0680936A0664E070E08BEC9A
:10B4200091E00E9436C1C7010E94081D91E00134DD
:10B43000134009F490E080919504892B8093950442
:10B4400080919504811105C060E08DE797E00E942E
:10B450005C579091950481E08927CA57DF4F0FB65A
:10B46000F894DEBF0FBECDBFDF91CF911F910F913A
:10B47000FF90EF90DF90089581E08093E5020E94B5
:10B480001D411092E50281110C941D410E947B41E7
:10B490000E9493570E94227B8DE897E00E94697A70
:10B4A00080E008950C943C5A0C9493572F923F924D
:10B4B0004F925F926F927F928F929F92AF92BF92C4
:10B4C000CF92DF92EF92FF920F931F93CF93DF9370
:10B4D00000D01F92CDB7DEB70E94AD17582E0E9444
:10B4E00075BE20912B062A83422E2B5F2B8383E08F
:10B4F000782E741803E713E022E5E22E2AE5F22EF7
:10B5000034E8C32E33E0D32E44E5A42E4AE5B42E0E
:10B5100052E9852E53E0952E82E08419898381E0DB
:10B52000382E3418242C21948A818111A0C0809156
:10B530002E06882309F477C080915B01882359F097
:10B5400081E090912E06911180E024E04AEC53E0D6
:10B55000622D0E9421BD511050C18A81833009F0B3
:10B560003CC180912E06833009F4D5C080915B01E7
:10B570008111E2C084E0682E81E0860D51104AC03E
:10B580009A8189131FC080912E06891709F407C17B
:10B5900080915B018823B1F0FF92EF92DF92CF920E
:10B5A0008A8184198F9381E090912E062A819213CB
:10B5B00080E08F930E948E1D0F900F900F900F9040
:10B5C0000F900F9082E0860D9A81891321C080919F
:10B5D0002E06891709F4F2C080915B018823C1F01F
:10B5E00087EC92E49F938F931F930F938A81841922
:10B5F0008F9381E090912E062A81921380E08F93A1
:10B600000E948E1D0F900F900F900F900F900F9033
:10B6100083E0860D9A819F5F9A832B81921384CF5A
:10B6200080932C060EC0809128061092280688234D
:10B6300009F482CF0E94394680912D06882309F4AF
:10B640007BCF0F900F900F90DF91CF911F910F91B3
:10B65000FF90EF90DF90CF90BF90AF909F908F9032
:10B660007F906F905F904F903F902F9008959A81B8
:10B67000913051F580912E068130B9F080915B01B7
:10B68000882309F468CF81E090912E06913009F06B
:10B6900080E023E048EB53E0632D0E9421BD511070
:10B6A000ACC085E094E0692E6BCF809128061092A3
:10B6B0002806882319F389EA91E50E941D468091A6
:10B6C0002D068823D9F2BDCF2A81223009F043CF3D
:10B6D00080912E06823081F080915B01882309F4ED
:10B6E0003ACF81E090912E06923009F080E023E07D
:10B6F00049EA53E06981D1CF80912806109228064B
:10B70000882351F384E096E50E941D4680912D0622
:10B71000882311F396CF809128061092280688235B
:10B7200009F424CF86E492E50E941D4680912D06FF
:10B73000882309F41BCF85CF81E090912E069330AA
:10B7400009F080E023E041EA53E0672D0E9421BD2B
:10B7500011CF8091280610922806882309F447C04B
:10B760000E94935780912D06882309F440C069CF29
:10B77000BF92AF929F928F928A8184198F9381E0BA
:10B7800090912E062A81921380E08F930E948E1D45
:10B790000F900F900F900F900F900F902CC08091F2
:10B7A000280610922806882309F4F2CE0E943C5AFB
:10B7B00080912D06882309F4EBCE43CF8091280693
:10B7C00010922806882309F407CF0E947B418091BC
:10B7D0002D06882309F400CF34CF8A81843009F004
:10B7E00060CF80912E069A81891709F4B2CF80919B
:10B7F0005B018111BDCF8A81BECE9A8184E09330F6
:10B8000009F008CFEECFCF9380912B04811109C0AE
:10B8100083EA92E0909369048093680481E08093C6
:10B820002B040E94F64520E040E070E060E086E1F5
:10B830009EE10E94F317C1E0C0932A060E947B2676
:10B8400010922A060E943946C0932A0660E089E1D8
:10B8500096E20E945C578FE992E09093F7058093FF
:10B86000F605CF9108952F923F924F925F926F927B
:10B870007F928F929F92AF92BF92CF92DF92EF9280
:10B88000FF920F931F93CF93DF9300D000D000D08F
:10B89000CDB7DEB790915D068091241782FB4424DA
:10B8A00040F8913011F44424439483FB222720F97B
:10B8B0002983212C83FF03C00E94E777282E0E9452
:10B8C00075BE80912B068D83582E8B5F8A830FE384
:10B8D00015E081E0382E351883E0782E751882E067
:10B8E00085198B8333E0E32E3CE5F32E49E6C42E25
:10B8F00045E0D42E952D91959C8358EEA52E54E0CD
:10B90000B52E6BE0862E65E0962E2D8121113EC06E
:10B9100080912E068823A9F080915B01882359F03D
:10B9200081E090912E06911180E024E045E755E0FA
:10B930006C810E9421BD442009F4ABC024E0622E3A
:10B94000C2C08091280610922806882329F30E94FD
:10B95000394680912D068823F9F226960FB6F89481
:10B96000DEBF0FBECDBFDF91CF911F910F91FF9032
:10B97000EF90DF90CF90BF90AF909F908F907F908F
:10B980006F905F904F903F902F900895442009F45E
:10B9900080C08D81813061F580912E068130D9F093
:10B9A00080915B018823A1F0FF92EF92DF92CF920A
:10B9B0003F9281E090912E06913009F080E08F93C4
:10B9C0000E948E1D0F900F900F900F900F900F9070
:10B9D00094E0692E91C08091280610922806882351
:10B9E000F9F20E94035C80912D068823C9F2B5CF3D
:10B9F0009D81923031F580912E06823099F08091B0
:10BA00005B01882361F081E090912E06923009F06D
:10BA100080E023E04EE555E06B810E9421BD84E08B
:10BA2000682E85C08091280610922806882339F355
:10BA300086EC9DE10E941D4680912D068823F9F237
:10BA40008CCF2D81233009F079CF80912E06833061
:10BA500089F080915B01882311F381E090912E069B
:10BA6000933009F080E023E049E555E0672D0E941E
:10BA700021BDAECF8091280610922806882349F375
:10BA800080E596E40E941D4680912D06882309F3E7
:10BA900064CF80915D06823029F00E94F57788237B
:10BAA00009F4CFC08D81813009F0E9C080912E0664
:10BAB000813009F49EC080915B018111A9C092E0A0
:10BAC0009E836E8063948D81681216C080912E06CD
:10BAD000861509F4E6C080915B01882369F06D81C9
:10BAE000651981E090912E062D81921380E023E06C
:10BAF0004CE255E00E9421BD81E0860D9D818913B5
:10BB000016C080912E06891709F4DCC080915B0174
:10BB1000882369F06D81651981E090912E062D8151
:10BB2000921380E023E04EE155E00E9421BD82E0C7
:10BB3000860D411055C09D81891316C080912E0637
:10BB4000891709F4D0C080915B01882369F06D8169
:10BB5000651981E090912E062D81921380E023E0FB
:10BB60004FE055E00E9421BD83E0860D9981992325
:10BB700009F4ECC0211034C02D81821314C09091BF
:10BB80002E06921709F4C0C080915B01882359F0FA
:10BB90006D81651981E02D81921380E020E24DEFE7
:10BBA00054E00E9421BD84E0860D9D81891316C05A
:10BBB00080912E06891709F4B8C080915B01882313
:10BBC00069F06D81651981E090912E062D819213A7
:10BBD00080E023E04CEE54E00E9421BD85E0860D1C
:10BBE0009D819F5F9D832A8192138FCE80932C0627
:10BBF000B4CE8091280610922806882309F45BCFE2
:10BC00000E94BF4580912D06882309F454CFA5CE0C
:10BC10008FEB95E49F938F931F930F933F9281E057
:10BC200090912E06913009F080E08F930E948E1D36
:10BC30000F900F900F900F900F900F9082E08E83D7
:10BC400040CF91E09E838E819D8189133ACF809170
:10BC50002E062E818217B1F080915B01882309F4B2
:10BC600030CF6D81651981E090912E062D81921360
:10BC700080E023E048E355E00E9421BD22CF22E08E
:10BC80002E83E1CF8091280610922806882321F385
:10BC90008CEA9AE40E941D4680912D068823E1F2E9
:10BCA0005CCE8091280610922806882309F413CFD1
:10BCB0008DEF97E40E941D4680912D06882309F49C
:10BCC0000ACF4BCE8091280610922806882309F4CB
:10BCD0001DCF86E59AE50E941D4680912D0688239A
:10BCE00009F414CF3ACE80912806109228068823B2
:10BCF00009F429CF8EE890E50E941D4680912D061B
:10BD0000882309F420CF29CE809128061092280696
:10BD1000882309F439CF9092F7058092F605809137
:10BD20002D06882309F430CF18CE80912806109272
:10BD30002806882309F441CF83EA9EE40E941D4629
:10BD400080912D06882309F438CF07CE9D81891371
:10BD500014C090912E062D81921789F080915B017D
:10BD6000882359F06D81651981E02D81921380E05F
:10BD700020E24CE455E00E9421BD84E030CF809168
:10BD8000280610922806882349F3B092F705A0925E
:10BD9000F60580912D06882309F3DFCD1092450228
:10BDA00010925A01809124178064809324178AE8A6
:10BDB00092E00E9454B560E081E992E00E945C57F5
:10BDC0000C942B464F925F926F927F928F929F922C
:10BDD000AF92BF92CF92DF92EF92FF920F931F9399
:10BDE000CF93DF9300D000D0CDB7DEB70E949EC1C5
:10BDF0004B015C01809110018F3FF1F10E949EC1C7
:10BE0000C0901804D0901904E0901A04F0901B041C
:10BE10006C197D098E099F0997FD2EC08091B81578
:10BE20009091B9158F5F8F70891731F1E0911001F2
:10BE3000E43008F0E2C024E0E29FF0011124ED5468
:10BE4000FE4F80819181A281B38189839A83AB83E4
:10BE5000BC83C12CD12C76018E010F5F1F4F28E7C8
:10BE600036E044E756E060E776E08CE696E00E9434
:10BE7000A8B88FEF809310010E94141980912604B6
:10BE800082FFC4C08091230481111DC091E0909372
:10BE90002304809145028927809328061092450249
:10BEA00083E080935B01109226040E949EC16C5037
:10BEB0007E4F8F4F9F4F6093270470932804809389
:10BEC000290490932A048091410290914202A0910A
:10BED0004302B0914402A5019401281B390B4A0B7F
:10BEE0005B0BDA01C901B7FF05C080916A048823A2
:10BEF00009F4D2C1D501C4018C599F4FAF4FBF4F38
:10BF00008093410290934202A0934302B093440273
:10BF100060912404062E000C770B77FF03C0719507
:10BF2000619571099091240480912204981371C045
:10BF3000633008F06EC01092240480912404809332
:10BF40002204643008F075C0809128068111F3C086
:10BF50008091CA159091CB158D51924641F48091F4
:10BF60001101882309F4F9C08150809311010E94C6
:10BF7000A228C090A006D090A106E090A206F09062
:10BF8000A30681110E949277D701C6013AE0B695C7
:10BF9000A795979587953A95D1F7009741E0A40723
:10BFA000B10520F08FEF9FEFA0E0B0E09695879568
:10BFB00020915B012111E3C030916A0431119AC1D3
:10BFC0008091CA159091CB158D51924609F479C193
:10BFD00080912A06811175C180911E0490911F04E1
:10BFE000A0912004B0912104881A990AAA0ABB0AD8
:10BFF000B7FC75C10E942B4672C180915C01909183
:10C000005D01A0915E01B0915F011FCF10922304EA
:10C010005ACF633009F091CF8091240487FD07C087
:10C0200081E0880F880F8093240464E086CF8FEF2F
:10C03000F8CF8091400621E030E040E050E08823D6
:10C0400009F456C0C0903C06D0903D06E0903E06F4
:10C05000F0903F06C114D104E104F104E9F170E06D
:10C0600090E080E00E94A0E020E030E040E85EE365
:10C070000E9401E12B013C01C501B4016C197D094D
:10C080008E099F090E94A0E09B01AC01C301B2018F
:10C090000E9415E820E030E04AE754E40E9401E104
:10C0A0006B017C0120E030E042E053E40E9415E99E
:10C0B00024E630E040E050E087FF12C020E030E0AE
:10C0C00040EA52E4C701B6010E9415E92AE030E0D7
:10C0D00040E050E087FF04C021E030E040E050E065
:10C0E00080923C0690923D06A0923E06B0923F069A
:10C0F000A09124040A2E000CBB0B0E942FE724E021
:10C1000030E040E050E00E9405E7809130069091D9
:10C110003106A0913206B0913306820F931FA41FFF
:10C12000B51F8093300690933106A0933206B093EA
:10C13000330610922404D501C4018856954CAF4FA4
:10C14000BF4F80931E0490931F04A0932004B093CC
:10C15000210481E080935B01FBCE8CE08093110190
:10C1600080911C0490911D04009729F001979093F1
:10C170001D0480931C0481E080935B01F8CE00973E
:10C1800041F040911C0450911D044817590708F0D4
:10C1900017CF80916A0481111DC0223038F02430FD
:10C1A00008F44CC0243011F410925B018091091600
:10C1B000811105C081E0809309160E94E7C2809139
:10C1C000D2159091D3150E94C0C281E080932F06B2
:10C1D00080936A0483E00E94E46F81E08093F0150D
:10C1E000E091CA15F091CB15099510922F06809118
:10C1F0006A04811127C0109228068091CA15909177
:10C20000CB158D51924609F0E3CE0E949EC1DC0110
:10C21000CB0188199909AA09BB09C0901C04D090C8
:10C220001D04F12CE12CC816D906EA06FB0608F01D
:10C23000C7CE90931D0480931C04C2CE81E08093EE
:10C240005B01B4CF80ED95E10E9431C691E0811190
:10C2500001C090E090936A04882369F28091CA1526
:10C260009091CB158D519246B9F40E949EC1DC018C
:10C27000CB0188199909AA09BB09C0901C04D09068
:10C280001D04F12CE12CC816D906EA06FB0620F4A1
:10C2900090931D0480931C040F900F900F900F90AB
:10C2A000DF91CF911F910F91FF90EF90DF90CF9092
:10C2B000BF90AF909F908F907F906F905F904F90C6
:10C2C000089548E9840E4AE3941EA11CB11C809293
:10C2D0001E0490921F04A0922004B0922104809129
:10C2E0006A048111D9CF80915B018130A9F6109247
:10C2F0005B01D2CF009709F46DCF43CFCF938091EC
:10C30000E903811154C0109207161092081610927A
:10C3100009161092D5151092D4151092D7151092B7
:10C32000D6151092D91581E08093D81582E28093BA
:10C33000DA151092DF151092DE15E3EFF5E121E03A
:10C3400036E18FEF81932E173F07E1F7C1E0C093ED
:10C35000F01522EE36EA3093E6152093E515C093EA
:10C36000E7151092E8151092E91590E49093EA15FC
:10C370001092EB1520EB36EA30930216209301164B
:10C3800028E031E03093D3152093D2159EE19093AD
:10C39000F71591E19093F8159CE19093F515809332
:10C3A000F4158093F3150E94E7C2C093E90381E07E
:10C3B0008093400287ED91E09093FC148093FB14EE
:10C3C0001092FE141092FD1453985B9A52985A9A48
:10C3D0003898409A0E94141910922404CF9108951D
:10C3E000FC01A081B1811C92A281B3818C918F5FED
:10C3F0008C930280F381E02D90818CE0989F800DDA
:10C400001124ECECF5E113AE84AF0895FC0180E05B
:10C410009491992331F0907C903809F08F5F319698
:10C42000F7CF0895FC0180E09191992329F0907C49
:10C430009038D1F38F5FF8CF08954F925F926F924B
:10C440007F928F929F92AF92BF92CF92DF92EF92A4
:10C45000FF920F931F93CF93DF9300D000D01F92D2
:10C46000CDB7DEB7109240068091280610922806BC
:10C470008823E9F020E040E070E060E083E39CE5A1
:10C480000F900F900F900F900F90DF91CF911F9111
:10C490000F91FF90EF90DF90CF90BF90AF909F9063
:10C4A0008F907F906F905F904F900C94F317209136
:10C4B0001601309117014091300650913106CA01A2
:10C4C000820F931F2436310509F015C447305105FA
:10C4D00044F006978A3091050CF01CC48AE090E085
:10C4E00023C406964A3F5F4FACF380912F06882302
:10C4F00009F4C0C120915E0630915F06409160064C
:10C500005091610660916C0670916D0680916E0687
:10C5100090916F060E9492E74B015C0120916206A8
:10C5200030916306409164065091650660917006F3
:10C530007091710680917206909173060E9492E745
:10C5400069837A838B839C8320916606309167068A
:10C550004091680650916906609174067091750665
:10C5600080917606909177060E9492E72B013C011C
:10C5700020E030E040E251E40E9401E120E030E0C0
:10C5800048EC52E40E9401E16B017C0120E030E0C4
:10C59000A901C301B2010E949BE020E030E040EA23
:10C5A00050EC87FD04C020E030E040EA50E4C701D1
:10C5B000B6010E9492E720E030E040E251E40E94A0
:10C5C00015E80E9487E82B013C0180E277FE09C054
:10C5D0007094609450944094411C511C611C711CD7
:10C5E0008DE28093340660E2F0E14F16F7E25F06D9
:10C5F000610471048CF0C301B20120E137E240E034
:10C6000050E00E9405E7CA01B9012AE030E040E0AD
:10C6100050E00E9405E7605D6093350660E228EE19
:10C62000421623E05206610471048CF0C301B2018A
:10C6300028EE33E040E050E00E9405E7CA01B9016E
:10C640002AE030E040E050E00E9405E7605D609342
:10C650003606C301B20124E630E040E050E00E941B
:10C6600005E76AE0C62ED12CE12CF12CCA01B901F4
:10C67000A70196010E9405E7605D60933706C3013C
:10C68000B201A70196010E9405E76D83CA01B901B5
:10C69000A70196010E9405E7CD80CC2009F454C380
:10C6A0008EE280933806605D609339062C2D205D04
:10C6B00020933A0664E376E080E194E00E94EDE99D
:10C6C00020E030E0A901C501B4010E949BE020E018
:10C6D00030E040E05FEB87FD04C020E030E040E068
:10C6E0005FE3C501B4010E9492E70E9487E8CB0195
:10C6F0000E940F15BC018BE094E00E94EDE920E060
:10C7000030E0A90169817A818B819C810E949BE044
:10C7100020E030E040E05FEB87FD04C020E030E047
:10C7200040E05FE369817A818B819C810E9492E77E
:10C730000E9487E8CB010E940F15BC0186E094E0BF
:10C740000E94EDE9409146024F774983411127C08D
:10C750000E94E777882319F180911C1790911D178B
:10C76000A0911E17B0911F170097A105B105B9F050
:10C77000BC01CD016D597F4F8F4F9F4F24E630E0B4
:10C7800040E050E00E94E3E660912017709121178D
:10C7900080912217909123170E94E3E629830E943B
:10C7A0004E45B62E872E982EA92E6D8380910F01AF
:10C7B000C9808C15C1F0C0920F0128E4C29EB0015F
:10C7C000112490E080E00E94A0E02AE037ED43E2EF
:10C7D0005CE30E9401E10E948EE860930504C110B1
:10C7E000C5C21092000480910E01CD80C81609F4D4
:10C7F00041C0B0920E016B2D782D892D9A2D20E12C
:10C800003EE040E050E00E94E3E669012CE3422E66
:10C81000512C612C712C6B2D782D892D9A2DA30113
:10C8200092010E94E3E6CA01B901A30192010E94AC
:10C83000E3E624E6C216D10408F0BFC27F936F93EB
:10C84000DF92CF9281EE91E09F938F9380EF93E000
:10C850009F938F930E9432E00FB6F894DEBF0FBE15
:10C86000CDBF85E0982F990F990F891B880F8058AD
:10C870008093EF030E949EC10091EB031091EC03A3
:10C880002091ED033091EE036B017C01C01AD10AB7
:10C89000E20AF30A9701860137FD11C02091EA03ED
:10C8A00020952093EA036A547C4F8F4F9F4F6093EB
:10C8B000EB037093EC038093ED039093EE03D09021
:10C8C000EA03D98281E00E94E46F809104168431EA
:10C8D00058F480910616883038F026E632E04CE0B5
:10C8E00068E080E50E945FC3809104168431A0F463
:10C8F00080910616823080F0E980EE2031F0809140
:10C90000A40620E332E0811102C02AEF31E042E1C7
:10C9100062E088E60E945FC3809104168C3108F0C3
:10C92000D0C0E0900915F0900A15883028F5809164
:10C930000B1590910C150E948E15FC01808193E0DF
:10C94000803229F4818192E0803209F491E043E061
:10C9500050E0491B51094E0F5F1F892F880F880F28
:10C96000981B892F67E0815F0E94677269E070E021
:10C9700080E090E00E94F56F809104168C3130F5D4
:10C9800080910616843110F1C7010E948E15FC01BA
:10C99000808193E0803229F4818192E0803209F431
:10C9A00091E043E050E0491B51094E0F5F1F892F72
:10C9B000880F880F981B892F6CE1815F0E94677236
:10C9C00069E070E080E090E00E94F56FE090020680
:10C9D000F090030680910416883028F580910406B3
:10C9E000909105060E948E15FC01808193E08032B3
:10C9F00029F4818192E0803209F491E043E050E033
:10CA0000491B51094E0F5F1F892F880F880F981BF4
:10CA1000892F67E0865A0E94677269E070E080E0C3
:10CA200090E00E94F56F809104168C3130F5809172
:10CA30000616843110F1C7010E948E15FC01808119
:10CA400093E0803229F4818192E0803209F491E010
:10CA500043E050E0491B51094E0F5F1F892F880F9B
:10CA6000880F981B892F6CE1865A0E94677269E0D3
:10CA700070E080E090E00E94F56F809104168C31A8
:10CA800000F5809106168431E0F08091A406882399
:10CA9000C1F024E6829FC001112481589F4F6FEF9F
:10CAA00070E00E9474E7CB010E948E15AC016CE12E
:10CAB00087E60E94677265E270E080E090E00E9485
:10CAC000F56F0E94E777882369F18091041684331B
:10CAD00048F5809106168A3228F107E028E04AE2FC
:10CAE0006AE280ED95E10E9468C405E022E04CE234
:10CAF00062E380ED95E10E9468C46AE08AE20E94E8
:10CB000021C46091D2157091D31582E38093EC1506
:10CB10008BE28093ED152CEE35E142E380ED95E15B
:10CB20000E94BCC280910416853340F480910616A1
:10CB3000813320F06AE486E30E9421C480910416C8
:10CB4000843368F480910616823348F002E0209125
:10CB5000050442E367E380ED95E10E9468C480919B
:10CB600004168033D8F4809106168832B8F080918C
:10CB70000004882361F040E054E060E387E30E9412
:10CB8000677265E270E080E090E00E94F56F40EF30
:10CB900053E060E38091EF030E9467728091041676
:10CBA000873208F055C0809106168F3108F450C0C6
:10CBB00083E08093071646E24093081668E570E02C
:10CBC00080E090E00E94F56F8BE08093071666E2AC
:10CBD00060930816C980CC2009F404C18BE094E06E
:10CBE0000E94267188E280930716F6E2F0930816F9
:10CBF00069E570E080E090E00E94F56F80E380934B
:10CC0000071696E2C92EC0920816D980DD2009F4D5
:10CC10000AC186E094E00E9426718DE48093071695
:10CC2000F6E2F09308166AE570E080E090E00E947A
:10CC3000F56F85E58093071686E2C82EC092081628
:10CC4000D980DD2009F412C180E194E00E942671B0
:10CC500080910416833338F5809106168B3218F1D3
:10CC600083E00E94E46F83E08093071683E3809360
:10CC7000081666E070E080E090E00E94F56F81E0C9
:10CC80000E94E46F80911601909117010E948E1509
:10CC9000AC0163E38CE00E94677265E270E080E0C3
:10CCA00090E00E94F56F80910416813408F007C16E
:10CCB00080910616863308F402C1109207168EE39F
:10CCC0008093081688EC92E10E941262898360E8E2
:10CCD00070E088EC92E10E94C870F981F53108F0AB
:10CCE000EEC060E270E080E090E00E94F56F298184
:10CCF0002F5F2983F2CF243631054CF48536910518
:10CD000004F58A30910534F48AE090E009C0843655
:10CD10009105BCF0883EE3E09E0714F087EE93E0B7
:10CD20002817390709F4E1CB909317018093160176
:10CD3000109230061092310610923206109233068D
:10CD4000D4CB84E690E0F0CF662351F08EE280935E
:10CD50003806605D6093390680E280933A06AACC7B
:10CD600080E28093390680933806F6CF498180E2CD
:10CD7000443628F0842F64E60E9446E7805D809365
:10CD80003806698190E26A3040F02AE0862F622FEF
:10CD90000E9446E70E9446E7905D9093390689819C
:10CDA0006AE00E9446E7905D90933A0668E376E079
:10CDB00080E094E00E94EDE916CD7F936F93DF92BF
:10CDC000CF9287ED91E09F938F9380EF93E09F93B5
:10CDD0008F930E9432E00FB6F894DEBF0FBECDBF36
:10CDE00086E040CD87E00E942B3480FF13C00BE02B
:10CDF00014E0F80161918F01662309F4F3CE6F32DC
:10CE00000CF06FE3062E000C770B880B990B0E9439
:10CE1000F56FEFCF8091450680FDE0CE85EF91E084
:10CE20000E94C470DFCE87E00E942B34869580FF7D
:10CE300013C006E014E0F80161918F01662309F444
:10CE4000ECCE6F320CF06FE3062E000C770B880BE4
:10CE5000990B0E94F56FEFCF80914506869580FD76
:10CE6000D8CE85EF91E00E94C470D7CE87E00E94B3
:10CE70002B348695869580FF17C080E194E09A83D5
:10CE80008983E981FA816191FA83E983662309F450
:10CE9000DFCE6F320CF06FE3062E000C770B880BA1
:10CEA000990B0E94F56FEDCF80914506869586958A
:10CEB00080FDCACE8DEE91E00E94C470C9CE0F9065
:10CEC0000F900F900F900F90DF91CF911F910F91C6
:10CED000FF90EF90DF90CF90BF90AF909F908F909A
:10CEE0007F906F905F904F900895AF92BF92CF92D6
:10CEF000DF92EF92FF920F931F93CF93DF93EC019A
:10CF00005B018A01FB01099587FD16C0C82ED12C53
:10CF1000F12CE12C2196F801C082D182E282F382C9
:10CF2000CE01DF91CF911F910F91FF90EF90DF9095
:10CF3000CF90BF90AF900895982F907E903CA9F429
:10CF40008F7190E0B0E0A0E06C017D0156E0CC0C68
:10CF5000DD1CEE1CFF1C5A95D1F7CE010196F501A0
:10CF600009958F73C82A2296D6CF982F907F903E2E
:10CF700011F58F7090E0B0E0A0E06C017D0136E02B
:10CF8000CC0CDD1CEE1CFF1C3A95D1F7CE010196AE
:10CF9000F50109958F73C82A46E0CC0CDD1CEE1C08
:10CFA000FF1C4A95D1F7CE010296F50109958F73C2
:10CFB000C82A2396B0CF982F987F903F79F5877035
:10CFC00090E0B0E0A0E06C017D0186E0CC0CDD1CBF
:10CFD000EE1CFF1C8A95D1F7CE010196F50109954B
:10CFE0008F73C82A96E0CC0CDD1CEE1CFF1C9A95B2
:10CFF000D1F7CE010296F50109958F73C82A26E074
:10D00000CC0CDD1CEE1CFF1C2A95D1F7CE0103963B
:10D01000F50109958F73C82A24967DCF982F907CAF
:10D02000903841F4807C803869F42196CE01F50176
:10D030000995F8CF8E7F8D3F28F02196CE01F5011E
:10D040000995F8CFC12CD12C760165CFAF92BF9254
:10D05000CF92DF92EF92FF920F931F93CF93DF93C4
:10D0600000D000D0CDB7DEB77C01062F6A01122FA9
:10D0700086E0A82EB12C11160CF040C0AE014F5F17
:10D080005F4F60EC77E1C7010E9475677C016981A1
:10D090007A818B819C81611571058105910571F102
:10D0A0006D3371058105910509F450C06E37710526
:10D0B0008105910509F44AC06A327105810591051F
:10D0C00069F507FF12C08DEC91E00E3F11F089EC7D
:10D0D00091E026E01202B00111240E94667066E021
:10D0E00070E00E9474E7161B61C065E470E080E0A8
:10D0F00090E00E94F56F115059F510E0812F0F90CC
:10D100000F900F900F90DF91CF911F910F91FF9093
:10D11000EF90DF90CF90BF90AF900895643271058B
:10D120008105910579F4C114D10461F026E0120261
:10D13000B0011124C6010E946670B5010E9474E717
:10D14000161B99CF0E94F56F115095CF07FDBBCFED
:10D1500061E089819A81AB81BC81CD97A105B10540
:10D1600009F460E0600F6A30ACF01150862F6AE07D
:10D170000E9452E7092F682F880F770B605D7F4F61
:10D18000072E000C880B990B0E94F56F112309F4F0
:10D19000B4CF602F062E000C770B605D7F4F072EFB
:10D1A000000C880B990B0E94F56F1150112309F4A4
:10D1B000A4CF86E01802B0011124C7010E94667056
:10D1C00066E070E00E9474E7161B98CF119800008B
:10D1D000000087FD52C0419800000000119A000035
:10D1E000000011980000000086FD53C04198000027
:10D1F0000000119A0000000011980000000085FD59
:10D2000046C0419800000000119A000000001198EB
:10D210000000000084FD39C0419800000000119A10
:10D220000000000011980000000083FD2CC0419810
:10D2300000000000119A000000001198000000009A
:10D2400082FD1FC0419800000000119A00000000FC
:10D2500011980000000081FD12C0419800000000FC
:10D26000119A000000001198000000004198000091
:10D270000000119A000000000895419AADCF419A34
:10D28000EDCF419AE0CF419AD3CF419AC6CF419A90
:10D29000B9CF419AACCF90E080E00895CF93DF936F
:10D2A000DB01F9019C919130C1F0943080F09450F1
:10D2B0009C938830D1F480819181009771F001971F
:10D2C00091838083480F591FEA01188206C08C356C
:10D2D00039F49C5F9C93943041F4DF91CF91089591
:10D2E0008B3339F781E08C93F8CF20813181B901FC
:10D2F0006F5F7F4F71836083420F531FEA01888302
:10D30000808191818F3591056CF7E7CF0F931F9343
:10D3100081E0009120171091211720912217309160
:10D32000231740911C1750911D1760911E17709183
:10D330001F17041715072607370708F480E01F9109
:10D340000F910895282F90916C05833021F495FD5D
:10D350000FC094FD0FC0892F90E0B0E0A0E004C0A2
:10D36000B695A795979587952A95D2F781700895D8
:10D3700081E0089580E008952F923F924F925F924E
:10D380006F927F928F929F92AF92BF92CF92DF92D5
:10D39000EF92FF920F931F93CF93DF93CDB7DEB73A
:10D3A0002E970FB6F894DEBF0FBECDBFE82ED62E57
:10D3B000042F122F282F30E03C872B87462F50E078
:10D3C0005A87498765E0F62EF29EC001F39E900DC4
:10D3D00011249E878D87FA01E80FF91FEE0FFF1FBA
:10D3E000EE0FFF1FEF58FD4F6081718182819381A5
:10D3F0009B01AC010E9493E9882309F434C1E00E3B
:10D40000612F6D0DFE9CF0011124A985BA85AE0F28
:10D41000BF1FAA0FBB1FAA0FBB1FAF58BD4FAC90B9
:10D420001196BC9011971296CC9012971396DC909F
:10D43000E00EFE9CA0011124A985BA85A40FB51F9A
:10D44000AA0FBB1FAA0FBB1FAF58BD4FEC90119680
:10D45000FC90119712960C91129713969C90862F20
:10D4600090E0AD85BE85A80FB91FAA0FBB1FAA0FFC
:10D47000BB1FAF58BD4F8C9011967C9011971296A0
:10D480006C90129713965C90610F70E0AD85BE852D
:10D49000A60FB71FAA0FBB1FAA0FBB1FAF58BD4FC8
:10D4A0004C9011963C90119712961C9112971396DE
:10D4B0002C90E80FF91FEE0FFF1FEE0FFF1FEF5824
:10D4C000FD4FB081B98321812A8332813B838381DF
:10D4D0008C83FA01E60FF71FEE0FFF1FEE0FFF1F01
:10D4E000EF58FD4F90819D83A181AE83B281BF83B0
:10D4F000238128879701402F592DB701802F992D1F
:10D500000E9493E9882321F0E12CF12C00E0912C7A
:10D510009501A601B501C6010E9493E9882319F07F
:10D520005701C02ED92C242D332D412F522D642D7F
:10D53000732D812F922D0E9493E9882321F0412C95
:10D54000312C10E0212C282D372D462D552D682DFE
:10D55000772D862D952D0E9493E9882321F0842C28
:10D56000732C612E522C2D813E814F8158856D8107
:10D570007E818F8198850E9493E9882321F01D8206
:10D580001E821F82188629813A814B815C816981C4
:10D590007A818B819C810E9493E9882341F03D81AF
:10D5A00039834E814A835F815B8388858C8385E0E4
:10D5B000EB85FC858E9FD0018F9FB00D11242985AE
:10D5C0003A85A20FB31FAA0FBB1FAA0FBB1FAF58EC
:10D5D000BD4FBA87A9879501A601B501C6010E9472
:10D5E00092E79701402F592D0E9491E76B017C0132
:10D5F000282D372D462D552D682D772D862D952DCF
:10D600000E9492E7242D332D412F522D0E9491E745
:10D610009B01AC01C701B6010E9492E76B017C013E
:10D6200029813A814B815C8169817A818B819C81DE
:10D630000E9492E72D813E814F8158850E9491E79B
:10D640009B01AC01C701B6010E9492E720E030E0E7
:10D6500040E450E40E9415E8A985BA856D937D9356
:10D660008D939C9313972E960FB6F894DEBF0FBE42
:10D67000CDBFDF91CF911F910F91FF90EF90DF9081
:10D68000CF90BF90AF909F908F907F906F905F9062
:10D690004F903F902F900895AF92BF92CF92DF921C
:10D6A000EF92FF920F931F93CF93DF936B01E901EA
:10D6B0004A3009F4B8C0453109F06AC0DB0112965E
:10D6C000ED91FC91F280C681D781139A88E28A9508
:10D6D0000000E9F7BF2CB29420EFB22230E1A32E74
:10D6E000AF0C48E2E42E88EF0E94E6688E2D8A9502
:10D6F0000000E9F7BFE1BF1508F481C08F2D8077E6
:10D7000080680E94E6688B2D0E94E6688E2D8A95BF
:10D710000000E9F780E80E94E66880E00E94E66881
:10D720008E2D8A950000E9F78AEF0E94E6688E2D1B
:10D730008A950000E9F78E01005F1F4F8881807F86
:10D740000E94E66889918295807F0E94E668C017F2
:10D75000D107A1F78E2D8A950000E9F7F394E0E157
:10D76000BE0EFA10C0CF1398D6011296CD91DC915F
:10D77000CE010E9489C28111EEC1DF91CF911F912C
:10D780000F91FF90EF90DF90CF90BF90AF900895F2
:10D79000FB0102811381423309F498C108F49CC152
:10D7A000463409F489C1473409F48CC14B3329F557
:10D7B00089812B81D80112966C91129713964C9106
:10D7C000213009F4DFC1233009F0A9C138EF380F47
:10D7D000582F91E0431708F490E041E0531708F008
:10D7E00040E031E0561708F430E0592F542B352330
:10D7F00009F0BDC1942309F0BAC181E0BECF80EE2B
:10D800008F0D8068807F0E94E6688F2D8295807FD3
:10D810000E94E6688E2D8A950000E9F780E80E9454
:10D82000E66880E87BCF0B9A1398399A4198099A59
:10D83000119A139A88E28A950000E9F788E790E048
:10D84000CEE9DFE0FE013197F1F70197D9F788EFD4
:10D850000E94E66818E2812F8A950000E9F780E2CD
:10D860000E94E66880E00E94E668812F8A950000A9
:10D87000E9F780E00E94E66880E80E94E668812F70
:10D880008A950000E9F780E00E94E66880E10E9446
:10D89000E668812F8A950000E9F7CE010197F1F73C
:10D8A000CE010197F1F7CE010197F1F7CE01019773
:10D8B000F1F7CE010197F1F7CE010197F1F7CE0113
:10D8C0000197F1F7CE010197F1F7CE010197F1F73A
:10D8D000CE010197F1F7CE010197F1F7CE01019743
:10D8E000F1F7CE010197F1F7CE010197F1F72197FA
:10D8F000F1F780E20E94E66880E40E94E668812FEA
:10D900008A950000E9F780E20E94E66880E60E94BE
:10D91000E6681A950000E9F710E0D0E0C8E28D2F24
:10D92000807780680E94E668812F0E94E6688C2FCD
:10D930008A950000E9F780E80E94E66880E00E948E
:10D94000E6688C2F8A950000E9F78AEF0E94E66866
:10D950008C2F8A950000E9F780E211980000000002
:10D96000419800000000119A00000000119800008A
:10D970000000419800000000119A0000000011987A
:10D9800000000000419800000000119A0000000013
:10D99000119800000000419800000000119A00005A
:10D9A0000000119800000000419800000000119A4A
:10D9B00000000000119800000000419800000000E5
:10D9C000119A00000000119800000000419800002A
:10D9D0000000119A0000000011980000000041981A
:10D9E00000000000119A00000000119800000000E3
:10D9F000419800000000119A0000000011980000FA
:10DA00000000419800000000119A000000001198E9
:10DA100000000000419800000000119A0000000082
:10DA2000119800000000419800000000119A0000C9
:10DA30000000119800000000419800000000119AB9
:10DA40000000000011980000000041980000000054
:10DA5000119A000000001198000000004198000099
:10DA60000000119A00000000119800000000419889
:10DA700000000000119A000000009C2F9A95000001
:10DA8000E9F7815009F069CF88EF0E94E6688C2F92
:10DA90008A950000E9F7DF5F105FD03209F03FCFD1
:10DAA00080E00E94E66880EC0E94E668CA9500006B
:10DAB000E9F7139881E061CED80115968C9188839F
:10DAC00081E05BCEF80181818883FACFB901C8017A
:10DAD0000E94A6C281E051CE443171F0473109F075
:10DAE0008CCE1882F80182818983858181508A8356
:10DAF00083818B8381E041CED80115964C91159797
:10DB000050E0440F551F70E060E016968D919C9197
:10DB10000E94BDE9C8010E949FC281E02ECE481735
:10DB200008F46BCE861708F468CEFA80E12CD12C6D
:10DB3000243070F41DC0BE01C8010E94A6C28981B4
:10DB400098819D0D98838E0D8983FF0C09F455CE25
:10DB5000F7FEF6CFF0CF4D8150E0440F551F70E037
:10DB600060E08E819F810E94BDE981E006CEFA804F
:10DB700030E0F901E151FE4FD08025513E4FF901CF
:10DB8000E080E6CF58E0580F382F23CEEF92FF9277
:10DB90000F931F93CF93DF93EC018B017A018A855A
:10DBA0009B858617970731F0888199810E9463C60B
:10DBB0001B870A87B701888199810E949ABD2E81AF
:10DBC0003F81820F932F911D9F838E8390E080E091
:10DBD000DF91CF911F910F91FF90EF9008959F9249
:10DBE000AF92BF92CF92DF92EF92FF920F931F936B
:10DBF000CF93DF93EC018B01942EA52E8A859B8514
:10DC00008617970731F0888199810E9463C61B8728
:10DC10000A8788859985019649F5BC800A818E819D
:10DC2000080FC880D980D6015596ED91FC91C601A8
:10DC30000995B80EE92CFA2C10E0F70121917F012B
:10DC4000211127C08E819F81810F911D9F838E831B
:10DC500090E080E0DF91CF911F910F91FF90EF90C6
:10DC6000DF90CF90BF90AF909F9008950E811F815D
:10DC7000692D7A2D888199810E949ABD800F912FFC
:10DC8000911D288539852817390738F681E090E0FD
:10DC9000E1CF4B2D602FC6010E94BBC6080F180FA5
:10DCA000CCCFDF92EF92FF920F931F93CF93DF932E
:10DCB000EC01D62E1CAD0BAD7C0184E0E80EF11C0E
:10DCC000E98DFA8DC7010995412F480F2D2D602F41
:10DCD000C7010E94BBC69BAD890F8BAF81E090E06E
:10DCE000DF91CF911F910F91FF90EF90DF900895FA
:10DCF000EF92FF920F931F93CF937C0100916F05DA
:10DD000010917005C0E0F701EC0FF11D60816623F2
:10DD100051F0062E000C770BC8010E94E2E9892B16
:10DD200049F4CF5FF0CF80E0CF911F910F91FF902A
:10DD3000EF90089581E0F8CF682F880F770B8091DE
:10DD40006F05909170050E94E2E9FC0181E0309737
:10DD500009F480E0309781F0918120ED290F2A307D
:10DD600030F09E3251F4928190539A3098F431966B
:10DD7000F0936705E093660508959D3211F09B329C
:10DD800049F4928120ED290F2A3088F39E3211F454
:10DD90009381EACFF0E0E0E0EBCF0E949C6E882315
:10DDA00041F081E02091660530916705232B09F44D
:10DDB00080E00895CF93DF9300D000D0CDB7DEB7D9
:10DDC00080E090E0A0EAB0E489839A83AB83BC83CF
:10DDD00061E0CE0101960E94CA350F900F900F901E
:10DDE0000F90DF91CF91089580916605909167051E
:10DDF000009731F04AE050E070E060E00C94BDDE46
:10DE000060E070E0CB010895809166059091670510
:10DE1000009731F04AE050E070E060E00C948FDD54
:10DE200060E070E0CB0108950E94046F97FD0CC084
:10DE30000E94046F6F3F71058105910509F034F46C
:10DE40000E94046F862F089580E008958FEF089553
:10DE5000CF93C62F0E94CD6E882319F0CF910C94DA
:10DE6000146F8C2FCF91089580916605909167056E
:10DE7000892B41F00E94146F91E0811101C090E064
:10DE8000892F089591E0FCCFCF93DF93C82FD62F31
:10DE90000E94CD6E882321F0DF91CF910C94346FD6
:10DEA0008C2F0E949C6E811101C08D2FDF91CF912C
:10DEB00008950E94046FCB010895CF93DF93EB0187
:10DEC0000E94CD6E882321F0DF91CF910C94596F81
:10DED000CE01DF91CF9108950F931F93CF9380913F
:10DEE0006605909167050097E9F0FC018F01C191EB
:10DEF0002C2F2F7D81F0C53411F0C536B9F7F8010C
:10DF0000108270E060E00E9431DCF801C083CF91A4
:10DF10001F910F91089570E060E0CF911F910F91D4
:10DF20000C9431DC60E070E0CB01F1CFCF92DF9256
:10DF3000EF92FF926A017B010E94CD6E882331F03F
:10DF4000FF90EF90DF90CF900C946C6FC701B601FB
:10DF5000FF90EF90DF90CF9008959CE0899F802DF7
:10DF6000112491E0980F909375052CE0280F2093D1
:10DF7000410630E02E5F3F4F4091041642171306D2
:10DF800019F014F080E00895209106169217D0F74A
:10DF9000662341F08E5F0E9408C4809141068E5F27
:10DFA0000E9408C48091410690910416891750F38D
:10DFB0002091061690917505291720F310920716E7
:10DFC0008093081681E0089520917405022E000CBC
:10DFD000330B8217130641F08093740564EA7CE1E9
:10DFE00080ED95E10C9463C60895CF92DF92EF9295
:10DFF000FF920F931F93CF93DF93CDB7DEB72C978C
:10E000000FB6F894DEBF0FBECDBF6F3F710581051F
:10E01000910509F0D0F48CEC95E10E94516EE091ED
:10E02000D415F091D5153196849190E02C960FB6C9
:10E03000F894DEBF0FBECDBFDF91CF911F910F913E
:10E04000FF90EF90DF90CF900895F0900716E0904A
:10E0500008162091400221110FC044E85CE16E2DAA
:10E060008F2D0E9427C790E080E0F80EF0920716EF
:10E07000E09208169927DACFC090D415D090D51524
:10E0800020ED35E13A8329832F2D30E03C832B832B
:10E090002E2D30E03E832D8318861F822FEF3FEF19
:10E0A0003A8729871C861B860FEE1DE69E012F5F8F
:10E0B0003F4FAB01BC01C6010E9463B5B60180EDC4
:10E0C00095E10E9463C68F819885CFCFCF92DF9272
:10E0D000EF92FF920F931F93CF93DF93CDB7DEB7ED
:10E0E0002C970FB6F894DEBF0FBECDBFF090071689
:10E0F000E09008162091400221111DC044E65CE129
:10E100006E2D8F2D0E9427C790E080E0F80EF092D0
:10E110000716E092081699272C960FB6F894DEBFE2
:10E120000FBECDBFDF91CF911F910F91FF90EF9068
:10E13000DF90CF900895C090D415D090D51520EDE4
:10E1400035E13A8329832F2D30E03C832B832E2D1C
:10E1500030E03E832D8318861F827A8769871C866C
:10E160001B860FEE1DE69E012F5F3F4F40EC57E1EF
:10E17000BC01C6010E9427B6B60180ED95E10E9460
:10E1800063C68F819885C2CF6FEF7FEF0C94667066
:10E19000CF92DF92EF92FF920F931F93CF93DF9373
:10E1A000CDB7DEB72C970FB6F894DEBF0FBECDBF4C
:10E1B000F0900716E09008162091400221111DC032
:10E1C00044E45CE16E2D8F2D0E9427C790E080E033
:10E1D000F80EF0920716E092081699272C960FB6C3
:10E1E000F894DEBF0FBECDBFDF91CF911F910F918D
:10E1F000FF90EF90DF90CF900895C090D415D0900D
:10E20000D51520ED35E13A8329832F2D30E03C836D
:10E210002B832E2D30E03E832D8318861F827A8734
:10E2200069871C861B860FEE1DE69E012F5F3F4F00
:10E2300043EC57E1BC01C6010E9427B6B60180ED50
:10E2400095E10E9463C68F819885C2CF6FEF7FEF03
:10E250000C94C870AF92BF92CF92DF92EF92FF9270
:10E260000F931F93CF93DF935C016B010E940662B3
:10E27000E82EC6010E941262F12C03E110E0081B97
:10E280001109C5E20E151F050CF4CFE18C2F90E0AB
:10E290009C012E5F3F4F409104164217130609F070
:10E2A000CCF5099720910616281719069CF1409184
:10E2B0004306509144066091420610920716C0939F
:10E2C000081625E1C5010E942668D1E0C114D104D9
:10E2D000B1F06AE370E080E090E00E94F56F0E1507
:10E2E0001F05D4F4C45F80910416C81740F0209134
:10E2F00006164C2F4950550B241715067CF4DF9158
:10E30000CF911F910F91FF90EF90DF90CF90BF9032
:10E31000AF900895D0E0DACFDD2389F3802F880F06
:10E32000080F000F00930716C093081660E270E014
:10E3300080E090E00E94F56FC601DF91CF911F91C0
:10E340000F91FF90EF90DF90CF90BF90AF900C9423
:10E3500026718F929F92AF92BF92CF92DF92EF92EF
:10E36000FF920F931F93CF93DF93CDB7DEB72C9718
:10E370000FB6F894DEBF0FBECDBF982F862F5A017F
:10E380007901D02E692F0E94AD6F882309F489C0CE
:10E39000C701002391F10E940662C82E8090D41517
:10E3A0009090D51580914002811145C01FEF23E167
:10E3B0002C19409143065091440660914206C501D4
:10E3C0000E942668CC2009F46CC0B6E08B9F5001F7
:10E3D00011246AE370E080E090E00E94F56F57E05E
:10E3E000A516B10408F444C060E270E080E090E05B
:10E3F0000E94F56FA81AB90AF2CF0E941262C82EC5
:10E400008090D4159090D51580914002882371F2A8
:10E41000FE0133968AE0DF011D928A95E9F780EDCF
:10E4200095E19A83898306EC1DE69E012F5F3F4F9D
:10E4300043EC57E112C0FE0133968AE0DF011D92E2
:10E440008A95E9F780ED95E19A83898306EC1DE6CC
:10E450009E012F5F3F4F40EC57E1B701C4010E947E
:10E4600027B6B40180ED95E10E9463C61F819FCF5E
:10E4700040914106212F30E0A6E0CA9EC001112440
:10E480002E5F3F4F281739070CF49C0180E8821B50
:10E490008093071640930816C701DD20A9F00E945B
:10E4A000C4702C960FB6F894DEBF0FBECDBFDF91BF
:10E4B000CF911F910F91FF90EF90DF90CF90BF9081
:10E4C000AF909F908F9008950E942671EACFECEC58
:10E4D000F5E183AF64AFCA010C9426710F931F93CB
:10E4E000CF9310926E0510926D052FE32093730564
:10E4F00010927205109271059C01F90190812F5FB5
:10E500003F4F9032D1F39E34C9F4818190ED980F42
:10E510009A3020F08D3211F08B3281F432969F01C7
:10E520002F5F3F4F808180538A3008F468C09F017D
:10E530002F5F3F4F8081803209F463C0F0934F0614
:10E54000E0934E068F010F5F1F4FC0816AE270E0BB
:10E55000C8010E94E2E9009731F0FC013197808107
:10E560008032E1F31182CD3429F0C43519F0C7347B
:10E5700009F041C0F80180810F5F1F4F8032D1F355
:10E5800080538A30C0F5C093730530E020E06AE024
:10E59000AF014F5F5F4F629FC001639F900D1124D9
:10E5A0009C01205331098081280F311D87FD3A9548
:10E5B000FA01808180538A3058F33093720520939A
:10E5C0007105CA01FC01019640814032D9F3F093F4
:10E5D0007005E0936F05CD3401F52E31310539F02A
:10E5E00090F42731310519F02C313105B1F4F09355
:10E5F0006E05E0936D05CF911F910F910895F9017C
:10E600008ECFF90194CF2537310538F02737310502
:10E6100070F3203A83E0380751F350E040E0CF0137
:10E6200001966081662309F45AC0613291F4CD34B9
:10E6300081F42032310569F490936E0580936D0565
:10E6400063E270E00E94E2E90097A9F2FC01108207
:10E65000D2CFFC01DF018D91803271F090ED980FE7
:10E660009A3008F18E3251F4918190539A30D8F05B
:10E6700041155105E1F414C0FD01ECCF8D3211F0CC
:10E680008B3259F4918160ED690F6A3060F09E32EF
:10E6900021F4928190539A3030F04115510519F4CC
:10E6A000AF014150510981548A3108F4B8CFDF01DC
:10E6B000FD018D91882309F4B2CF90ED980F9A3027
:10E6C000B8F393ED980F923098F38B3289F3CF0122
:10E6D00001966081603209F0A2CFFC01F8CF50931F
:10E6E0006E0540936D0587CFFC016591759185910D
:10E6F0009491089580914606882319F080E00E9445
:10E70000C94280E008954F925F926F927F928F92FC
:10E710009F92AF92BF92CF92DF92EF92FF92CF93F0
:10E72000DF93CDB7DEB728970FB6F894DEBF0FBEE4
:10E73000CDBF5C01DB01CD90DD90ED90FC90E091D0
:10E74000B315F091B415FE83ED8384819581A68184
:10E75000B78189839A83AB83BC839C01AD01C701D8
:10E76000B6010E9491E72B013C01F5018080918068
:10E77000A280B380AD81BE818D919D910D90BC91A1
:10E78000A02D8D839E83AF83B88727E137EB41EDC2
:10E7900058EBC301B2010E9415E987FDD0C027E004
:10E7A00030E04AE753E4C301B2010E949BE018162F
:10E7B0000CF4C5C02D813E814F815885C501B4013F
:10E7C0000E9491E72B013C0127E137EB41ED58EB2B
:10E7D0000E9415E987FDB3C027E030E04AE753E423
:10E7E000C301B2010E949BE018160CF4A8C020E0FF
:10E7F00030E0A9016D817E818F8198850E9492E72A
:10E800002B013C0120E030E040E450E40E949BE01A
:10E8100087FF05C0412C512C30E4632E762C27E174
:10E8200037EB41ED58E3C301B2010E9491E79B0130
:10E83000AC01C501B4010E9415E987FD80C020E04C
:10E8400030E04AE753E46D817E818F8198850E9494
:10E8500092E72B013C0120E030E043E653E40E94C4
:10E8600015E9181634F4412C512C23E6622E23E4CA
:10E87000722E27E137EB41ED58E3C301B2010E944C
:10E8800092E79B01AC01C501B4010E949BE0181600
:10E890000CF455C020E030E0A90169817A818B81B8
:10E8A0009C810E9492E74B015C0120E030E040E94E
:10E8B00051E40E949BE087FF06C0812C912C90E9D7
:10E8C000A92E91E4B92E27E137EB41ED58E3C501BC
:10E8D000B4010E9491E79B01AC01C701B6010E94FF
:10E8E00015E987FD2CC020E030E04AE753E4698158
:10E8F0007A818B819C810E9492E74B015C0120E030
:10E9000030E044E553E40E9415E9181634F4812CF4
:10E91000912C84E5A82E83E4B82E27E137EB41ED56
:10E9200058E3C501B4010E9492E79B01AC01B1E03C
:10E93000B983C701B6010E949BE018160CF4198236
:10E94000898128960FB6F894DEBF0FBECDBFDF9148
:10E95000CF91FF90EF90DF90CF90BF90AF909F90BE
:10E960008F907F906F905F904F9008954F925F923D
:10E970006F927F928F929F92AF92BF92CF92DF92CF
:10E98000EF92FF920F931F93CF93DF93EC012091AF
:10E99000D5023091D6024091D7025091D8026881B9
:10E9A00079818A819B810E9491E76B017C01209192
:10E9B000D9023091DA024091DB025091DC026C8185
:10E9C0007D818E819F810E9491E74B015C01A701AF
:10E9D00096016091420170914301809144019091B0
:10E9E00045010E949BE0882309F450C0C092420177
:10E9F000D0924301E0924401F092450120915E05DE
:10EA000030915F054091600550916105C701B601E5
:10EA10000E9401E12B013C010E94BDE86B017C01D9
:10EA200020E030E0A9010E949BE087FD70C020E05B
:10EA300030E040E450E4C701B6010E9415E9181621
:10EA40002CF4C12CD12CC0E4EC2EFE2CA701960195
:10EA5000C301B2010E9491E7609356057093570578
:10EA60008093580590935905C701B6010E9487E825
:10EA700060935405062E000C770B6F5F7F4F643058
:10EA8000710514F064E070E060935205D09140018C
:10EA900010915405A50194016091460170914701C0
:10EAA00080914801909149010E949BE0811133C0FF
:10EAB000D11381C020913A0530913B0540913C052E
:10EAC00050913D056091560570915705809158050C
:10EAD000909159050E9401E120913E0530913F053A
:10EAE00040914005509141050E9492E7DF91CF91FE
:10EAF0001F910F91FF90EF90DF90CF90BF90AF905C
:10EB00009F908F907F906F905F904F900895C12C51
:10EB1000D12C76019BCF8092460190924701A09222
:10EB20004801B092490120916205309163054091FE
:10EB3000640550916505C501B4010E9401E14B01D6
:10EB40005C010E94BDE86B017C0120E030E0A9017E
:10EB50000E949BE087FDF3C020E030E040E450E4F9
:10EB6000C701B6010E9415E918162CF4C12CD12C4E
:10EB7000B0E4EB2EFE2CA7019601C501B4010E9462
:10EB800091E760935A0570935B0580935C059093C1
:10EB90005D05C701B6010E9487E860935505062E02
:10EBA000000C770B6F5F7F4F6430710514F064E0E9
:10EBB00070E060935305C0915505D11305C0809155
:10EBC00041018C1709F470C080915405909155054E
:10EBD00090934101809340010C2E000CDD0B25E049
:10EBE0001203C0011124FC01EC0FFD1FEE0FFF1FEB
:10EBF000EE0FFF1FEF58FD4F20813181428153817D
:10EC000020934E0530934F05409350055093510586
:10EC100000915305002E000C110BFC01E00FF11FB9
:10EC2000EE0FFF1FEE0FFF1FEF58FD4F6081718148
:10EC3000828193810E9491E760934A0570934B050E
:10EC400080934C0590934D052091520535E02303A8
:10EC5000F0011124CE0FDF1FCC0FDD1FCC0FDD1F05
:10EC6000CF58DD4F288139814A815B812093460549
:10EC7000309347054093480550934905E00FF11F35
:10EC8000EE0FFF1FEE0FFF1FEF58FD4F60817181E8
:10EC9000828193810E9491E76093420570934305BE
:10ECA000809344059093450580905A0590905B05AC
:10ECB000A0905C05B0905D0520914A0530914B0510
:10ECC00040914C0550914D05C501B4010E9401E1F0
:10ECD00020914E0530914F054091500550915105BE
:10ECE0000E9492E76B017C01C0923E05D0923F05E5
:10ECF000E0924005F0924105209142053091430594
:10ED00004091440550914505C501B4010E9401E1BF
:10ED1000209146053091470540914805509149059D
:10ED20000E9492E7A70196010E9491E760933A053D
:10ED300070933B0580933C0590933D05BBCEC12C61
:10ED4000D12C760118CF1F93CF93DF93CDB7DEB7C9
:10ED50002C970FB6F894DEBF0FBECDBF182F8823B7
:10ED600079F020E030E0A9016091DD027091DE02CF
:10ED70008091DF029091E0020E949BE08823F9F0ED
:10ED800080916B028117D9F00E947B268CE0EFEC1A
:10ED9000F1E0DE01119601900D928A95E1F7CE0126
:10EDA00001960E94B67480916B02882391F08CE6E4
:10EDB00096E00E94B42610926B020E94A2362C9616
:10EDC0000FB6F894DEBF0FBECDBFDF91CF911F917C
:10EDD000089581E080936B028CE696E00E949C2669
:10EDE000ECCF80E00E94A3761092D9021092DA0252
:10EDF0001092DB021092DC021092D5021092D60221
:10EE00001092D7021092D8021092E1021092E20200
:10EE10001092E3021092E4021092DD021092DE02E0
:10EE20001092DF021092E002E1E7F2E025ED32E01D
:10EE300080E090E0A0ECBFE780839183A283B3835E
:10EE400084839583A683B78380879187A287B387BE
:10EE500084879587A687B787808B918BA28BB38B8E
:10EE600074962E173F0741F708958F929F92AF92A5
:10EE7000BF92CF92DF92EF92FF92C090DD02D090CE
:10EE8000DE02E090DF02F090E00220E030E0A90135
:10EE9000C701B6010E949BE08823E1F1A70196011A
:10EEA00060E070E080E89FE30E9415E86B017C0160
:10EEB0008090E1029090E202A090E302B090E40220
:10EEC00020E030E0A901C501B4010E949BE0882345
:10EED00029F1A501940160E070E080E89FE30E94C1
:10EEE00015E8C0925E05D0925F05E0926005F09251
:10EEF0006105609362057093630580936405909348
:10EF00006505FF90EF90DF90CF90BF90AF909F90FE
:10EF10008F900895C12CD12C7601CACF60E070E0AB
:10EF2000CB01DFCFEFE6F0E080818260808308953F
:10EF300080914B0690914C06892B79F480914B0679
:10EF400090914C06892B49F420914B0630914C0648
:10EF500081E0232B19F480E0089581E00895CF9299
:10EF6000DF92EF92FF926B017C0183E3C816D1041C
:10EF7000E104F10470F082E3C81AD108E108F10855
:10EF800062E370E080E090E00E9403C10E94A4363A
:10EF9000ECCFC701B6010E9403C1FF90EF90DF9054
:10EFA000CF900C94A4365E9A809145068E7F809314
:10EFB00045065E9A809145068D7F80934506159A99
:10EFC000809145068B7F809345065E9A08959091C7
:10EFD000241793FB882780F993FF06C081E0909166
:10EFE0001F15911101C080E008950E94E7778823E2
:10EFF00039F08091241782FB882780F991E08927D6
:10F00000089581E00895DC01EC918E2F90E0FC01E1
:10F01000EE0FFF1FE80FF91FE158FA4E80818F773E
:10F02000808308951092900082E080939100109266
:10F03000950010929400C19AE1E7F0E0808182602F
:10F04000808308957F928F929F92AF92BF92CF92CA
:10F05000DF92EF92FF920F931F93CF93DF93EC0118
:10F060007B0188818C3008F0C4C090E0FC01EE0F79
:10F07000FF1FE80FF91FE158FA4E80818F770E9439
:10F080000EB819821A8288812CE0622F0E9446E70E
:10F09000829FB001112430E020E0AB01420F531FEA
:10F0A000FA01EE0FFF1FE40FF51FE158FA4E9081B1
:10F0B00097FD09C02F5F3F4F2C30310571F781114B
:10F0C00002C00E9412787880072D10E06801CC0CF5
:10F0D000DD1CF601E00FF11FE158FA4E80818068D7
:10F0E000808377FC86C080E2E81682E0F8060CF0A8
:10F0F0003FC08A8128E532E0281B310987FD33951E
:10F10000220F331F220F331F032E000C440B550B0D
:10F11000898178E8872E912C881A910887FD93942D
:10F12000880C991C880C991C092C000CAA08BB0897
:10F1300060E070E0CB01F7FC0AC0B701653B7105E8
:10F1400014F064EB70E0072E000C880B990B281963
:10F1500039094A095B090E94D3E624EB30E040E01C
:10F1600050E00E9405E7820E931EA41EB51E740196
:10F170008BE08715D8F0298188E890E0821B9109FF
:10F1800027FD9395880F991F880F991FE816F90698
:10F1900004F502972FB7F894E601C00FD11FC158AC
:10F1A000DA4E880F991F9A8389832FBF62E370E03C
:10F1B00080E090E0DF91CF911F910F91FF90EF9051
:10F1C000DF90CF90BF90AF909F908F907F900C94E6
:10F1D000AF772A8188E592E0821B910927FD9395FC
:10F1E000880F991F880F991FE816F90694F6C70132
:10F1F000D0CFDF91CF911F910F91FF90EF90DF90D3
:10F20000CF90BF90AF909F908F907F900895CF93B5
:10F21000DF93EB01682F70E084EA95E10E94227889
:10F22000688179818A819B81643F21E07207810531
:10F23000910520F464EF71E080E090E00E94AF77E8
:10F2400086B182958170DF91CF910895CF93DF933E
:10F2500000D000D0CDB7DEB78EEE92E0A0E0B0E0F7
:10F2600089839A83AB83BC83BE016F5F7F4F8AE53E
:10F270000E9407790F900F900F900F90DF91CF9120
:10F280000895CF93DF9300D000D0CDB7DEB78EEED8
:10F2900092E0A0E0B0E089839A83AB83BC83BE0197
:10F2A0006F5F7F4F8AE00E9407790F900F900F9059
:10F2B0000F90DF91CF910895CF93DF9300D000D0CE
:10F2C000CDB7DEB784EF91E0A0E0B0E089839A8308
:10F2D000AB83BC83BE016F5F7F4F8CE30E940779D5
:10F2E0000F900F900F900F90DF91CF910895CF93D3
:10F2F000DF9300D000D0CDB7DEB784EF91E0A0E07F
:10F30000B0E089839A83AB83BC83BE016F5F7F4F7C
:10F3100080EA0E9407790F900F900F900F90DF9175
:10F32000CF9108951F920F920FB60F9211240BB632
:10F330000F922F933F934F935F936F937F938F938E
:10F340009F93AF93BF93EF93FF938091270587FF20
:10F3500027C01092950010929400809127058F5F2E
:10F360008093270580912705082E000C990B20918A
:10F37000A3152817190629F024F0809127058C3051
:10F38000DCF18091940090919500049680349C4922
:10F3900008F47DC08091940090919500049679C006
:10F3A00080912705082E000C990B2091A315281792
:10F3B000190699F294F2E09127058E2FEE0F990B22
:10F3C000FC01EE0FFF1FE80FF91FE158FA4E808194
:10F3D00087FFC3CFE09127058E2FEE0F990BFC011D
:10F3E000EE0FFF1FE80FF91FE158FA4E808160E031
:10F3F0008F770E94A7C0B1CF2091940030919500E3
:10F40000E09127058E2FEE0F990BFC01EE0FFF1FE9
:10F41000E80FF91FE158FA4E81819281820F931F04
:10F420009093990080939800E09127058E2FEE0F1E
:10F43000990BFC01EE0FFF1FE80FF91FE158FA4E80
:10F44000808187FF11C0E09127058E2FEE0F990B69
:10F45000FC01EE0FFF1FE80FF91FE158FA4E808103
:10F4600061E08F770E94A7C0FF91EF91BF91AF91AC
:10F470009F918F917F916F915F914F913F912F91CC
:10F480000F900BBE0F900FBE0F901F90189580E449
:10F490009CE990939900809398008FEF80932705C3
:10F4A000E3CF9091C00095FFFCCF8093C6000895F4
:10F4B000CF93DF93EC018991882319F00E94517A50
:10F4C000FACF8DE00E94517A8AE0DF91CF910C94BF
:10F4D000517ACF93DF93EC01FE018491219688232A
:10F4E00019F00E94517AF8CFDF91CF910895E09101
:10F4F0009B0C81E6E89FF0011124E350F34F8081DB
:10F50000811107C08AEC94E20E94697A8AE00C9427
:10F51000517A0895AF92BF92CF92DF92EF92FF920D
:10F520000F931F93CF93DF938BE194E10E94697A4D
:10F53000C0E0D7E0D15021F080E20E94517AFACFAA
:10F540008C2F0E94B5C7CF5FC53099F78AE00E9423
:10F55000517A01E712E0C0E080E20E94517A8C2FDC
:10F560000E94B5C75801D5E080E20E94517AF501AA
:10F57000C080D180E280F380A7019601C701B60167
:10F580000E9493E9882369F180E20E94517A8DE319
:10F590000E94517A8DE30E94517A8DE30E94517A44
:10F5A0008DE30E94517A8DE30E94517AD150F4E1AB
:10F5B000AF0EB11CD111D8CF8AE00E94517ACF5F33
:10F5C0000C5F1F4FC53041F68AE0DF91CF911F914C
:10F5D0000F91FF90EF90DF90CF90BF90AF900C9481
:10F5E000517A20E030E0A901C701B6010E9415E977
:10F5F00087FD03C08BE20E94517A43E0C701B60148
:10F600000E944C22D3CFCF92DF92EF92FF926A01F9
:10F610007B010E94697A42E0C701B601FF90EF903A
:10F62000DF90CF900C944C22CF93DF93EB010E949C
:10F63000697ACE01DF91CF910C9404B784E194E113
:10F640000C94697A8EE094E10C94697ACF9384E506
:10F650000E94CD6EC0E08823D9F00E94146FC82F9D
:10F660001816B4F40E94227B8DE40E94517A809196
:10F670007105909172050E94BCC76C2FCC0F770B5F
:10F680008AE995E10E94147B8AE00E94517ACFEFCB
:10F690008C2FCF9108952F923F924F925F926F924D
:10F6A0007F928F929F92AF92BF92CF92DF92EF9212
:10F6B000FF920F931F93CF93DF93CDB7DEB766977B
:10F6C0000FB6F894DEBF0FBECDBF83E50E949C6EDF
:10F6D0008A83882309F4FCC00E94346F8983809058
:10F6E0006C0690906D06A0906E06B0906F064090EC
:10F6F000700650907106609072067090730680914B
:10F70000740690917506A0917606B0917706898B64
:10F710009A8BAB8BBC8B9A81992331F0A981A11173
:10F7200003C080E00E94A37686E50E949C6E8A87D3
:10F7300020E030E0A9016091DD027091DE0280914D
:10F74000DF029091E0020E949BE0882309F4C3C08D
:10F7500083E40E949C6E882309F4A3C00E946C6F0E
:10F760006D877E878F87988BE1E7F2E0FD83EC83DE
:10F77000FB83EA8305E0312C212C18EC92EC9E8B64
:10F780001E821F82A8ECA887B2E4B987EA81FB81B8
:10F79000FC87EB87F5E0FD8BAB85BC85CD90DD90DC
:10F7A000ED90FD90BC87AB872E813F8148855985C0
:10F7B000C701B6010E949BE087FF04C0CE82DF82B2
:10F7C000E886F986232D322D412F5E89C701B601C7
:10F7D0000E9415E9181624F43C2C2D2C1E2DFE8AAF
:10F7E000BD89B150BD8BB111D7CF0150EA81FB81EA
:10F7F0007496FB83EA830111C9CF232D322D412F4B
:10F800005E896E817F81888599850E9492E720E0DC
:10F8100030E040E05FE30E9401E12D853E854F85A9
:10F8200058890E9492E76B017C012DEB37E346E893
:10F8300055EB0E9415E987FD0AC02DEB37E346E83A
:10F8400055E3C701B6010E949BE0181654F580E00D
:10F850000E94A37695E0392E8C819D819B838A83BB
:10F8600085E0282EAA81BB816D917D918D919D911E
:10F87000BB83AA838D0104501109A70196010E9440
:10F8800091E7F80160837183828393832A94211026
:10F89000E9CF3A948C819D8144969D838C8331106D
:10F8A000DBCFBA85BB2381F020E030E0A901609175
:10F8B000DD027091DE028091DF029091E0020E94F1
:10F8C0009BE081110E948A7A89810E94A3760FC0F1
:10F8D00080916B0203CF9981911103C0AA85AA235D
:10F8E00099F30E94227B8BED94E10E94697AE98171
:10F8F000EE2351F080916B02811106C00E941E7BA5
:10F900008CEB94E10E94697A0E94227B8EEA94E15A
:10F910000E94697A80916B0281114DC08DEA98E155
:10F920000E94697A8AE00E94517AA501940160914F
:10F930006C0670916D0680916E0690916F060E9424
:10F940009BE081111EC0A30192016091700670912D
:10F95000710680917206909173060E949BE081115E
:10F9600010C029893A894B895C896091740670912D
:10F97000750680917606909177060E949BE0882319
:10F98000E9F066960FB6F894DEBF0FBECDBFDF91EB
:10F99000CF911F910F91FF90EF90DF90CF90BF908C
:10F9A000AF909F908F907F906F905F904F903F901F
:10F9B0002F900C942D3D81EB98E1B2CF66960FB657
:10F9C000F894DEBF0FBECDBFDF91CF911F910F9195
:10F9D000FF90EF90DF90CF90BF90AF909F908F906F
:10F9E0007F906F905F904F903F902F9008950E946E
:10F9F0009D230E94D5458091F9058130A1F40E9494
:10FA00001E7B87E993E10E94697A60E08DE893E1CB
:10FA10000E945C576EE571E080E090E00E94AF7755
:10FA200088E08093F9050895CF92DF92EF92FF92DC
:10FA30001F93CF93DF9300D000D0CDB7DEB78EEE0B
:10FA4000C82E82E0D82EE12CF12CC982DA82EB821A
:10FA5000FC82BE016F5F7F4F8AE50E9407798111AA
:10FA60000EC010E0812F0F900F900F900F90DF913C
:10FA7000CF911F91FF90EF90DF90CF9008950E945B
:10FA80007779C982DA82EB82FC82BE016F5F7F4F99
:10FA90008AE50E940779182F882319F30E941E7B9C
:10FAA00081E794E10E94697A0E94F77CDBCFCF92D4
:10FAB000DF92EF92FF921F93CF93DF9300D000D09D
:10FAC000CDB7DEB78EEEC82E82E0D82EE12CF12C19
:10FAD000C982DA82EB82FC82BE016F5F7F4F8AE0CF
:10FAE0000E94077981110EC010E0812F0F900F90B6
:10FAF0000F900F90DF91CF911F91FF90EF90DF90CB
:10FB0000CF9008950E9477790E9426790E944179CA
:10FB10000E942679C982DA82EB82FC82BE016F5F85
:10FB20007F4F8AE00E940779182F8823E9F20E940C
:10FB30001E7B84E394E10E94697A0E94F77CD5CF12
:10FB4000EC018B01F42E0E949D230E941E7B8DE60A
:10FB500093E10E94697A0115110511F40EE415E292
:10FB6000209711F4C4E6D3E10E947E611F930F93A6
:10FB7000DF93CF9384E593E19F938F93D1E0DF935D
:10FB80000E9443570E942B46C091D115C695C69539
:10FB90008DB79EB707960FB6F8949EBF0FBE8DBF68
:10FBA00080910916811104C0D09309160E94E7C202
:10FBB0008091D2159091D3150E94C0C2DC2FDD0F29
:10FBC0001D2F1C0F83E00E94E46F48EC52E16C2F64
:10FBD00080E00E94677210920716D093081685E4A1
:10FBE00093E10E94C470109207161093081688E3E0
:10FBF00093E10E94C47080ED95E10E9431C68111AD
:10FC0000E1CF8BE593E10E9454B589EE93E030E6B5
:10FC1000019729F0232F2A950000E9F7F9CFF894EE
:10FC200089EE93E038EE019729F0232F2A95000002
:10FC3000E9F7F9CF0E949D23FF2021F00E94D3779E
:10FC4000A895FECF5E9AFCCF8091B10B9091B20B3C
:10FC50002FEF3FEF981751F0E92FF0E0EF54F44FFA
:10FC6000228130E09F5F9F779093B20BC901089586
:10FC70001F920F920FB60F9211240F900FBE0F908C
:10FC80001F9018951F920F920FB60F9211240BB66A
:10FC90000F922F933F934F935F938F939F93EF9385
:10FCA000FF938091C6004091B20B9091B10B31E06F
:10FCB000390F3F77209126052C3008F072C0E22FD3
:10FCC000F0E0EB59F1480C9488E7717E987EA77EAE
:10FCD000B27EB97ED17EBD7ED17EC17EC57ED17E13
:10FCE000C97E803229F0E8F48A3011F08D30F1F4C9
:10FCF000431731F0E92FF0E0EF54F44F8283932F54
:10FD00009093B10BFF91EF919F918F915F914F91E4
:10FD10003F912F910F900BBE0F900FBE0F901F9031
:10FD200018958D3481F021E08E3471F02BE00CC0F9
:10FD30008A3338F48033E0F68032D1F28D32B1F775
:10FD4000D7CF8D3499F722E020932605D1CF813388
:10FD500029F0843329F0803249F7CACF23E0F4CF69
:10FD600028E0F2CF24E0803379F326E0813361F399
:10FD7000DDCF25E08833D1F6E7CF27E08233B1F637
:10FD8000E3CF29E0813391F6DFCF2AE0803371F6AB
:10FD9000DBCF8A3019F08D3009F0AACF10922605FA
:10FDA000A7CF8A3019F08D3009F0A2CF50910A16F2
:10FDB0005523A1F3273049F02A3059F0253071F747
:10FDC00010925A0110924502E9CF21E02093E702F8
:10FDD000E5CF21E02093E602E1CF8EBD0DB407FE12
:10FDE000FDCF08958FEF8EBD0DB407FEFDCF8EB50C
:10FDF0000895909164009B7F90936400982F906A7F
:10FE000096959CBD80FD03C091E0863009F490E09A
:10FE10009DBD0895CF92DF92EF92FF92CF936B0139
:10FE20007C01C42F4A3069F4F7FE0BC0F094E094D3
:10FE3000D094C094C11CD11CE11CF11C8DE20E9425
:10FE4000517A4C2FC701B601CF91FF90EF90DF9010
:10FE5000CF900C944EC7CF92DF92EF92FF926A013F
:10FE60007B010E94697A4AE0C701B601FF90EF90DA
:10FE7000DF90CF900C940A7F2F923F924F925F9227
:10FE80006F927F928F929F92AF92BF92CF92DF92AA
:10FE9000EF92FF920F931F93CF93DF93CDB7DEB70F
:10FEA000EB970FB6F894DEBF0FBECDBF70E060E0F9
:10FEB00085E40E945D6F811171C283E50E94CD6E61
:10FEC000882309F458C00E94596F9A83898365E09A
:10FED00070E083E40E945D6FB82E60E085E50E94CB
:10FEE000446F8FAB60E087E39CE10E945C574981DF
:10FEF0005A81BA01550F880B990B0E94A2E06D83BD
:10FF00007E831C010E949EC16B877C878D879E87A4
:10FF100060915801709159016F507109072E000CC2
:10FF2000880B990B0E94A2E09B01AC016D817E8140
:10FF3000C1010E9415E918161CF588EE9BE10E948C
:10FF4000697AEB960FB6F894DEBF0FBECDBFDF9196
:10FF5000CF911F910F91FF90EF90DF90CF90BF90C6
:10FF6000AF909F908F907F906F905F904F903F9059
:10FF70002F900C94EBB924EB30E03A832983A7CF80
:10FF80008B859C85AD85BE85805B9C43AF4FBF4F05
:10FF90008BAB9CABADABBEAB84ED9BE10E94697AB1
:10FFA0000E949D238FE780930D1581E080935A0175
:10FFB0004B845C846D847E844AA65BA66CA67DA679
:10FFC0001C8E1D8E1E8E1F8E18A219A21AA21BA295
:10FFD00019821A821B821C822FE730E040E050E039
:10FFE0002F87388B498B5A8B1F8230E43D8B4CE135
:10FFF0004E8B56E45F8B188E198E1A8E1B8EFFE780
:020000021000EC
:10000000CF2ED12CE12CF12C1EA61FA618AA19AABE
:100010001AAA1DA21EA21FA218A68CA31C8A1B8AA4
:1000200000E010E01AAE1BAEAB2DBB0CBB0BB9AFA2
:10003000A8AF80915A01882309F485C00E949EC10F
:100040004B015C01B091E802B9A7BB2309F467C07A
:100050000E944A246091091570910A15072E000C20
:10006000880B990B0E94A2E08B018AAF9BAF288D71
:10007000398D4A8D5B8D0E9415E9181634F4088F6E
:10008000198F2AAD2A8F3BAD3B8F2F813D894E8939
:100090005F89B8018AAD9BAD0E949BE087FF06C0D7
:1000A0000F831D8B4AAD4E8B5BAD5F8B8CA198018E
:1000B0004AAD5BAD6D817E81882309F48BC1C1019E
:1000C0000E949BE087FF2BC0B501A401441955098C
:1000D00066097709DB01CA0188589341A109B10972
:1000E000B7FD1DC08F859889A989BA898C199D098A
:1000F000AE09BF09B595A7959795879580930D157E
:100100004DA35EA36FA378A79D81988FAE81A98F21
:100110002A8E3B8E8B869C86AD86BE861CA220E0F6
:1001200030E040EF51E46D817E81C1010E9492E791
:1001300098014AAD5BAD0E949BE087FF22C081E63B
:100140009BE10E94697A10925A010E949D23F9CE88
:100150004BEEC42ED12CE12CF12C8EC184E190E029
:10016000A0E0B0E08F87988BA98BBA8B34E1C32EC7
:10017000D12CE12CF12C8EC1CF86D88AE98AFA8A5B
:1001800089C1D501C4012AA53BA54CA55DA5821B4B
:10019000930BA40BB50BB7FD48C080E00E94F02282
:1001A0008AE00E94517AD501C4018053984FAF4F25
:1001B000BF4F8AA79BA7ACA7BDA79EA5911163C0FF
:1001C0002FA538A949A95AA9B8018AAD9BAD0E94AB
:1001D00015E918160CF043C020E030E040E050E490
:1001E000B8018AAD9BAD0E9492E76FA778AB89AB4F
:1001F0009AABA5019401205B3C434F4F5F4F2BAB63
:100200003CAB4DAB5EAB20E030E040EC50E46D81A8
:100210007E81C1010E9491E798014AAD5BAD0E94C9
:100220009BE0881F8827881F8EA78B859C85AD85BE
:10023000BE85481659066A067B0610F4D301C20132
:10024000881A990AAA0ABB0A31E883163FE4930682
:1002500032E1A306B10470F183E49BE172CFD501D2
:10026000C4012BA93CA94DA95EA9821B930BA40B29
:10027000B50B44E250E163E370E1B7FDD6CF80E017
:100280000E946224D2CF20E030E040EF51E46D8143
:100290007E81C1010E9491E79B01AC01B8018AAD4A
:1002A0009BAD0E949BE087FFC0CF40ED50E160EE28
:1002B00070E1E5CF48AD59AD8B899C894817590746
:1002C0000CF069C003970CF466C086EE9AE10E94B8
:1002D000697A89EC9AE10E94697A49815A816B8135
:1002E0007C8182EE9AE10E94037B8AE00E94517A2F
:1002F00089EC9AE10E94697A48A159A16AA17BA17F
:100300008EED9AE10E94037B8AE00E94517A89EC8B
:100310009AE10E94697A4C8D5D8D6E8D7F8D8AED9C
:100320009AE10E94037B8AE00E94517A9FA9992357
:1003300009F407CE29813A814B815C8120930E1507
:1003400030930F1540931015509311152CEA35EC8E
:1003500047E25EE368A179A18AA19BA10E9401E125
:1003600060931215709313158093141590931515BF
:100370002CEA35EC47E25EE36C8D7D8D8E8D9F8D92
:100380000E9415E860931615709317158093181541
:1003900090931915D6CD0E94E25E4BCE83E19CE18D
:1003A000EB960FB6F894DEBF0FBECDBFDF91CF91B5
:1003B0001F910F91FF90EF90DF90CF90BF90AF9083
:1003C0009F908F907F906F905F904F903F902F9075
:1003D0000C94697AC1010E9415E918160CF09FCEA1
:1003E000D501C4012B853C854D855E85821B930B11
:1003F000A40BB50BAC01BD0148585341610971090B
:1004000077FD8DCE4B895C89452B09F4FEC04DA04C
:100410005EA06FA078A4480E591E6A1E7B1E2DA1F7
:100420003EA14FA158A5281B390B4A0B5B0BC701F6
:10043000B6010E94D3E6A30192010E9405E7CF8492
:10044000D888E988FA88C20ED31EE41EF51E54E14E
:10045000C516D104E104F1040CF480CE8CEEC8166C
:10046000D104E104F1040CF073CE90E8C916D10474
:10047000E104F1040CF480CECF86D88AE98AFA8AA6
:100480002EEF30E040E050E02C193D094E095F09A5
:1004900069017A014F85588969897A898CEC9BE1D9
:1004A0000E942B7FB701A60187EC9BE10E942B7F66
:1004B0004F815D896E897F8980EC9BE10E94037B7F
:1004C000488D598D6A8D7B8D89EB9BE10E94037B62
:1004D000AB89BC8913970CF498C0C701B6010E9480
:1004E000A2E020E030E040E850E40E9401E16983AE
:1004F0007A838B839C832F813D894E895F89688DA8
:10050000798D8A8D9B8D0E9491E72BED3FE049E428
:1005100050E40E9401E120E030E040E05FE30E940F
:1005200001E19B01AC0169817A818B819C810E94F0
:1005300015E86F83788789879A87C301B2010E9483
:10054000A2E02FE632E143E85AE30E9401E12B01E9
:100550003C012AE939E949E15FE36F8178858985C2
:100560009A850E9401E169837A838B839C839B0136
:10057000AC010E9492E7A30192010E9415E868A3D2
:1005800079A38AA39BA329813A814B815C81C30112
:10059000B2010E9401E120E030E040E05EE30E9411
:1005A00001E16C8F7D8F8E8F9F8F4F81588569857C
:1005B0007A8583EB9BE10E94037BB301A2018DEA64
:1005C0009BE10E94037B8AE00E94517A8EE99BE1C5
:1005D0000E94697A49815A816B817C8188E99BE11B
:1005E0000E94037B48A159A16AA17BA182E99BE1FA
:1005F0000E94037B4C8D5D8D6E8D7F8D8CE89BE121
:100600000E94037B8AE00E94517A8F859889A9898C
:10061000BA898C0D9D1DAE1DBF1DB595A7959795EB
:10062000879580930D152B893C892F5F3F4F3C8B1D
:100630002B8B3D813F834E814D8B2E8A3F8A240137
:10064000350159A55CA36BCDCF93DF93EB010E94DD
:10065000697ACE01DF91CF910C94D8CB4F925F9203
:100660006F927F928F929F92AF92BF92CF92DF92C2
:10067000EF92FF920F931F93CF93DF9300D01F92BF
:10068000CDB7DEB780919A0C803108F0C7C131E652
:10069000E32E80919A0C803108F0F8C08091B10B64
:1006A0009091B20B891B8F7709F4F0C00E94247ED1
:1006B00097FF0BC00E941E7B82E093E10E94697A43
:1006C0008091B10B8093B20BE4CF8A3019F08D305A
:1006D00009F0D3C01092990C8091370C9091380C8E
:1006E000FC01ED5CF34F1682892B19F40E94A436AD
:1006F000D0CF1092380C1092370C09E31CE0F801AF
:100700008191803209F446C08E3409F0A1C06DEFAA
:1007100072E1C8010E9418E06C01892B41F06EE47F
:1007200070E0C80104960E94E2E9009709F4C8014C
:100730004AE050E070E060E001960E948FDD4B01DE
:100740005C018091330C9091340CA091350CB091E8
:10075000360C0196A11DB11D88169906AA06BB0686
:1007600029F060E08AEC92E1CD2851F16AE270E074
:10077000C8010E9411EA9C01009729F1982F901B53
:10078000F12C992349F09150F801E90FF11D808176
:10079000F826F7CF8F01B3CF4AE050E070E060E079
:1007A000C90101960E948FDD4F2C512C712C612CB8
:1007B000641575058605970551F060E08BEA92E1B6
:1007C0000E9484B866CF60E081E892E1F9CF809220
:1007D000330C9092340CA092350CB092360C809170
:1007E000F9058130E1F067E470E0C8010E94E2E9B8
:1007F0000097A9F04AE050E070E060E001960E94A6
:100800008FDD623071058105910548F480EE91E13C
:100810000E94697A60E086ED91E10E945C578091C8
:10082000390C8B3309F435CF80919A0C803108F064
:1008300030CF80919C0C8E9DC001112469E37CE037
:100840008356934F0E94EDE980E00E9450B821CF7B
:100850008091241780FFC3CF67EF74E2C8010E9424
:1008600018E0009731F0FC01838180538A3008F052
:10087000B6CF60E087E592E1A3CF27E33CE049E310
:100880005CE069E97CE00E944E6903CF8091241707
:1008900082FFC4C01A82198281E6F82E90E1B92E37
:1008A00029E6A22E80919A0C803108F0B7C00E94F0
:1008B00086698111B3C041E050E0BE016D5F7F4F9A
:1008C0008CE195E10E945BCD0B8110E0019711F066
:1008D0000FEF1FEF8091241590912515A0912615FB
:1008E000B09127158093201790932117A09322177A
:1008F000B09323170E9486690F3F100749F48111B6
:1009000007C00E941E7B8AE193E10E94697ACACFE8
:1009100040919C0C242F30E00A3061F00D3051F0F2
:10092000882309F46DC089819A81009719F0019696
:100930009A8389831092340589819A81F29EF0010D
:10094000F39EF00D1124E656F34FDF01A80FB91FF7
:1009500013961C92892BB9F50E94A4360E948669D1
:10096000882309F49FCF0E947B268CE195E10E94A9
:10097000231E80911B178823F1F1815080931B1750
:100980008A9DC001112462E086589A4F0E9492CF3E
:10099000E0911B1724E0E29FF0011124EA58FA4F7E
:1009A00040815181628173814093201750932117B8
:1009B00060932217709323178CE195E10E9433CC4A
:1009C0000E94D1C76FCF1A82198283818D3479F446
:1009D0008481823361F48581853349F48681805333
:1009E0008A3028F0809124178B7F8093241781E030
:1009F0000E9450B8B3CF0E94C2C7B092F90552CF3F
:100A00004F9DA00111244356534F9E012F5F3F4F2E
:100A100064E375E0802F0E944E6944CF0E949EC11E
:100A20004B015C018091680590916905A0916A0570
:100A3000B0916B050097A105B10551F140914706B2
:100A4000509148066091490670914A06840F951F9F
:100A5000A61FB71FA5019401281B390B4A0B5B0B7E
:100A6000DA01C901B7FD14C00E941E7B60914E06D9
:100A700070914F0689E991E10E9424838AE00E94E7
:100A8000517A40E070E060E090E080E00E94A07D5C
:100A900080914A0190914B01A0914C01B0914D0180
:100AA000892B8A2B8B2B79F09091B8158091B915F1
:100AB000981709F4FCC08092470690924806A092CD
:100AC0004906B0924A060E949EC16B017C0180914A
:100AD0004502811108C02091B8159091B91581E0A7
:100AE000291301C080E02091091530910A1591E089
:100AF00089272A3A31050CF480E091E040913005D5
:100B0000509131056091320570913305452B462B8C
:100B1000472B09F490E0981789F0882309F401C164
:100B2000D701C60180569444A24FBF4F8093300531
:100B300090933105A0933205B09333054090780629
:100B40005090790660907A0670907B0620912C0573
:100B500030912D0540912E0550912F05C301B20112
:100B60000E949BE0882319F1809130059091310516
:100B7000A0913205B091330540922C0550922D057D
:100B800060922E0570922F05892B8A2B8B2B09F4EE
:100B900049C0D701C60180569444A24FBF4F8093ED
:100BA000300590933105A0933205B09333058091C1
:100BB000300590913105A0913205B0913305009731
:100BC000A105B10579F1C81AD90AEA0AFB0AF7FCAE
:100BD00029C0109230051092310510923205109202
:100BE000330584E891E10E94697A60E080E791E151
:100BF0000E945C5780910B1590910C1518161906E0
:100C000024F490E080E00E94EA45809104069091EF
:100C100005061816190634F41092050610920406FB
:100C20000E94C6178091350590913605A091370531
:100C3000B0913805A5019401281B390B4A0B5B0BB9
:100C4000DA01C901B7FD8FC09091B8158091B9152F
:100C5000F090A406981749F0E091B9153BE4E39FA2
:100C6000F0011124E250F94FF0800E949EC1FF2054
:100C700009F4CFC0009128051091290520912A057B
:100C800030912B05011511052105310509F04DC0E5
:100C90006C597F4F8F4F9F4F6093280570932905A4
:100CA00080932A0590932B05FF24FA9444C00E9458
:100CB0009EC1009147061091480620914906309147
:100CC0004A06C0904A01D0904B01E0904C01F09050
:100CD0004D010C0D1D1D2E1D3F1D601B710B820B48
:100CE000930B97FF03C010923905EDCE8091390523
:100CF0008111E9CE81E0809339055E9A80914506A5
:100D00008E7F809345065E9A809145068D7F809305
:100D10004506159A809145068B7F809345065E9A1D
:100D2000D2CE80E090E0DC0101CF601B710B820B22
:100D3000930B97FDB9CF0F2D10E084E00E940EB801
:100D4000F11070C060E084E00E94A7C044E6840E09
:100D5000911CA11CB11C8092350590923605A09281
:100D60003705B09238050E94A4368091F905882392
:100D7000E1F110913F011130B1F1809124178062AF
:100D80008093241781E080933F0164EF71E080E05D
:100D900090E00E94AF770E94F3D18091241783FFE7
:100DA000A3C0123028F460E089E293E10E945C570E
:100DB00001E083E080935B010E949EC16C597F4FEC
:100DC0008F4F9F4F60934102709342028093430282
:100DD00090934402002339F0123029F481E080938B
:100DE0001A170E944ED20E94E25E0F900F900F9051
:100DF000DF91CF911F910F91FF90EF90DF90CF90F7
:100E0000BF90AF909F908F907F906F905F904F902A
:100E10000895109228051092290510922A05109223
:100E20002B0589CF0F3F110511F461E08CCFE2E370
:100E3000F5E2E491E150EA3008F051C0F0E0ED5DF8
:100E4000F8470C9488E72D873287378741876F876B
:100E50006F874B8753875B87658784B5806884BDC0
:100E6000F7BC74CF84B5806284BDF8BC6FCF80912D
:100E70008000806880938000109389000093880030
:100E800065CF8091800080628093800010938B00FA
:100E900000938A005BCF8091B00080688093B0009F
:100EA000F092B30053CF8091B00080628093B00085
:100EB000F092B4004BCF80919000806880939000B6
:100EC000109399000093980041CF80919000806228
:100ED0008093900010939B0000939A0037CF0038C6
:100EE00011050CF0A2CF2ECF00E0112309F47BCF27
:100EF00060CF2F923F924F925F926F927F928F922C
:100F00009F92AF92BF92CF92DF92EF92FF920F9398
:100F10001F93CF93DF93CDB7DEB763970FB6F894E7
:100F2000DEBF0FBECDBF8091680B83FD9FC189E4FA
:100F30000E94CD6E882309F48BC10E94146F90E04B
:100F40001816190614F481E090E026E0289FF001BD
:100F5000299FF00D1124E95FF94F828193811A8254
:100F60008C38910514F08CE890E0909305068093FE
:100F700004060E94C6172091040630910506809150
:100F8000020690910306821793070CF422C18BEAA4
:100F90009AE160E00E945C5781E080935A011B82D5
:100FA0001C821D821E8219861A861B861C861E863E
:100FB0002CE32F873CE1388B46E4498B312C212CE4
:100FC00050E859838FEB8A8B1B8A91E09D87812C97
:100FD000912C54010091040610910506B801012ED0
:100FE000000C880B990B0E94A2E06B017C01232D61
:100FF000322D49815A890E949BE0882389F0809193
:10100000020690910306AA81A111E6C0B1E0BB8B54
:10101000081719070CF01B8A3C2C2D2CE982FA8A40
:101020000E949EC16B017C01DC01CB0129853A85C0
:101030004B855C85821B930BA40BB50BB7FD2FC0B2
:10104000D701C60188519C4FAF4FBF4F89879A8700
:10105000AB87BC8780E00E94F02287EA9AE10E9479
:10106000697A81149104A104B10409F4DFC0C501B7
:10107000B40168577C4E8F4F9F4F6C197D098E09C4
:101080009F0928EE33E040E050E00E94E3E6CA0109
:10109000B9014AE00E940A7F8AE00E94517A0E94C8
:1010A0002E830E949EC160934706709348068093EA
:1010B000490690934A066091020670910306072E36
:1010C000000C880B990B0E94A2E06F8378878C013B
:1010D0009B01AC01632D722D89819A890E9491E751
:1010E0002B013C0120E030E0A9010E9415E987FFB7
:1010F00004C077FA709477F8709481149104A10475
:10110000B10409F097C020E030E040E85FE3C3019C
:10111000B2010E949BE087FF10C09D85812C912C1D
:101120005401992331F082E8882E86E0982EA12C74
:10113000B12C8C0C9D1CAE1CBF1CAB89AA2391F159
:101140002B813C814D815E81211531054105510581
:1011500041F0D701C601821B930BA40BB50BB7FD61
:1011600021C02F813885A8016E857F85888999895E
:101170000E9491E720E030E040E85FE30E949BE0BE
:1011800087FD2DC0D701C601805A9541AF4FBF4F93
:101190008B839C83AD83BE839F819E87A885AF8709
:1011A000088B198B80915A018823C9F0811491040E
:1011B000A104B10461F0B8E8CB1AB3E1DB0AE1089D
:1011C000F108C818D908EA08FB08F7FE08C01D8610
:1011D00001CF8AEB9AE1DDCE081719070CF5809153
:1011E0005A01882309F442C010925A0163960FB63F
:1011F000F894DEBF0FBECDBFDF91CF911F910F914D
:10120000FF90EF90DF90CF90BF90AF909F908F9026
:101210007F906F905F904F903F902F900C94EBB920
:101220003C2C2D2CE982FA8A1B8AFACE8FE30E948D
:10123000517A32CF20E030E040E450E4C301B20103
:101240000E9415E918160CF078CF4601570175CFAA
:1012500083E50E94CD6E8A83811105C082E50E94DC
:10126000CD6E882319F00E94596F7ACE63960FB61F
:10127000F894DEBF0FBECDBFDF91CF911F910F91CC
:10128000FF90EF90DF90CF90BF90AF909F908F90A6
:101290007F906F905F904F903F902F9008952F9286
:1012A0003F924F925F926F927F928F929F92AF92F6
:1012B000BF92CF92DF92EF92FF920F931F93CF9343
:1012C000DF93CDB7DEB764970FB6F894DEBF0FBEDD
:1012D000CDBF8091680B83FDB0C10E94267B8987BA
:1012E00087FDABC189E40E94CD6E882309F497C1C4
:1012F0000E94146F90E01816190614F481E090E033
:1013000026E0289FF001299FF00D1124E95FF94F95
:10131000808191811B8A0E94EA4520910B153091B2
:101320000C158091091590910A15821793078CF47A
:1013300087E99AE19F938F9382EA9AE19F938F9333
:101340001F920E9443570F900F900F900F900F9095
:1013500005C02B898CE89AE1222361F381E0809318
:101360005A011C821D821E821F821A861B861C86C1
:101370001D861F862CE3288B3CE1398B46E44A8B83
:10138000212C312C50E85A838FEB8B83198291E00A
:101390009E87812C912C540101C01E8600910B1553
:1013A00010910C15B801012E000C880B990B0E94AE
:1013B000A2E0D62EE72EF82E988791014A815B8114
:1013C0000E949BE0882391F08091091590910A1565
:1013D0003B893111E7C041E04983081719070CF038
:1013E00019822D2C3E2CFA8258855B830E949EC167
:1013F0006B017C01DC01CB012A853B854C855D8539
:10140000821B930BA40BB50BB7FD2FC0D701C601F0
:1014100088519C4FAF4FBF4F8A879B87AC87BD8752
:1014200089850E94F02288E89AE10E94697A8114F5
:101430009104A104B10409F4E0C0C501B4016053F2
:10144000784F8F4F9F4F6C197D098E099F0928EEA9
:1014500033E040E050E00E94E3E6CA01B9014AE00F
:101460000E940A7F8AE00E94517A0E942E830E9485
:101470009EC16093470670934806809349069093F7
:101480004A066091091570910A15072E000C880B09
:10149000990B0E94A2E06887072F182F9C8B262F9C
:1014A000372F482F592FB1018A819B810E9491E7E4
:1014B0002B013C0120E030E0A9010E9415E987FFE3
:1014C00004C077FA709477F8709481149104A104A1
:1014D000B10409F096C020E030E040E85FE3C301CA
:1014E000B2010E949BE087FF10C09E85812C912C49
:1014F0005401992331F08AE9882E82E0982EA12C9C
:10150000B12C8C0C9D1CAE1CBF1CA981AA2399F187
:101510002C813D814E815F812115310541055105A9
:1015200041F0D701C601821B930BA40BB50BB7FD8D
:1015300022C02885302F412F5C896F857889898961
:101540009A890E9491E720E030E040EC5FE30E943E
:101550009BE087FD2AC0D701C601805A9541AF4F55
:10156000BF4F8C839D83AE83BF8398859F87088BF5
:10157000198BAC89AA8B80915A018823B1F0811410
:101580009104A104B10409F408CFB0EDCB1AB7E07F
:10159000DB0AE108F108C818D908EA08FB08F7FCDB
:1015A000FCCE03C0081719070CF580915A01882357
:1015B00009F443C010925A0164960FB6F894DEBF46
:1015C0000FBECDBFDF91CF911F910F91FF90EF9094
:1015D000DF90CF90BF90AF909F908F907F906F9053
:1015E0005F904F903F902F900C94EBB92D2C3E2C98
:1015F000FA8288858B831982F9CE8FE30E94517A13
:1016000031CF20E030E040E450E4C301B2010E9459
:1016100015E918160CF079CF4601570176CF83E50E
:101620000E94CD6E8B8B811105C082E50E94CD6E2C
:10163000882319F00E94596F6ECE64960FB6F89405
:10164000DEBF0FBECDBFDF91CF911F910F91FF90F5
:10165000EF90DF90CF90BF90AF909F908F907F9052
:101660006F905F904F903F902F9008952F923F92F0
:101670004F925F926F927F928F929F92AF92BF92A2
:10168000CF92DF92EF92FF920F931F93CF93DF934E
:10169000CDB7DEB7ED970FB6F894DEBF0FBECDBF66
:1016A00080916B02888B87E50E949C6E882309F4E9
:1016B0001BC120E030E0A9016091DD027091DE02E3
:1016C0008091DF029091E0020E949BE0811107C0AF
:1016D0000E941E7B88E895E10E94697A18C18AE51C
:1016E0000E94CD6E882339F10E946C6F20916606AE
:1016F0003091670640916806509169060E9491E713
:101700006B017C0120E030E040E251ECC701B60102
:101710000E9415E987FD0AC020E030E040E251E474
:10172000C701B6010E949BE0181674F40E941E7B4C
:101730008BE795E1D1CFC0907406D0907506E0900C
:101740007606F0907706DECF40E050E060EC7FE771
:1017500088E50E94966F20915E0630915F06409169
:101760006006509161060E9491E72B013C0140E028
:1017700050E060EC7FE789E50E94966F2091620659
:101780003091630640916406509165060E9491E78E
:101790004B015C016FEF89E40E94286F182F6FEFF7
:1017A0008AE40E94286F082FA3019201C301B201AD
:1017B0000E9493E981116EC0A5019401C501B40195
:1017C0000E9493E9811166C08BA19CA1ADA1BEA12D
:1017D0008BAB9CABADABBEAB2091D5023091D602AA
:1017E0004091D7025091D802C301B2010E9491E703
:1017F0002B013C0120E030E040E05FE36BA97CA9D5
:101800008DA99EA90E9401E19B01AC01C301B20117
:101810000E9492E72BA93CA94DA95EA90E9415E858
:101820000E9487E8162F4FA058A469A47AA420919B
:10183000D9023091DA024091DB025091DC02C501FD
:10184000B4010E9491E74B015C0120E030E040E0F0
:101850005FE3C301B2010E9401E19B01AC01C5013C
:10186000B4010E9492E7A30192010E9415E80E9430
:1018700087E8062F812F012E000C990B97FD2CC0B5
:10188000059764F5802F002E000C990B97FD28C05A
:10189000059744F51530D8F50530C8F580E00E946D
:1018A000A37695E01902F0011124E00FF11D07FD68
:1018B000FA95EE0FFF1FEE0FFF1FEF58FD4FC0828E
:1018C000D182E282F38288890E94A3768889882364
:1018D000F1F00E942D3D1BC010E0D4CF14E0D2CF18
:1018E00000E0D8CF04E0D6CF8AE40E949C6E81113C
:1018F0000CC070E060E086E50E945D6F9A8389838A
:101900000597F0F086E595E1E7CE0E94F176ED9639
:101910000FB6F894DEBF0FBECDBFDF91CF911F9100
:101920000F91FF90EF90DF90CF90BF90AF909F907E
:101930008F907F906F905F904F903F902F90089581
:1019400060E084E40E94446F8F8740E050E0BA0179
:101950008AE50E94966F6BA77CA78DA79EA740E0A3
:1019600050E86BE376E483E50E94966F20E030E078
:1019700040E752E40E9415E860935C0170935D01BA
:1019800080935E0190935F010091B3151091B4159F
:10199000D801CD90DD90ED90FC9020E030E0A901E1
:1019A000C701B6010E9492E76AAF7BAF8CAF9DAFD3
:1019B00020E030E040E450E40E949BE087FF06C056
:1019C0001AAE1BAEB0E4BCAFE0E4EDAF20E030E017
:1019D0004AE753E4C701B6010E9492E76BAB672E5A
:1019E0008FAB98AF20E030E043E653E40E9415E966
:1019F000181634F41BAA612CF3E6FFAB23E428AFDE
:101A0000D80114968D909D90AD90BC90179720E0D2
:101A100030E0A901C501B4010E9492E77B018C016D
:101A200020E030E040E951E40E949BE087FF04C0E1
:101A3000E12CF12C00E911E420E030E04AE753E426
:101A4000C501B4010E9492E7B62EC72ED82E99AFD9
:101A500020E030E044E553E40E9415E9181634F420
:101A6000B12CC12CF4E5DF2EB3E4B9AF88E40E94B9
:101A70009C6E882309F40DC20E946C6F0E9487E857
:101A80001B0177FF02C06F5F7F4F7595679571955A
:101A9000619571096D587F4F072E000C880B990BCB
:101AA0000E94A2E0762E872E982EA92E9701A801DB
:101AB0000E9415E9181624F4E72CF82C092D1A2D8C
:101AC0002AAD3BAD4CAD5DAD672D782D892D9A2D9E
:101AD0000E9415E9181624F07AAC8BAC9CACADAC26
:101AE000872D982DA92DBA2D8B8B9C8BAD8BBE8B02
:101AF000C701D8018F8B988FA98FBA8FB101330C92
:101B0000880B990B0E94A2E01B012C01AC019B01E8
:101B1000B701C8010E9492E77B018C012B2D3C2D5F
:101B20004D2D59AD0E949BE087FF04C0BE2CCF2CE9
:101B3000D02E19AFA2019101672D782D892D9A2DF4
:101B40000E9492E77B018C012BA9362D4FA958AD3D
:101B50000E949BE087FF04C0EBAA6F2C0FAB18AF6D
:101B60008BA9962DAFA9B8AD8B8F9C8FAD8FBE8FF3
:101B70008B2D9C2DAD2DB9AD8F8F98A3A9A3BAA3A2
:101B8000BE01695E7F4FCE0143960E948373882316
:101B900009F4AEC1BE01615E7F4FCE014B960E943B
:101BA0008373E82E882309F4A3C12F89388D498DCA
:101BB0005A8D6F8D78A189A19AA10E9491E720E0AA
:101BC00030E040E85EE30E9401E14B015C012B89BB
:101BD0003C894D895E896B8D7C8D8D8D9E8D0E949B
:101BE00091E720E030E040E85EE30E9401E16BA372
:101BF0007CA38DA39EA38FA298A6A9A6BAA689812D
:101C00009A811816190674F484E295E10E94697AA3
